:020000040800F2
:100000000050002061280108012901084912010857
:100010000129010801290108012901080000000047
:10002000000000000000000000000000012901089D
:10003000012901080000000001290108E9840008E5
:1000400001290108012901080129010801290108E4
:100050000129010801290108C19C0008BD9C000874
:1000600001290108012901080129010801290108C4
:100070000129010801290108DD9C00080129010866
:10008000DDB9000801290108012901080129010839
:10009000012901080129010801290108B99C00086A
:1000A00001290108A99A000801290108B99A000844
:1000B000999A0008899A0008799A00085351000813
:1000C000575100084D5100085151000801290108FD
:1000D00001290108D19C0008C59C000801290108DC
:1000E000F984000801290108012901080000000025
:1000F0000000000000000000000000000000000000
:0C01000000000000000000005FF808F1A3
:100110002DE9F04F684B694EA1B033600023736046
:100120000FF084FD18B90FF0A3FD07F05FF907F099
:1001300027FA634A634C1378634D43F0010313704D
:100140000023089309930A934FF4E0130B93236859
:10015000A87B43F480332360A36943F01003A361B9
:10016000236803F400330993089B01330893099B28
:100170001BB9089BB3F5A06FF2D12368514913F462
:10018000003301D0022315E00A6842F001020A6040
:100190000893236803F002030993089B0133089333
:1001A000099B1BB9089BB3F5A06FF2D123689A078E
:1001B00039D501230A93454B45491A6842F010028C
:1001C0001A601A6822F003021A601A6842F00202EA
:1001D0001A606368636063686360636843F48063A4
:1001E00063603C4B1A68043B22F070425A603A4A02
:1001F0001160616821F47C116160596841F000412F
:100200005960D96821F40041D9609B681B0449BF3B
:10021000324B4FF4E01313604FF480130B930A9B9F
:10022000012B01D117E0FEE7022B18D168B10B9B1F
:10023000B3F5801F02D14FF4A01305E00B9BB3F57B
:10024000E01F02D14FF400130B930B9963680B432B
:1002500043F4803302E0636843F46013636023680F
:1002600043F0807323602168164B8F01FBD55968DA
:1002700021F003015960596841F002015960636837
:10028000104903F00C03082BF9D14B68DFF85480B8
:1002900003F00C03042B03D0082B03D00C4B29E0F4
:1002A000136827E04B684868C3F38343C00303F136
:1002B000020319D40A4A1CE0FF6B0008A0090020C1
:1002C0007030002000100240CC11002000200240BD
:1002D00000127A00041001402C000020001BB7001F
:1002E00000093D004800002049681268890348BFA2
:1002F00052085343C8F800306368DFF870A3C3F3B3
:10030000031353441A7BD8F80030DFF874B3D3409A
:10031000C8F80030C04B0DF18009CBF80C30A36950
:10032000002743F00103A361636ABC48B360636ABA
:1003300043F080736362A36943F01C03A3614FF62B
:10034000FF7329F82C3D49468DF856700BF03CFCA4
:10035000B34849460BF038FC4946B2480BF034FC30
:10036000B14A4846536843F0007353600DF0E0F81B
:10037000159BAE4A6420B3FBF2F3AD4A1360AD4B5C
:100380004FF47A721F60D8F80030DFF8F882B3FBC0
:10039000F2F3A94A013B5360F0238BF82330072383
:1003A00097601360AB68C8F8003008F06AF8394607
:1003B000A248A02214F021FEE369394643F0070366
:1003C000E361A36943F4006343F00C03A361544663
:1003D0009B4B4FF0000A03F10C0201F802A001311F
:1003E0000E29F5D1FF229A76DA761A775A77954B4D
:1003F000954A51461A6095483022D8F8008014F08A
:10040000FCFD5146C8F380170423914ADFF83CE213
:10041000885C0C224A4302F80E0047B91E380128B6
:100420009FBFFF2003F1FF3302F80E00DBB2013162
:100430000429EAD1874A95F805B01370864B87499D
:1004400083F800B0864B7E4A3362C0330B60854B25
:1004500018F0200F03EBCB035B7818BF0123536226
:10046000002340F2DC51804A22F813100133082B9C
:10047000F7D10EA800211C2214F0BFFD18F4007A59
:100480001DBF7A4BCDF850900393CDF80CA0BBF173
:100490000E0F03D00BF0EF03082B02D101238DF8D0
:1004A0004A30012007F0C2FD18B14088003018BF63
:1004B0000120C8F340038DF83E30C8F340338DF877
:1004C0003830C8F3C03300F001008DF83B3018F429
:1004D00000638DF83D008DF8407004D095F88631AA
:1004E0005F1E7B427B418DF83C30C8F300438DF8A2
:1004F0004130736A1AF1000A18BF4FF0010A003345
:1005000018BF01238DF84330C8F300538DF84430F1
:10051000B5F84A31B5F8480118F4805FADF84830B5
:10052000B5F85631ADF84E0018BF5148ADF8463019
:10053000C8F3804318BFB0F850018DF83F30B5F8CC
:10054000543118BFADF84E00B3F5FA7FADF84C301A
:1005500084BF0023ADF84E3095F8D631454886F873
:100560002830002386F8293043709DF84A3008F07F
:100570000101002BC8F3C0028DF839108DF83A2024
:100580008DF842A00CBF0023022301B902B1013350
:1005900004EB8304E3694FF00008A3F102091A3366
:1005A00005934FF6FF7339F8026F9E4200F09C816D
:1005B0009DF83D20F3B21AB19A1E012A40F29081B3
:1005C0009DF8402032B12C491A0189582B4A91429A
:1005D00000F086819DF8412032B127491A018958DF
:1005E000264A914200F07C819DF83E2052B1224A79
:1005F0000A4802EB03125168814203D11289102A82
:1006000000F06E819DF83B20002A44D01A4A03482E
:1006100002EB031238E000BF0005FA0500080140B4
:10062000000C0140001001400000014040420F005A
:10063000D81A0020DC1A002010E000E0602A002018
:10064000A00900206C280020C01300207028002082
:10065000D2A10108A1110020AC0400207C2B0020B5
:10066000E01100201C9901080C11002008770108F6
:10067000CC110020C9090020849601080004004024
:1006800000ED00E0782E00205168814203D11289EC
:10069000022A00F025819DF83C2052B1B74AB848A3
:1006A00002EB03125168814203D11289022A00F041
:1006B0001781149A7AB1B14C116804EB0314606885
:1006C000884208D121899088884200F00981D28827
:1006D0008A4200F00581360A022E02D19DF83820A8
:1006E00003E0012E04D19DF83920002A00F0F880A3
:1006F000DFF888A29DF844101F010AEB0704524658
:1007000031B19DF84A1019B9043B032B40F2D08057
:10071000012EF0B246D19B4D3A44FF23517B85F820
:10072000703085F87130506802F1080312894FF07B
:10073000000BADF854208DF85610022215A985F84B
:1007400074B0C5F8804004938DF8572085F82CB01C
:10075000C5F830B0C5F834B0C5F838B0C5F86CB0DD
:1007600085F872B085F873B00BF02EFA049B5AF836
:10077000070099785A460BF0DBF820465946324676
:1007800009F0F6F9804BC5F88CB0C5F884307F4B82
:100790002046C5F8883005F1840105F1880209F08A
:1007A0002FFA9DE002284BD15FFA88F34FF01C0C22
:1007B0000CFB03FC714ADFF8CCA1D1194B680692FF
:1007C00001F1080209890AEB0C0692F805E0002500
:1007D0004FF0010B86F87580ADF854108DF8570076
:1007E00015A9184686F8765086F87E5086F874B0BB
:1007F000C6F88040CDF81CC08DF856E004920BF08E
:10080000E3F9049B069A9978D0592A460BF090F8A0
:10081000204629465A4609F0ABF95D4ADDF81CC06E
:10082000C6F88420E2445B4A0AF18401C6F88820B5
:10083000C6F88C5020460A1D09F0E2F9D8444FE072
:10084000032833D19DF83F304E4D534E3BB195F8C0
:100850002A70204608214FF6FF7200231AE0BDF8E7
:100860004C2095F82A70B2F5FA7FBDF84E300BD9BE
:100870004A492046B1FBF2F2082192B20BF098FAF5
:10088000474B46F827000AE046492046B1FBF2F202
:10089000012192B20BF08CFA434B46F82700C3605B
:1008A00095F82A30013385F82A3019E0042817D149
:1008B000BDF846203B4B334D93FBF2F22046BDF88A
:1008C0004830012192B295F829600BF071FA95F841
:1008D000293005EB86060133C6F8540185F8293026
:1008E000059B99457FF45DAE264C304F94F8292046
:1008F000002384F874212E4A3B701678A6F1170263
:10090000022A1AD81D46236A0021585903EB05080C
:1009100010F056FF18B1636A002B51D126E0254B29
:1009200005EB030E98E80F008EE80F003B781035BA
:100930000133C02D3B70E6D1EDE71F4A12F836E0D7
:1009400002EBC602D2F804C087F800E0BCF1000F49
:10095000E1D01D467545DEDA164A2B0103EB02088D
:1009600063440FCB013588E80F00F3E7134B1A6897
:10097000984612F4805F49D142E000BF8496010896
:10098000000C0140A009002021B7000801B80008B0
:100990006DB90008F9B60008302A002000127A006C
:1009A00021B8000840420F0011B800082F2A00208B
:1009B000AC040020E80300201C990108782E0020D8
:1009C000B64BB74A13F8360003EBC6035D681070E8
:1009D000002DCBD000238342C8DAC3EBC3016A18D1
:1009E000D2F80080DFF8F0C2013341F80C8001EB4F
:1009F0000C0E9188AEF8041092798EF80620EAE782
:100A000006F0EF03082BA74B24D125E03B78012B00
:100A1000F6D9A54D05EB031303F110071035BD42C0
:100A2000EED055F8100C4FF07C5110F035FD4FF022
:100A30007C5145F8100C55F8140C10F02DFD4FF0BA
:100A40007C5145F8140C55F80C0C10F025FD45F8B8
:100A50000C0CE3E70E2E08D11A78182E42F0100283
:100A60001A7008D10DF028FE05E01A78192E22F030
:100A700010021A70F5E70DF003FED8F800300120DF
:100A80005E035EBF894B01221A70894A894D137833
:100A90004FF0100A43F00403137004F0A3F8D8F8E1
:100AA0000060284606F4006300215246049314F0C7
:100AB000A4FA022306F4004900271E408DF83630C0
:100AC0008DF837700CD07C480DA9ADF834A00CF02F
:100AD000A3FE04232B70012607236F70AE70EB700A
:100AE000202375480DA9ADF834304FF0010B0CF000
:100AF00093FE4FF007080523DFF8B8A12B72771C8F
:100B00006E7285F80AB085F80B80B9F1000F0FD02E
:100B1000022269480DA9ADF834200CF07DFE8AF858
:100B200005708AF804B08AF806B08AF80780B71C06
:100B3000049B7BB1022361480DA9ADF834300CF061
:100B40006BFE092301222B73AA737B1C07226F7390
:100B5000EA73DFB25A4A5B485368002643F44043C5
:100B600053605369DFF85C8143F00103536193697B
:100B700043F4007393610CF063FC534B012F159306
:100B8000524B15A916930CBF334680231A934FF48A
:100B900080731B934FF480631C9320231D93404666
:100BA0004FF400531E931796189719961F960CF042
:100BB00029FCD8F80030464943F00103C8F800305A
:100BC0004A68012F22F4702294BF0023012322F4EB
:100BD000807242EA03224A608B683E4A1A4042F41D
:100BE000602242F002028A60CB6A23F470027B1E0C
:100BF000DBB242EA0353CB620123AA1991780029A0
:100C00007CD0A85D591C0928C9B2D278DFF8C0E0B1
:100C100011D9A0F10A07DEF80C8007EB47074FF067
:100C2000070C0CFA07FC28EA0C0CBA404CEA02024A
:100C3000CEF80C200EE0DEF8107000EB40084FF00C
:100C4000070C0CFA08FC27EA0C0702FA08F23A43F0
:100C5000CEF81020062B1E4F0ED8013B7A6B03EB0B
:100C600083034FF01F0E0EFA03FE22EA0E0200FA73
:100C700003F313437B6340E00C2B2FD8DA1FD7F824
:100C800030C002EB82021F2393402CEA030E00FACD
:100C900002F34EEA03033B632FE000BF9480010898
:100CA000082B0020C0190020F003002018090020A4
:100CB00070300020CC28002000080140000C0140CA
:100CC00000100240080002404C240140DC280020B3
:100CD00000240140FDF7F1FF092B0020A3F10D02D4
:100CE000D7F82CC002EB82021F2393402CEA030E9C
:100CF00000FA02F34EEA0303FB620B460436102EA1
:100D00007FF47BAF7E4B9A6842F480729A609A6857
:100D100042F001029A609A6842F008029A6099686B
:100D2000774A0D07FBD4936843F004039360744B38
:100D30009A6812F00408FAD19A6842F4A0029A6004
:100D4000704BB3F85C019A46002840F0B287BAF9BC
:100D50005E31002B40F0AD87BAF96031002B40F0D6
:100D6000A887694B00211B680C22B3F856306748EE
:100D7000BAF864519AF863B19AF86B719AF86C6199
:100D80000493BAF80C909AF80FA014F036F9604B5F
:100D9000002118461422059314F02FF95D49002212
:100DA0000A70C4F8782104F0D7F9059B002800F0F8
:100DB0006587594AB5F5807F1A60584A5A60584A83
:100DC000DA60584A1A61584B01D1002216E0BB2D57
:100DD00001D9012212E0612D01D902220EE0292D54
:100DE00001D903220AE0132D01D9042206E0092DBE
:100DF00001D9052202E0002DE7D006221A70012356
:100E00004A4A13704A4A136843F0010313605A4672
:100E1000092A4FF0000101D90A46F9E74FF0010B0A
:100E20000BFA02F313F04D0005D113F46C7357D095
:100E3000404B18704AE03F4BC4F87811197004F029
:100E40008BF9002842D006210A4615AB682004F031
:100E500019F89DF8591001F001029DF8571001F0A2
:100E600001014B0043EA82019DF8552002F0010385
:100E70000B430AD05BB2012B01D1002302E0022B0D
:100E80000ED1012384F87C3111E00DAB68200C21D8
:100E90005A4603F0F7FF9DF8343013F00F0303D1E7
:100EA000032007F0F8FA02E0042BEAD1E5E7174B3C
:100EB000214A1A60214A5A6094F87C21002A0CBF0A
:100EC0006F226E221A72032300F0E1BE0F4B1C4A00
:100ED0001A601C4A5A6000221A72092300F0D7BE19
:100EE000012A9B4693D8134A1370042E00F2018105
:100EF000DFE816F02A0008012A002A00C90000BF16
:100F000000240140CC1100201C110020782C00206E
:100F1000402700206C020020E5500008B54F000873
:100F2000494B000890C1793D140000204400002086
:100F3000BC19002094300020B94B0008F74F00087E
:100F400091D00008ADD0000894F87D31BB4E002B45
:100F500040F0CF86142007F094FA7720D0210122A8
:100F60000DAB03F08FFF002800F08D809DF834302A
:100F70000322552B86F89731A6F8A02140F08380F4
:100F8000D12101220DAB772003F07CFF9DF8343096
:100F9000772003F00F021B0986F8982186F8993113
:100FA000162215ABAA2103F06DFF9DF854209DF881
:100FB000553043EA0223A6F880319DF856209DF86B
:100FC000573043EA0223A6F882319DF858209DF855
:100FD000593043EA0223A6F884319DF85A209DF83F
:100FE0005B3043EA0223A6F886319DF85C209DF829
:100FF0005D3043EA0223A6F888319DF85E209DF813
:101000005F3043EA0223A6F88A319DF860209DF8FC
:10101000613043EA0223A6F88C319DF862209DF8E6
:10102000633043EA0223A6F88E319DF864209DF8D0
:10103000653043EA0223A6F890319DF866209DF8BA
:10104000673043EA0223A6F892319DF868209DF8A4
:10105000693043EA022341F27072A6F89431784B6A
:101060001A8046F678125A80764A5A60764A9A6012
:10107000764ADA60764A1A61764A5A61012386F81E
:101080007D3100F036BE94F8A4B16C4EBBF1000F78
:1010900040F00686142007F0F4F906F2A513762036
:1010A000D021012203F0EEFE96F8A531582B29D16C
:1010B00006F5D47388211822762003F0E3FE31224E
:1010C0007620F42103F0B8FF0123634A86F8A431A7
:1010D0005B4B9A60614AA3F800B05A6045F6D8129B
:1010E0005A805F4ADA605F4A1A615F4A5A6100F0CB
:1010F000D7BD012E06D05D4B5D4A9E70136843F04C
:10110000040313605A4E3368980702D5594B1B6885
:101110009847EDB2584ABAF1000F29D033684DB95B
:1011200040F2596113F0020F40F2712318BF0B46D1
:101130007D2108E0990759BF4FF47A7319464FF49F
:10114000FA634FF47A71994505DBB9F57A6FA8BF58
:101150004FF47A6900E099464B1E4B44B3FBF1F320
:10116000013BDBB203FB011184F8C431116003E0E1
:1011700084F8C4A1C2F80090404D2B689847404ABB
:1011800000231370914617B1022F40F08C854FF069
:10119000000A20AB03F82CAD1E200A210122C4F85E
:1011A000C8A103F06FFE002800F0A6859DF854301A
:1011B000482B0CD1334B344A1A60344A5A602B4BBB
:1011C0000222DA70336843F00803336002E05046CD
:1011D00000F092BD2E4C94F858310BB12D4A13708B
:1011E00094F859310BB12C4A137094F85A310BB161
:1011F00089F800303368DFF8ACB013F0080F53D033
:10120000BDF910A04FF064099AFBF9F7384610F0C9
:10121000EFF8049009FB17A000B210F0E9F81F499D
:1012200010F03AF9049B0146184610F02DF81C49BD
:1012300010F032F9CBF8000039E000BFA00900201F
:1012400000010020DD5000088D4F0008C550000847
:101250004D4F00086D4A0008694A00086B4A0008B3
:10126000BD500008014F0008054800084400002058
:10127000BC190020782C0020A02C00204027002042
:1012800095300020DC00002065C0000845B800084B
:10129000CC1100206C020020943000208988883C0A
:1012A00000002041882B00200023CBF80030A54F00
:1012B0004FF00A093B78049743F002033B70192072
:1012C00007F0DFF809F1FF39192007F0DAF819F013
:1012D000FF09F4D133681B0705D59B4B1B68984762
:1012E0009A4B01221A709A4B9A4F1B68187B10F088
:1012F0007FF8994910F0D0F805F054FF82463888FD
:1013000010F076F8514610F0C7F814F083F8934BBC
:101310001880388810F06CF80146914810F070F988
:10132000904910F06DF9904B8B491860286910F0C6
:10133000B3F88E4910F0B0F88D4D8E4BFF21186038
:101340001B22284613F059FE2846002129703168D7
:10135000894B012211F0020F18BF6A701A701FBF6B
:1013600003221A700222AA704F0741BF1A78551C37
:101370001D70032548BF855411F00A0F0CD01A7850
:1013800004218154511CC9B205254554D11C023297
:101390001970D2B206218154784D29688E0641BF5A
:1013A0001A78561C1E70072648BF86540A0608D5B0
:1013B0001A7809268654961C01321E70D2B20A266B
:1013C00086546679082E01D00E2E08D11A7802F1C3
:1013D000010E83F800E04FF00B0E00F802E01A78DF
:1013E000CF0302F1010E4FF00C0C48BF624F00F822
:1013F00002C05FFA8EFE48BF023283F800E041BFB0
:101400003A705B4A4FF00E0C02F80EC04A0748BF14
:101410001A784FF0120C41BF02F1010E83F800E080
:101420004FF0100E00F802E01A784F0502F1010E9D
:101430005FFA8EFE83F800E000F802C00AD594F847
:1014400018723FB14C4F02323A70494A4FF0130CB8
:1014500002F80EC01A788F0502F1010E4FF0140C3D
:1014600048BF454F00F802C05FFA8EFE48BF023207
:1014700083F800E041BF3A703D4A4FF0150C02F886
:101480000EC0182E13D11A784FF0160E00F802E095
:1014900002F1010E5FFA8EFE4FF0170C00F80EC03D
:1014A00002F1030E0232D2B283F800E086540F0339
:1014B00041BF1A78561C1E70192648BF8654CE05A7
:1014C00041BF1A78511C19701A2348BF8354002158
:1014D00098222B4813F091FD0BF07FFE294A2A4BEE
:1014E000B4F852111A60294BB4F8980119802849B0
:1014F00000230B808B7027490A6081B2264A22F8AC
:1015000013100133122BF9D12B68D9045CBFB4F846
:101510009E1111801B0740F1EA8094F89241062C3D
:1015200000F2DF80DFE804F004073C6782A2A2003B
:1015300045F2F05201E042F6F822184B1A800BF007
:10154000E6FECDE070300020DC000020F40000203A
:10155000F80200201600002035FA8E3C140300200B
:101560000AE81C4100401C4628020020BD37863591
:10157000E5100020F4020020E4100020782E002066
:10158000C827002056130020840F0020880F002059
:10159000483000203C300020702F002054030020F1
:1015A00042F6F8227A4B1A800FF022FF79490FF0A9
:1015B00073FF79490FF066FE10F05AF90023774A5D
:1015C00042F823000133122BF9D1754A75494020A6
:1015D0001160754A137006F003FE002800F0818048
:1015E00001234FF0070990F9000040218DE808021F
:1015F0006E4A6F4B6FE042F6F822654B40201A802E
:101600006C4A674B1A60684B10221A7006F0E8FDAE
:10161000002866D001234FF0000C90F90000402113
:101620008DE80810644A4FF4E13354E042F6F822A2
:10163000574B40201A80614A594B1A605A4B082276
:101640001A7006F0CDFD00284BD001234FF0000E9C
:1016500090F9000040218DE80840594A4FF4E133E9
:1016600006F055FF574BC3F8CC0136E042F6F8229E
:10167000474B0C261A804C4B53485449544A1E7011
:10168000062C4FF00003DFF87CC1524F03700B7043
:10169000137009D01B238CF800304F4B05223E708D
:1016A0001A704FF4E13406E021238CF800304A4BE5
:1016B0003E701C70494C4A4A394B40201A6006F073
:1016C0008FFD70B10123002790F900008DE888009C
:1016D0002346444A402106F01AFF003018BF01207B
:1016E00028B9082005F050FE3F4A2D4B1A602A68A1
:1016F0002D4912F4804F1FBF08230B703B48284B25
:1017000018BF186042F2010313409BB144F62060F9
:101710001F4B9604188041BF08230B703448204BA0
:1017200048BF1860D40741BF0C230B7031481C4BD5
:1017300048BF18600B781006A3F104034B7040F10A
:101740009B8020482C4E0024DFF8BC90C0F8D0616C
:1017500021461522294F00F5EA7089F80140C9F8A1
:101760000440C9F80840053E13F047FC20463E609F
:1017700008F016F8224B02201B68BA46C9F80C3054
:1017800006F02EFD002841D1802005F0FDFD6BE024
:1017900054030020CDCCCC3F0000B044282F0020C3
:1017A00028000020DD0E01086428002085100108B3
:1017B000A0860100C90E0108D90F0108B50E010865
:1017C0008D0F0108A009002038300020A12700203B
:1017D000A027002037300020C427002090D003002D
:1017E00099D00008C9D000083D0F01080D0F01086D
:1017F0002D0F01081D0F0108C013002064020020F6
:101800009C2E0020C327002044020020447999F830
:101810000130BC490C2202FB03125278A24204D0D0
:101820000133DBB2042BF4D9002389F80130DAF854
:10183000003099F801201B7890F90000002B4FF040
:101840000C0303FB021314BF0324012400225B7862
:1018500000940192022106F05AFEAB4B186000285A
:1018600092D0012007F09CFFA84B1868A84B00F508
:10187000C5721A6008F03CF82B6899056CD5A54A2A
:10188000A54C039BA548236093690DA943F0010370
:101890009361039B1B88ADF8343010238DF83630EC
:1018A00002238DF837300AF08FF923689B485B8854
:1018B0000DA9ADF8343004238DF836300AF084F9E0
:1018C00020680F21037A03F0030203F0FC0303F105
:1018D000804303F580339C689200914024EA010123
:1018E00099609968012404FA02F20A439A604368F5
:1018F0008B4AD943536116680E40166056680E40F5
:10190000566016681E43166096680E409660D6684C
:101910003140D160916819439160D1680B43D36025
:10192000437A15A88DF8543003238DF855300023E1
:101930008DF856308DF857400EF0C2FE794B7A4A3A
:101940001B683C3B1360794A136843F01003136033
:10195000774B4FF0FF321A60764B774A774C136023
:10196000774A803313602B680026DA03267040F133
:10197000AA8040F22A3ADFF8F4B1664F0CF0DEFF9D
:101980004FF0010952465846314684F8009013F052
:1019900034FBBB696B4843F00403BB614023ADF8E3
:1019A000303018238DF833300CA903238DF83230F2
:1019B0000BF032FFFB69644943F00203FB61634BA8
:1019C000634C1B68A7F69477B3FBF1F32188013BC6
:1019D00021F45C710904090C21809BB21D21A185B1
:1019E0002385A4F81490238C23F001031B041B0C03
:1019F0002384238CA088218B23F0020321F0730120
:101A000009041B04090C1B0C41F0600180B243EA7D
:101A10000903A0802183A6862384238B23F0080357
:101A20001B041B0C43F008032383B4F844306FEA13
:101A300043436FEA53439BB2A4F84430D7F8A83F1E
:101A400043EA0903C7F8A83F38460BF0F9FC414BBD
:101A5000CDF858B0159380231A934FF480734FF04C
:101A6000100B1B9338464FF4005315A91E9319967B
:101A70001C961D961F96CDF85CB0CDF860A00BF0BB
:101A8000C1FCA3890DA89BB243F40073A3813B68FA
:101A900043F002033B608DF834B08DF835908DF83B
:101AA00036608DF837900EF00BFE2B4B1A682B4BDF
:101AB00043F8282008F10108B8F1200FF5D109F00A
:101AC000A5FF09F0A3FF2B685B0540F19180DFF8CB
:101AD000A090234BD9F814A50420C3F800A006F069
:101AE0007FFB0421C9F8180506F056FB1D4B89F849
:101AF0001C050820C3F800A006F072FB1A4B082151
:101B000038E000BFC4750108201D00201C11002012
:101B1000E00F00200010024040020020000C0140B5
:101B2000000401409C2E00203C020020BC19002033
:101B30003C110020F41300205C1D00201909002036
:101B4000581D00200008014000366E0148000020AA
:101B50000004004034040040347701081A090020D2
:101B6000B0190020081A0020541A0020890B002008
:101B7000A0090020186006F00FFB634C89F81D05D2
:101B8000002120462C2213F038FA8E2363704FF088
:101B90007C08E0237D26E37084F8008084F82B60C5
:101BA0005A4C2C220021204613F027FA8A23637016
:101BB0001020A023E37084F8008084F82B60C9F81B
:101BC00020A506F00DFB1021C9F8240506F0E4FA63
:101BD00089F828052020C9F82CA506F001FB202152
:101BE000C9F8300506F0D8FA89F834050FF04EF838
:101BF0002B68474A13F4002318BF0123137006F023
:101C000019FC444B1860444B5A791946052A02BF07
:101C1000424B4FF4C8721A80414B4FF47A721A80CB
:101C2000404BC8221A80404A137843F008031370CF
:101C30003E4A137823F00203137040F602032A6829
:101C400013406BB13A4A3B4B1A603B4B03221A706C
:101C50003A4B01221A703A4A00231380394A138002
:101C60008B6801222B60384B1A70049B049A1B78F6
:101C700063F07F03137021B0BDE8F08F334A1A6020
:101C8000334A5A60334A9A600823FFF7B9B8324A98
:101C90005370324A136843F002031360FFF725B90B
:101CA0000426FFF728BA012F7FF694AA1F46FFF7F4
:101CB00066BA2B4B00221A7000B20FF099FB29492B
:101CC0000FF0EAFB1590BAF95E010FF091FB254980
:101CD0000FF0E2FB1690BAF960010FF089FB214981
:101CE0000FF0DAFB2049179015A805F065FAFFF709
:101CF00038B80226FFF7FFB9012F7FF66BAA00273D
:101D000089F80000FFF743BAD81900200D1A002007
:101D10009C2C002034030020CC110020960F0020C2
:101D20008E3000208C300020C01900209730002019
:101D300048130020A81900200C1A00203C000020A5
:101D400080100020821000201809002097D0000881
:101D5000BBD0000893D0000844000020BC1900202C
:101D60003000002035FA8E3CA8280020954A2DE945
:101D7000F04F1568944C05F59C43944E2033236036
:101D8000336889B013F4804F059205D10FF042FA01
:101D900010B92379013323718D4A13784BB18D49E2
:101DA00009688D4240F2E58003F1FF3882F8008037
:101DB000DFE09846884B5FFA88F51F78DFF83892A5
:101DC000AF4231D9D9F80030072D98BF595D834B08
:101DD00088BF29461B6880489847032D1ED8D9F82C
:101DE000002005F10E0302EB83039988DA88A8B17D
:101DF0004FF47A73401A5843531A90FBF3F040F6AD
:101E0000C90300F57A70984205DC40F2EE2398424F
:101E1000B8BF184601E040F6CA0080B204EB4505A1
:101E2000E88008F10108C5E794F804800325B8FBB1
:101E3000F5F50F2384F82A3094F82B3005EB45058F
:101E4000019394F82C30C5EB08050393D9F80030C2
:101E5000DFF8ACA10293EBB204930025BD4255DA42
:101E60005F4B4FEA450933F815B0019B53B90FF0AA
:101E7000D1F928B1039B002B08BF4FF0000B01E004
:101E8000DDF804B0029B988A584502D8D88A584594
:101E90000ED2E8B20FF06AF9032D8346DFBF94F843
:101EA0002AE00120A8402EEA0000D8BF84F82A00CA
:101EB0000FF0B0F918B14B4829F800B022E0049BAC
:101EC00094F876002AF813B030B9B8F1020F15D99A
:101ED0003D4B012083F87600BAF80000BAF80230D2
:101EE0000344BAF8040003443F489BB229F8003089
:101EF0001BB2032093FBF0F39BB200E05B46394832
:101F000029F8003001350AF1060AA7E794F82A20DB
:101F10003648A2F10F014A424A4184F89020344BDE
:101F20006AB1344A1268520109D40268D9689A60C9
:101F3000521AC82A1DD9012283F8212019E002680B
:101F40009868DA605B68121A9A4288BF284B4FF093
:101F5000000184F82B1088BF83F821100025BD42B2
:101F600007DAE8B20FF002F91E4B23F8150001352D
:101F7000F5E73368DD0405D51E4B1B68D80701D48F
:101F80000EF06AFB059B1F681B4B1A68907A0028AD
:101F900038D01449137B013831F810001BB1C0F55B
:101FA0003B60083080B200B2A0F57A70B0F57A7F5D
:101FB000A8BF4FF47A7020EAE0700FF019FA0F49C9
:101FC00055E000BF7C300020D80E0020782E002085
:101FD00044300020403000206428002028000020E9
:101FE000DE0E0020702F0020500F00209C2E0020BD
:101FF00048300020E01000203C30002000007A44EF
:10200000060F0020336819043AD5D4F89430934D64
:10201000FB1A002B34DB07F59C432033C5F89430C2
:102020008F4BD27A59798F4B33F8113095F898103D
:102030009BB293FBF2F3013101F00F0285F8982077
:102040002A4482F899300346874A825C013013445F
:1020500010289BB2F8D11BB293FBF0F000B26428B9
:10206000A8BF642020EAE0700FF0C2F97F490FF0AA
:10207000C7FA7F490FF010FA0FF0FAFB7D4B18807A
:1020800033687D4D13F4807F00F00F817B4BDFF8C8
:10209000F0919F4205D999F8022012B9012289F8DE
:1020A000022099F80220002A00F0FF80744A95F877
:1020B000008092F82170C8F380087A1E5742574179
:1020C000704A002F9246116818BF4FF0000BC1F301
:1020D0008063019308BF4FF0030B99F82020052A75
:1020E00000F2DD80DFE802F0034E537988A5B8F1F5
:1020F000000F3AD0D4F8AC00B4F8B01006F00DF9E7
:10210000012809D16049614A09681268C9886420B8
:1021100000FB0122C9F81020019B6BB15A4A1268DA
:1021200012794AB10AF080FF032289F820204FF487
:102130007A72C9F81C20D0E7002F40F0B080534AD3
:10214000D9F8101010684E4A88420AD902920AF053
:102150006BFF029A032182F8201040F6B831D1615A
:10216000BBE7012182F82010B7E7019B4FF48060A4
:1021700013B105F0F9F801E005F0E5F80022C9F81F
:1021800010208CE0002F49D10AF04EFFA5E727B1BF
:10219000052289F82020012000E03846B8F1000F20
:1021A0000CD0D4F8AC204FF0020BD189384A118002
:1021B00051809180344909684988D180334A116837
:1021C000D9F81420914202D8B8F1000F64D147F237
:1021D0003052C9F81C20032221E02A7842F0020282
:1021E0002A700EF039FA294AD9F81C1012680A44EC
:1021F000C9F81820042212E0244A9FB11168D9F8C6
:10220000182091424BD9234A12781AB9DAF80020E3
:10221000D30744D42A7822F002022A70052289F8D2
:1022200020205AE71268D9F81C100A44C9F818206F
:1022300035E01549154A09681268C988642000FB11
:1022400001224FF48060C9F81020002289F8202074
:1022500089F8032005F077F83FE700BFD80E00208B
:10226000CC280020DC280020710F00200000C8428C
:1022700000C07F444011002097300020404B4C00AC
:1022800048300020E0100020782700209C2E0020FD
:10229000702F00201500002000287FF41EAFBBF136
:1022A000000F02D0584606F08BF8934F07F5C57023
:1022B000B7F8521106F031F80197834668B90AF071
:1022C000A5FE8E4B0022C3F800B0C3F804B0C3F8DB
:1022D00008B08B4B1A605A609A602B785F0736D52E
:1022E0003368D80633D5874B1B78D9062FD4864B55
:1022F0001B789BB1019B93F8E231BBF1000F15D124
:102300007BB1824B1A68D4F8B4309B1A002B08DAE0
:102310000EF0A2F97E4B83F8B8B018E0BBF1000FC5
:102320000DD1102006F04CF801230EE03BB1774AA6
:102330004FF47A71126801FB0323C4F8B43094F8A7
:10234000B83023B106F02CF8002384F8B830019B94
:1023500093F8E0A193F8E111B3F89AE1B3F89CC1C6
:10236000002318466B4F800837F91320013372455C
:10237000C4BF60F07F00C0B26245B8BF40F040000B
:10238000042BB946EED194F8B930614A834205D1A5
:1023900092F8BA30F92B04D8013300E0002382F818
:1023A000BA30594B84F8B9001A785B4F9846E2B9B5
:1023B0003B68DA0708D5BBF1000F16D12B78DB0795
:1023C00013D50DF0A5FF10E02B7858070DD5504B15
:1023D00093F82B304BB1514BDB7833B911B10EF080
:1023E0003BF902E0BBF1000FF9D094F8BA30484A4B
:1023F000142BDFF83CB140F0AD8098F800301AF1B2
:10240000000A18BF4FF0010A6BB392F8B9305F2B86
:1024100011D12B7803F0040303F0FF0113B10EF088
:102420001BF908E00B200391029205F0C9FF029A04
:10243000039982F8BA10BAF1000F14D094F8B930A9
:102440007D2B10D12B7803F0040303F0FF0213B1AE
:102450000EF002F907E00B20029205F0B1FF2C4BC1
:10246000029A83F8BA202B7803F0040303F0FF01EB
:10247000002B6FD194F8B930254A572B15D1284B32
:102480004FF47A721A803368190601D507F080FA82
:10249000244B1B685A0742BF234A0A21118013F0BC
:1024A000080357D1214A138054E03068400717D5FC
:1024B0005A2B15D192F8BB302BB1012382F8BB10F7
:1024C00082F8BC3046E092F8BD3083F0010382F818
:1024D000BD300BB10C2000E00D2005F071FF39E09C
:1024E0005D2B00F012855B2B00F011855E2B21D156
:1024F000032000F00DBD00BFCC110020902900206A
:102500000C2A0020C0190020150000209C2E00205D
:10251000D80E0020702F0020E0100020483000204E
:102520008E300020BC1900208C300020BC1100200F
:102530001C110020562B03D1029305F0F5F9029BE4
:1025400098F80020002A00F0F9846F2B40F0F08406
:102550000DF0DEFE33685B0736D594F8BD30B64A21
:1025600093B12B7858070FD5019BB9F90610B3F832
:102570009A31994208DD3B6813F0010302BF322112
:10258000A2F8C01082F8BD303B68D9030DD594F88D
:10259000C220A94B2AB993F8BB2012B93222A3F862
:1025A000C020012384F8C2300EE094F8BB30A24A68
:1025B00053B12B7803F0040303F0FF0123B9012387
:1025C00082F8BB1082F8BC30DBF8009000233B603F
:1025D00009F17B0809F1CB0A98F8002098F801303E
:1025E00018F8010C9A420BD2414605F061FE38B151
:1025F00018F8022C012303FA02F23B6813433B60F4
:1026000008F10408D045E7D18C4B1B784BB18C4BBB
:10261000DFF844921A68984612F0020F40F03183B6
:1026200029E309F1CA0709F589783A787B7817F820
:10263000010C9A4225D2394605F03AFE08B397F8C4
:1026400004E00C21BB7801FB0E417E4A013B03EB09
:1026500043031344D1F8C82097F803909A42764870
:102660000FD0C1F8C830002390F8F420C1F8CC3066
:10267000012303FA0EF322EA030381F8C49080F8E1
:10268000F43006374745D0D16F4BDFF8D0A1D3F8EF
:1026900000806E4B4FF0000B1B68029394F82B30B8
:1026A0000393DAF80030002B00F0DC8293F80090FE
:1026B000B9F1000F00F0D682DAF8042002998A1AE4
:1026C000002A0CDB01F5FA72CAF8042094F8F41021
:1026D000012202FA0BF221EA020284F8F420039AA2
:1026E000002A00F0BF821AF8042C59780432D2B2C2
:1026F000002940F07882564931F91210554AB2F853
:10270000982102F1C800814201DD9F7814E0C83AA7
:10271000914202DA99784F420EE094F8F4200123B6
:1027200003FA0BF322EA030384F8F430029B03F567
:10273000FA73CAF8043095E294F8F43043FA0BF3D4
:10274000DA0700F18F82002FCCBF0220012005F0B4
:1027500059FE09F1FF32384B132A00F27B82DFE881
:1027600012F0140023003200440061007F00E400F6
:102770004901AE01E30112027902440055007F00D5
:10278000E4004901B6001B01800198F800104046A2
:102790000F44FA2FA8BFFA2727EAE77788F80070D6
:1027A00005F06CFD01201EE098F8011040460F4432
:1027B000642FA8BF642727EAE77788F8017005F03F
:1027C0005DFD02200FE098F8031040460F44642F8F
:1027D000A8BF642727EAE77788F80370D3F8F810D2
:1027E00005F004FD03203946CAE198F805100D20D4
:1027F00039446429A8BF642121EAE17188F80510F1
:1028000005F0BAFDB9F10D0F00F0248298F804101C
:102810000E2039446429A8BF642121EAE17188F8B7
:102820000410ADE198F806100520394481F3080141
:1028300088F80610A4E100BFD80E002098300020D0
:10284000E0100020A4770108441100209C2E0020F5
:10285000702F0020CC110020BC190020A00F0020F8
:10286000D3F8FC301A78022A22D1384604930EF0AD
:10287000BFFDA9490EF0C4FE049B596A05930EF0F2
:1028800003FD002104900EF0A5FF059B48B9049AB2
:10289000A24910460EF0BCFF049A059B10B19F4A56
:1028A00000E000225A620F20114605F051FD0AE0B7
:1028B00099780F203944C829A8BFC82121EAE171BD
:1028C000997005F059FDB9F10F0F00F0C381944BD9
:1028D000D3F8FC9099F80030022B1AD138460EF04C
:1028E00087FD8D490EF08CFED9F820100EF0CCFC3F
:1028F000002107460EF06EFF30B9384687490EF0CA
:1029000087FF10B1854F00E00027C9F82070122022
:1029100059E199F8011012203944C829A8BFC821EB
:1029200021EAE17189F801102AE1D3F8FC301A7824
:10293000022A22D1384604930EF05AFD77490EF050
:102940005FFE049B196B05930EF09EFC0021049022
:102950000EF040FF059B48B9049A704910460EF0EE
:1029600057FF049A059B10B16C4A00E000221A63DD
:102970001020114605F0ECFC0AE0197B10203944C8
:10298000C829A8BFC82121EAE171197305F0F4FC38
:10299000B9F1100F00F05E81614BD3F8FC9099F80B
:1029A0000030022B1AD138460EF022FD5B490EF0A2
:1029B00027FED9F82C100EF067FC002107460EF018
:1029C00009FF30B9384655490EF022FF10B1534F78
:1029D00000E00027C9F82C701320F4E099F80B10E0
:1029E00013203944C829A8BFC82121EAE17189F818
:1029F0000B10C5E0D3F8FC301A78022A22D13846F1
:102A000004930EF0F5FC47490EF0FAFD049BD96BD8
:102A100005930EF039FC002104900EF0DBFE059BBF
:102A200048B9049A3D4910460EF0F2FE049A059BFF
:102A300010B13A4A00E00022DA631120114605F095
:102A400087FC0AE0997D11203944C829A8BFC82114
:102A500021EAE171997505F08FFCB9F1110F00F0D1
:102A6000F9802F4BD3F8FC9099F80030022B1AD143
:102A700038460EF0BDFC2B490EF0C2FDD9F83810D7
:102A80000EF002FC002107460EF0A4FE30B93846D5
:102A900022490EF0BDFE10B1204F00E00027C9F81A
:102AA000387014208FE099F8151014203944C82983
:102AB000A8BFC82121EAE17189F8151060E0D3F8B8
:102AC000FC9099F80030022B1AD138460EF090FC99
:102AD00011490EF095FDD9F828100EF0D5FB002114
:102AE00007460EF077FE30B938460C490EF090FEDE
:102AF00010B10A4F00E00027C9F82870092062E0F1
:102B000099F8031009203944C829A8BFC82121EA2F
:102B1000E17189F8031033E0000020410000C84251
:102B2000D80E002000007A44D3F8FC9099F80030C9
:102B3000022B1AD138460EF05BFCBB490EF060FD4B
:102B4000D9F834100EF0A0FB002107460EF042FE2B
:102B500030B93846B4490EF05BFE10B1B24F00E018
:102B60000027C9F834700A202DE099F80D100A20CA
:102B70003944C829A8BFC82121EAE17189F80D109C
:102B800005F0FAFB66E0D3F8FC9099F80030022BD0
:102B90001DD138460EF02CFCA4490EF031FDD9F8B9
:102BA00040100EF071FB002107460EF013FE30B905
:102BB00038469D490EF02CFE10B19B4F00E00027D7
:102BC000C9F840700B20394605F0C2FB42E099F885
:102BD00017100B203944C829A8BFC82121EAE17188
:102BE00089F81710CCE7012934D19878904B33F944
:102BF0001230B3F5617F05DB40F633029342A8BF84
:102C0000134601E04FF46173B9F10C0F22D14FF478
:102C1000966292FBF0F0A3F5617393FBF0F3854AA3
:102C2000DFB21378BB4215D0042F34BF3B460223DA
:102C30001370019A09FB03237F4A03F2B2731360F6
:102C400004F07AFC4846394605F096FB781CC0B281
:102C500005F0D8FB94F8F420012303FA0BF3134397
:102C600084F8F4300BF1010BBBF1040F0AF10C0AEC
:102C70007FF417ADCBE43368DB0511D56F4BDB7800
:102C800073B1D9F800309F070AD56D4B1B8813F03C
:102C900001070AD10AF0BAF9012004F065FB04E04B
:102CA000012004F050FB012300E00023D8F80020AD
:102CB00050070DD563B1012004F045FB604B1B8824
:102CC000990708D40AF0A2F9022004F04DFB02E0B3
:102CD000022004F038FBD9F8003013F00A0F29D095
:102CE000D8F80030DA060BD5554B1B885B070AD4A1
:102CF000042004F039FB534B1B88A4F8003102E098
:102D0000042004F020FBD8F800309F0607D54C4B78
:102D10001B88580606D4402004F026FB02E0402021
:102D200004F011FBD8F80030590642BF454B1B8810
:102D3000A4F80231D9F800309A0609D4D8F8003046
:102D40001B0540F1B2804FF4807004F00DFBB0E041
:102D50003D4BDFF8EC901B7813F0020F53D03B4B48
:102D60001B78042B4FD9D8F8003013F4007A0FD019
:102D7000B9F80030DF063AD4102004F0F5FA20202C
:102D800004F0E1FA3248011D06F06CFD02232AE04E
:102D9000B9F8007007F01007BFB22FB1102004F08F
:102DA000D2FA012784F804A1D8F80030580512D5CA
:102DB000D4F8083127495A89B1F90030002BB8BF3F
:102DC0005B42934207DAB1F90230002BB8BF5B4295
:102DD0009342C0F2F380B9F80030990608D520205C
:102DE00004F0B1FA002384F80431012700E0002741
:102DF00094F80C3193BB0E2005F0E2FA164B012239
:102E000083F80C212AE0B9F8003003F03003002BDE
:102E100094D0102004F097FA202004F094FA0023B4
:102E200084F804311DE000BF0000C84200007A446D
:102E3000702F0020582C0020441100204830002022
:102E4000841A0020BC110020C0190020C6190020DF
:102E50004C110020C4110020D80E0020002F3FF498
:102E60006DAF00221446624B002023F81400614B22
:102E7000191D03F10A0721F814000021D15117444C
:102E80007860B96023F8140003F132075A33D15146
:102E9000D150174413447860B96058609960143277
:102EA000002C7FF44BAF0124DDE74FF4807004F079
:102EB0004AFA514B5A791C46082A01D00E2A02D1EF
:102EC000402004F040FA33685A0540F18D8094F8B0
:102ED00018321BB92B7813F0040F03E0D8F8003038
:102EE00013F4002F0AD0454B00221A703C200AF040
:102EF00057FA002878D00CF09FFBF7E70DF0C6FEDC
:102F000009B0BDE8F04F0AF068B9012000E00220E6
:102F10005FFA80F8019A08F1FF3382F8B03704F0C5
:102F200065FA04F02DFB404605F06CFAFFF712BB82
:102F3000BAF1000F02D07E2B3FF40AAB972B05D1DC
:102F40004FF4C873A4F8BE30FFF704BBA72B06D11B
:102F50002B4A137843F004031370FFF7FBBA0022E7
:102F6000BB2B079201D1022303E0B72B04D14FF60C
:102F7000FE73ADF81E300AE0BE2B01D1022304E03F
:102F8000BD2B7FF4E7AA4FF6FE73ADF81C30DBF8DB
:102F90000030BDF81C10B3F858200A44A3F858209C
:102FA000BDF81E10B3F85A200A44A3F85A2004F0C2
:102FB000BBFC002384F8BA30FFF7CCBAB9F8003074
:102FC0009B063FF515AF202004F0CEF90D4B0E48BF
:102FD0001A685B68011D4360026006F043FC0B4BFE
:102FE000012783F8047103E709B0BDE8F08F00BF43
:102FF00090300020E60F0020CC110020692800202E
:10300000C0190020C819002054110020D80E00203B
:10301000B54B2DE9F04FB3F90610B44B85B01F68DE
:1030200001937A8991420EDBB1F5FA6FFC79BFBF4B
:103030008B1A6343A2F5FA6493FBF4F4ACBFC4F1BA
:103040006404643400E06424A94BAA4AB3F898B13C
:1030500093F9623112689BB20292154603930022E3
:1030600040F2E630A04B4FEA420C33F912E0CBEBD2
:103070000E0303F2F316864203D8002BB8BF5B425F
:1030800001E04FF4FA73022A2ED0029E96F81161E5
:103090001EB1B342CCBF9B1B0023642093FBF0F80E
:1030A000954E6FF0630A36F818900AFB083A08F15B
:1030B000010836F918600FFA89F8C8EB060606FB16
:1030C0000AF696FBF0F68D484E4420F80C60BE18C8
:1030D0003679642073438A4E93FBF6F364339BB2D4
:1030E000634393FBF0F02CE0029890F812611EB15C
:1030F000B342CCBF9B1B0023642093FBF0F0DFF8AE
:103100002C926FF0630808FB003A39F91060013027
:1031100039F91000002BA0EB060000FB0AFA9AFB1D
:10312000F8FA0398C6EB0A0A0AFB00FA7348B8BF1C
:103130005B42A0F804A0B8794343714893FBF0F0D8
:1031400064306B784FF06408434393FBF8F36D4EA3
:10315000022AB354EB7A6C4E00FB03F393FBF8F3B3
:10316000B3546B7D654E00FB03F090FBF8F0674BAA
:103170009854674B0ED1DE4583F802800DDB5C4C22
:10318000B4F89A21914214DBB1F5FA6FA8BF4FF45D
:10319000FA610FE0DE459C5404DA36F80C305B42ED
:1031A00026F80C300132032A05F101057FF458AFEF
:1031B000E5E71146891A4FF47A735943C2F5FA626A
:1031C000B1FBF2F1642391FBF3F2DFF874E16FF0ED
:1031D00063073EF8120007FB021101323EF912208C
:1031E00007B2D21B514391FBF3F30344F380494BE5
:1031F000424D1B885F063BD5474A484B10881B88C9
:10320000181A00B20EF0F4F845490EF045F90746D9
:1032100003F0C8FF8046384603F051FF0746B5F972
:1032200002000EF0E5F88146B5F900000EF0E0F876
:10323000414682460EF030F93946834648460EF044
:103240002BF9014658460EF01DF80EF0EBFA4146F8
:10325000288048460EF020F93946804650460EF048
:103260001BF9014640460EF00FF80EF0DBFA6880BD
:103270002C4D2B68980740F19E8045F207212A4B80
:103280002A4F1A687B69D31A8B4240F394807A6183
:103290000AF00AFC264BDFF8AC901A789846032A0D
:1032A000B9F8003050D10A2B58D90023282088F8CB
:1032B000003005F0E6F80AF0F7FB1E4B18880AF01C
:1032C000DDFB1D4B1A68D37890FBF3F00130082822
:1032D0001A4BA8BF08201870537980B243433B8330
:1032E00013795843788339E0702F0020441100206F
:1032F000CC1100201C110020BA1A0020C41100209B
:103300000CFEFFFF182A0020761000202C2A002037
:1033100070290020841A0020DA0F0020BC11002040
:1033200035FA8E3C782E00207C300020681000207A
:103330000C1A0020E4280020A81900203C000020DE
:10334000A21A0020AC1900200A2B07D803238E4AAA
:1033500088F80030002313703B837B8398F800309B
:103360008A4A012B0CD002D3022B1BD023E03A8BCC
:10337000B9F800309A421EDD012388F800300FE0D2
:10338000B9F800107B8B8B4202DD022313700FE033
:103390007F4B1B8B0133994202DD002313700AE03F
:1033A000082006E07B8BB9F8002001339A42E3DC69
:1033B000072005F005F82D68290577D5754B744F62
:1033C0001A68FB69C3EB020845F2072398456DDDD7
:1033D000714BB6F906B0D3F800904FF47A7099F8B3
:1033E0000A30FA61012B98FBF0F8B4F85211ABF5F2
:1033F0007A7B6A4E03D042D3022B20D041E0684B47
:10340000396A5A7B674B4FF0080E33F8122091FB54
:10341000FEF392B2C91A8B183B6293FBFEF3BA8497
:1034200040F6E4429BB25343B9F80820C2EB133391
:103430005843B9F9063090FBF3F0306021E05A4B65
:10344000B9F808A01B78C6F800A05A0719D5574844
:1034500004F063FF20B915F0100F18BF4FF0000BF8
:103460000BFB0BF3322293FBF2F3B9F906205B441A
:103470005A434FF47A7392FBF3F3534400E0002372
:1034800033603368D7E90A0103FB08F84FF47A7315
:1034900098FBF3F810EB080041EBE8710023C7E953
:1034A0000A01434A0EF004FA424B1860424E336858
:1034B000DB0427D52F0622D5404B1B789D071ED550
:1034C0003F4B187804281AD900223E4B0521D71803
:1034D000951C4FF00A0E122AD154E9B287F801E088
:1034E00004D0B0EB510F2A46EFD800E014215A184F
:1034F000322002F8010CFF225A540F2000E00A206B
:1035000004F05EFF304D2A68002A73D02F4B304FF5
:1035100018683968984681426CD82E4BDFF8C09005
:1035200018785168B0B901221A70B9F80030CB5C34
:10353000D3B1294B1A700DF079FEB9F800309BB960
:103540002B681B78053B012B0ED804F073FF234B2F
:10355000186009E000221A70B9F80030CB5C1BB18A
:103560001D4B1A700DF062FE2B68B9F800205B68E5
:103570001B499B5CFE2B02D100230B803AE0FF2B02
:1035800030D104F00DFF35E03C0000200C1A002083
:10359000681000207C300020A8190020B4190020F9
:1035A000CC280020DC280020973000205613002073
:1035B000407E0500B8190020E0100020C01900204E
:1035C000C6190020842C0020D41A00209C2E002034
:1035D000CC1A0020C91A0020C81A0020582E00203A
:1035E000D01A0020D8F800000A2505FB0303013299
:1035F0003B600A809D4D2B7858073DD43268D10737
:103600005CBF43F001032B70994B1B781F075EBF13
:103610002B7823F001032B70D60248BF2B78954AF4
:1036200044BF23F001032B70934B1B6813F0040F6E
:1036300002D09249098851B99149098809B198077E
:1036400005D4904B1B88003318BF012333B10223EC
:1036500013702B7823F001032B7004E02978C9073D
:1036600058BF0223137004F0E5FE874B1B68C01A95
:10367000002801DB0DF0DAFD0DF008FB834B1E780E
:103680009846002E00F0AB80814E3368002B00F08E
:10369000EE8630680AF04FFE002800F0E8867C4B8A
:1036A0007C4C18680AF044FE092801D03F2850D10C
:1036B0004FF0000A5746D4F80090774DB9F1000F4B
:1036C00005D0764829684A4611F0E4FC10B9AA46AC
:1036D00007B92F46724B10359D42EFD3C7B1D7F8CB
:1036E00000E0DAF800C023681EF803501CF803005D
:1036F000A8420DD15A1C694938B92D2B05D8654D02
:103700002A602025CD54885402E0CD542260EAE797
:1037100023680BB1574511D062480CF07DF857452E
:1037200007D857F8100B0CF077F809200CF06CF85C
:10373000F5E75D480CF070F84FF0000923689945F3
:10374000A7D2564B13F809000CF05EF809F10109F5
:10375000F4E72368002B40F06F86042840F0A88629
:103760004E4806F0FFFB00F082BED9F80000DFF8FB
:1037700048A10AF0E0FD40B3DAF800000AF0D8FDF5
:10378000DBF80030024693F84810002935D1242890
:1037900040F09480012283F84820DBF80030DFF805
:1037A00014A193F84820062ADFD193F8490001F0CC
:1037B000E9FC8146002800F0AC803B6898790BF06A
:1037C00078FF3B68002283F84820384B93F8353067
:1037D000002B40F01F864C36982E00F04886344B64
:1037E000F21892F84A100129F5D1324FF3583A6095
:1037F000314ABB4613609146B7E7012904D14D28F1
:1038000014BF00220222C6E7022904D13C2814BFBB
:1038100000220322BFE703290CD140284FF000010A
:1038200002D983F84810B8E758711971D9719871A5
:103830000422B0E7042906D1997983F849004A4067
:103840009A710522A7E70529A7D1587919798842E5
:10385000987906D950409871481C18710B441A7217
:103860009BE790420CBF0622002294E7973000208D
:10387000C0190020C81A0020BC1900208C3000207C
:10388000960F00208E3000206C30002098300020F1
:10389000742C0020541D00208C7E0108241D002063
:1038A0003C800108649701086997010868100020AE
:1038B000C8270020641A0020681A00202B78D849F5
:1038C00058073FF56AAF232ADAF8003014D10120F7
:1038D00088F80000D34803910360D3480292036341
:1038E000D2480BF099FFD2480BF096FF0399029A49
:1038F0000B7843F002030B70CE4B1B681B7893428E
:1039000001BFCD4ACD4B1A60CD4A04BFCD4BDA6022
:1039100043E7DAF8002092F849304C2B00F0698434
:103920005DD8332B00F0A08421D8292B00F02D8402
:1039300009D8252B00F00484272B00F00884232BC2
:1039400040F0B2852FE22D2B00F0308407D82B2BCE
:1039500040F0AA850BF090FE607100F03EBD2F2B69
:1039600000F0EE84312B00F0008500F09DBD3E2B71
:1039700000F0F2801DD8372B00F0AA8404D8352B34
:1039800000F04A8200F090BD392B00F0ED833C2B13
:1039900040F08A85DFF8B092D9F800A00BF06CFEF9
:1039A0008AF80000D9F8003018780AF033FF00F0E8
:1039B00014BD432B00F0698406D8412B40F0748578
:1039C0004FF0000900F055BC442B00F002854A2B53
:1039D00040F06A850BF05AFEA08100F0FEBCD02BAF
:1039E00000F0108355D8CA2B00F0C08009D8C82B2E
:1039F00000F0858000F23E834E2B00F0078400F03B
:103A000053BDCD2B00F0098304D8CC2B00F02C82C1
:103A100000F04ABDCE2B00F00983CF2B40F0448547
:103A20000BF034FE6FF4AF6283189BB2C62B98BFC5
:103A3000A4F898010BF02AFEA4F844010BF026FE2E
:103A4000A4F846010BF022FEA4F848010BF01EFE7C
:103A5000A4F8DA010BF010FE84F8EF010BF00CFE75
:103A60000BF00AFE84F8F0010BF006FE84F88701E3
:103A70000BF002FE84F894010BF0FEFD724BD3F8BC
:103A800000900BF003FE00EB80004000A9F8560008
:103A90006AE3D62B00F03B820AD8D22B19D0C0F0B3
:103AA0001083D32B25D0D42B00F03C8200F0FCBC3B
:103AB000EF2B41D005D8D82B40F0F6844FF0000909
:103AC00004E1F22B00F07682FA2B00F0B88200F0CD
:103AD000EBBC2B78590700F180840BF0CDFD022858
:103AE00084F8B00740F29482584B002283F8B02744
:103AF0008EE20BF0CBFD564B188000F06EBC92F8B6
:103B000005904FEA5909B9F1120F03D909F044FCA5
:103B100000F063BC4FF0000ACA4507D20BF0B6FDB7
:103B20004C4B23F81A000AF1010AF5E73E4B01223B
:103B300083F8342000F051BCDFF80C91D9F800A0D4
:103B40000BF0A4FDAAF85A00D9F800900BF09EFDE6
:103B5000A9F8580000F041BC0BF08EFD84F8E2019A
:103B60000BF08AFD84F8E10100F037BC364B1A688F
:103B70009A461278022A40F08E80DAF8003009F175
:103B8000080B02930BF078FD0DF02EFC32490DF07E
:103B900037FD029B43F82B00DAF800B00BF06CFD08
:103BA00009F10A030BEB830B0DF01EFC2B490DF002
:103BB00027FDDAF80030CBF8040002930BF05CFD2F
:103BC0000DF012FC26490DF01BFD09F10E0B029BB6
:103BD00009F10109B9F1030F43F82B00CDD1B9F177
:103BE000070FDAF800B03DD10BF046FD0DF0FCFBFD
:103BF00019490DF005FDCBF84400DAF800B00BF0E0
:103C00003BFD0DF0F1FB14490DF0FAFCCBF8480038
:103C1000DAF800B00BF030FD8BF84C0035E000BF57
:103C200097300020742C002068100020999701081C
:103C3000699701086C280020EFBEADDEF04F002030
:103C40000400FA0500ED00E01C110020CC1100205A
:103C5000D80F0020702F0020000020410000C84233
:103C600000007A440BF008FDCB448BF80100DAF831
:103C700000B00BF001FDCB448BF80B00DAF800B07C
:103C80000BF0FAFCCB448BF8150009F10109B9F1EE
:103C90000A0FA4D1A1E3DAF800B00BF0EDFCCB449D
:103CA0008BF80100DAF800B00BF0E6FCCB448BF89F
:103CB0000B00DAF800B00BF0DFFCCB4409F101098E
:103CC000B9F10A0F8BF81500E5D186E3DFF890A370
:103CD00009F1080BDAF8003002930BF0D7FC0DF075
:103CE00083FBD9490DF08CFC029B43F82B00DAF8DA
:103CF00000B00BF0CBFC09F10A030BEB830B0DF0CA
:103D000073FBD1490DF07CFCDAF80030CBF80400ED
:103D100002930BF0BBFC0DF067FBCB490DF070FC80
:103D200009F10E0B029B09F10109B9F1030F43F8E8
:103D30002B00CBD1B9F1070FDAF800B01AD10BF094
:103D4000A5FC0DF051FBC0490DF05AFCCBF8440026
:103D5000DAF800B00BF09AFC0DF046FBBA490DF012
:103D60004FFCCBF84800DAF800B00BF08FFC8BF872
:103D70004C0012E00BF08AFCCB448BF80100DAF81F
:103D800000B00BF083FCCB448BF80B00DAF800B0EA
:103D90000BF07CFCCB448BF8150009F10109B9F15B
:103DA0000A0FC7D119E30BF067FC132883463FF6CF
:103DB000ADAEDFF8ACA2DAF800900BF05DFC0023AA
:103DC000A2490C2202FB0312117A814220D11378FE
:103DD00009EB8B0989F879300BF04EFC89F87A00F1
:103DE0000BF04AFC89F87B000BF046FC984A994B93
:103DF00089F87C001A60DAF80000974B00211860FF
:103E0000793004F079FA954B80F001001870E4E203
:103E100001331C2BD4D179E60BF02EFC0B28824603
:103E20003FF674AE8E4BD3F800900BF025FC0328C0
:103E30003FF66CAE062303FB0A9989F8CE000BF01F
:103E40001BFC89F8C9000BF017FC89F8CA000BF0BD
:103E500013FC89F8CB000BF00FFC89F8CC000BF0B9
:103E60000BFC89F8CD00B8E25379092B7FF64EAEF2
:103E7000019BD3F800900BF0FFFB019B89F8000039
:103E8000D3F800900BF0F8FB89F801000BF0F4FB7D
:103E9000019B64281B68A8BF642018710BF0ECFB21
:103EA000019B64281B68A8BF642058710BF0E4FBD9
:103EB000019BFF281B68A8BFFF2098710BF0DCFB5B
:103EC000019B6428D3F8009028BF642089F807007C
:103ED0000BF0D2FB019B89F80200D3F800900BF0A5
:103EE000CBFB019B89F80300D3F800900BF0CEFBCD
:103EF0003B68A9F80A005B790A2B40F26E82594BA5
:103F0000D3F800900BF0B8FB89F8080065E20BF0DD
:103F1000BDFB554B23F8190009F10109B9F1080F50
:103F2000F5D15AE253790F2B7FF4F0AD0BF0A4FBDF
:103F3000072881463FF6EAADDFF824A1DAF800B0A1
:103F40000BF0A4FB0E2303FB09F9CB44ABF81901DA
:103F5000DAF800B00BF09AFBCB44ABF81B01DAF8AF
:103F600000B00BF093FBCB44ABF81D01DAF800B0C6
:103F70000BF082FBCB448BF81F01DAF800B00BF09A
:103F80007BFBCB448BF82001DAF800B00BF074FB1C
:103F9000CB448BF82101DAF800B00BF06DFBCB4479
:103FA0008BF82201DAF800A00BF07AFBD144C9F8B3
:103FB000230112E20BF060FB0F2881463FF6A6AD0D
:103FC0000BF05AFBC9EBC909A14489F8D4000BF0E6
:103FD00053FB89F8D5000BF04FFB89F8D6000BF0A6
:103FE0004BFB89F8D7000BF047FB89F8D8000BF0A2
:103FF00043FB89F8D9000BF03FFB89F8DA000AF09F
:104000005BFBEAE12B785B0700F1E7810BF030FE08
:1040100003F0ECF903F0B4FADFE12B78580700F174
:10402000DC81124B4FF4C8721A80D6E12B78590705
:1040300000F1D3810E4A137843F004033FE02B785C
:104040005A07E5D530E200BF00007A44387801080D
:1040500010130020D00F0020D40F002015000020E6
:104060001C110020441100205A2C0020960F002023
:10407000C01900200BF000FBDA4B1A7810B142F0A7
:10408000020201E022F002021A700BF0F5FAD64BA0
:10409000DFF8789318700BF003FBC9F800000BF001
:1040A000FFFAC9F804000BF0F1FAD04B18800BF0BE
:1040B000EDFACF4BCF4A1880137843F00203137008
:1040C0008BE10BF0D9FA02900BF0EAFA83460BF081
:1040D000E7FA82460BF0E4FA81460BF0D7FA0BF0D0
:1040E000D5FA0BF0C9FA029BA3B9C34B1020C3F851
:1040F00000B0C3F804A003F026F9BA4A137843F0DD
:1041000001031370B9F1000F00F06781BB4BC3F8D6
:10411000009062E1102B40F06081B94BC3F800B011
:10412000C3F804A0B9F1000F02D0B44BC3F800905B
:10413000B348B44B0222011D1A7005F093FB4CE109
:10414000A0600BF0ADFAA3681843A06045E10BF046
:104150009DFAA4F85C010BF099FAA4F85E010BF04B
:1041600095FAA4F8600138E10BF086FA84F87C0136
:104170000BF082FA84F880010BF07EFA84F87F015C
:104180000BF07AFA84F8810127E10BF07FFAA4F8AA
:1041900082010BF07BFAA4F884010BF06DFA84F82D
:1041A00086010BF073FAA4F8880116E10BF064FAAB
:1041B00084F892010BF06AFAA4F89C010BF066FAFD
:1041C000A4F898010BF062FAA4F89A010BF054FAE3
:1041D000DAF8003084F893015B79082B40F2FD8017
:1041E0000BF054FAA4F89E010BF050FAA4F8A001C9
:1041F000F3E00BF041FA84F8D8010BF03DFA84F8B3
:10420000D9010BF043FAA4F8DA01E6E092F8059040
:104210000323B9FBF3F9B9F1120F3FF677ACDFF8DE
:10422000F0A14FF0000BCB4580F0D7800BF024FAC3
:104230008AF8A2010BF02AFA40F2ED23984205DD3C
:1042400040F6CA039842A8BF184601E040F2EE20AB
:10425000A0F2EE20192390FBF3F00BF1010B8AF88A
:10426000A3010AF1020ADEE70BF006FA84F89401D2
:10427000B3E00BF001FA04EB090309F10109B9F10C
:10428000080F83F88A01F4D1A7E00BF0F5F9C4F820
:10429000089060710BF004FAA3681843A0600BF05B
:1042A000EBF984F892010BF0F1F9A4F85C010BF042
:1042B000EDF9A4F85E010BF0E9F9A4F860010BF048
:1042C000E5F9A4F882010BF0E1F9A4F8840184E097
:1042D00053794FF0070AB3FBFAF2C2EBC2029A1A03
:1042E00012F0FF0F7FF412ACB3FBFAFA0AF1FF3AB7
:1042F0005FFA8AFABAF1FF0F6FD00BF0BDF95FFADF
:1043000080FB4FFA8BF003F091FE814600283FF4CA
:10431000FDAB80F800B00BF0B9F9A9F802000BF082
:10432000ABF989F804000BF0A7F989F805000BF048
:10433000A3F989F807000BF09FF989F80600D5E783
:10434000DFF8CC9009F1400A0BF0A0F9A9F8A80217
:104350000BF092F989F8AA020BF08EF909F1040921
:1043600089F8A702D145EFD137E00BF085F91F2876
:1043700081463FF6CBAB3B685B79082B7FF4C6AB3D
:104380000BF084F909F18A0904EB890A00F03F0077
:10439000AAF802000BF07AF9BAF80230800100F4B2
:1043A000FE501843AAF802000BF066F9000104F869
:1043B00029000BF061F914F8293000F00F001843C0
:1043C00004F829000BF058F98AF801000AF0B6FA4F
:1043D00003E00D4B012283F8352000200BF098F903
:1043E000FFF7EBB9C0190020C6190020C41900203E
:1043F000C21900204A1100204C1100205C1100203D
:1044000054110020DC0F002068100020C819002083
:10441000CC110020584B985904F0C2F818B932203A
:1044200004F02FF8F6E70AF007F902F0B5FF534A57
:10443000534BDA60FFF7CFB90C283BD00A2842D1A2
:10444000504D51480BF0E8F92846232110F00BFE9F
:1044500008B1401B20602368002B57D14948002138
:104460003022236010F0C9FD98F800302BBB474B79
:104470001B689B060FD5464B46491B688A6B9A1AE8
:10448000002A08DB444A1278042A82BF03F512335B
:1044900003F5F8738B63414B9B68002B69D0404850
:1044A00005B0BDE8F04F184708F076FFFFF785B973
:1044B0000C2804D13B480BF0AFF93B480DE07F28B6
:1044C00012D1FFF7E6B80D28BAD07F2809D12D4ABE
:1044D000013B002135482360D1540BF09DF9FFF7D3
:1044E000D8B82F2B3FF6D5A8A0F12002D2B25E2A71
:1044F0003FF6CFA813B920283FF4CBA85A1C22605E
:10450000204AD0540BF080F9FFF7C3B85A1EA95CBB
:10451000202901D113469FE71A4A00212360D15474
:10452000234B244DD3F800A0D5F800B0DFF8549009
:10453000584610F0A6FD074659463A46484610F040
:10454000A9FD1D4A28B919F8073053445B785B0769
:1045500003D010359542E7D306E0954204D2781C8B
:10456000EB684844984702E014480BF055F90023E3
:1045700074E705B0BDE8F08FC82700200400FA05F5
:1045800000ED00E0241D002036A50108BC19002024
:104590007C30002068100020C61900204027002031
:1045A000A41000206E9701086997010895970108EB
:1045B000500000208C7E01083C800108799701089A
:1045C0008F4A70B51368988A80B2C1B2CE072ED5D3
:1045D000198821F400610904090C1980198889B22D
:1045E00041F48061198000211171517999B191795B
:1045F00011B9D179FF290ED101219171117A0229C6
:1046000001BF198889B241F400611980517A41F0E3
:1046100001011982DFE0517A01F0FE011982D3799C
:10462000FF2B00F0D880764BFF211971D3E08D0766
:104630003AD5BFF35F8F107AC0B2012813D15179F8
:1046400089B1917979B1198821F480610904090C43
:104650001980BFF35F8F198B1988907289B241F46A
:10466000007119801BE0198BBFF35F8F107A6449CA
:1046700002280AD1487940B1897931B1198821F4E9
:1046800080610904090C19809FE0107A5C490328B5
:1046900005D1487918B18979002940F09680998828
:1046A00089B241F4806195E04C0754D501219172A3
:1046B0005179002936D09179002933D0117A1888A0
:1046C000022911791CD920F480600004000C1880A4
:1046D0001C8AD568C8B2E4B249B26C54198889B250
:1046E00041F400711980811C1171198A0130C9B21D
:1046F00040B22954998889B241F48061998026E0BA
:1047000080B240F4007018801C8AD568C8B2E4B248
:1047100049B26C541C8A411C49B2E4B203306C5457
:10472000107114E09179364809B9017C41B11988BA
:1047300089B241F40071198011790131117106E0DB
:10474000198889B241F48071198001218171198819
:10475000C905FCD43FE001F0400101F0FF04E1B1E4
:1047600010791E8AD568C4B2611C40B2F6B22E54CC
:10477000C9B2157A117149B2C81C854201BF988827
:1047800020F480600004000C08BF9880137A8B42EC
:1047900021D11B4B02341C711DE006061BD511797B
:1047A00048B2451C0AD054690131205CC9B2188254
:1047B000107A117149B288420DD106E0D179147195
:1047C0001982517909B9117A29B9998821F480613E
:1047D0000904090C9980117A92F904000131884288
:1047E000074B0CD100219971997A31B119688B88E6
:1047F00023F440731B041B0C8B800023137670BDC5
:10480000A81000202DE9F04FDFF8589285B0074638
:10481000D9F81C000E460CF0EBFD8E4C804620882B
:104820000CF0E2FD4FF05C51054640460CF034FEC2
:104830004FF06451824628460CF02EFE0146504649
:104840000CF020FD4FF06251824640460CF024FEF1
:104850004FF06A51804628460CF01EFE0146404645
:104860000CF010FD0546B4F902000CF0C1FD014644
:1048700028460CF011FE5146054650460CF00CFE41
:104880008046B4F904000CF0B3FD014640460CF03C
:1048900003FE014628460CF0F7FC80460CF0C2FFF0
:1048A0006D490546A06140460CF0AAFED9F82030BB
:1048B0008046284601930CF09BFD4FF07C510CF094
:1048C000EBFD66490CF0DEFC0546E389B4F90A000D
:1048D00002930CF08DFD29460CF0DEFD29460CF00C
:1048E000DBFD4FF058510CF0D7FD8146B4F90800BC
:1048F000B4F810B0B4F80CA00CF07AFD29460CF016
:10490000CBFD014648460CF0BFFC4FF058510CF06F
:10491000C3FD4FF060510CF0BFFD4FF07E510CF025
:10492000B3FC8146E0880CF05FFD014648460CF080
:10493000B3FD002181460CF043FF00287BD12946BE
:1049400028460CF0A9FD03900FFA8BF00CF050FDF7
:10495000039B014618460CF09FFD4FF060510CF090
:104960009BFD8346BDF908000CF042FD0146284638
:104970000CF092FD01460CF087FC014658460CF005
:1049800083FC4FF07A510CF087FD834601980CF0C0
:104990002FFD01464FF093400CF074FC05460FFAD2
:1049A0008AF00CF025FD4FF08F410CF075FD0146AB
:1049B00058460CF069FC4FF066510CF06DFD014655
:1049C00028460CF05FFC26490CF066FD49460CF0C9
:1049D00017FE0546B4F916000CF00AFD29460CF046
:1049E0005BFD29460CF058FD4FF040510CF054FD92
:1049F0008146B4F914000CF0FBFC014628460CF08B
:104A00004BFD4FF060510CF047FD014648460CF05D
:104A10003BFC8146B4F912000CF0EAFC0146484622
:104A20000CF032FC4FF076510CF036FD0146284672
:104A30000CF02AFC00E0002017B10CF0F3FE386007
:104A40002EB140460CF0EEFE64235843306005B0B2
:104A5000BDE8F08F480B00200000A04500007A4719
:104A60000050C345A8100020704770472DE9F04161
:104A7000324C334D6289AB8CB4F904809A1A238985
:104A8000B4F902E05A43B4F91230D613B4F9142041
:104A9000DB02324493FBF2F232440A26E2615643CF
:104AA000A2F57A6202FB02F3B4F90EC002FB0EFE1D
:104AB00002FB08F2B4F90C801B130CFB03FC03FB94
:104AC00008F31B1403EB62320232E388921002F502
:104AD000004253434CF25032B4F920704FEAEE2EAC
:104AE000B4F900400EEBEC2C0CEB8404BC40AD6A36
:104AF0000234A5EBA4043A4162434FEAD3384EBFD7
:104B0000B2FBF8F35400B4FBF8F340F6DE3448BFD0
:104B10005B001A12524362430A4C08365C43241469
:104B200004EB224202F6CF62361103EB221300B1EE
:104B3000036001B10E60BDE8F08100BF200B0020D2
:104B4000A810002043E3FFFF064B93F82C2002F04F
:104B5000FF012AB101220270002283F82C20704745
:104B600001707047A8100020104B13B593F82D204A
:104B70001C46CAB90E4B1B68B3B11A681AB10D496D
:104B8000886902438A619A889868ADF804200222F5
:104B90008DF8072004220DEB02018DF8062007F0A6
:104BA00013F8012384F82D3002B010BDA8100020A6
:104BB000180B00200010024008B5FFF7D5FF074B87
:104BC0001B7813B1012B03D008BD4FF4006201E044
:104BD0004FF48052024B1A8008BD00BF1C0B00200E
:104BE00016000020012828BF01202DE9F04F0646BD
:104BF000142000FB06F3704F89B0F918FC586F4B76
:104C00000A691C6083F82E606D4BB1F80880DD697D
:104C1000B1F80AA02A43DA61A2884D6822F44072F2
:104C20001204120C4AEA0809A28003A9C5F81090E0
:104C300002228DF80E0028460193ADF80C908DF8F5
:104C40000F2006F0C1FF019B00971F464FF0080B95
:104C5000AA6818EA020F03D10A2003F007FCF7E75D
:104C60000A20C5F8148003F001FCC5F810800A2062
:104C700003F0FCFBBBF1010BEAD1C5F814A00A203C
:104C800003F0F4FBC5F814800A2003F0EFFBC5F82D
:104C900010800A2003F0EAFB0222C5F810A0284683
:104CA00003A98DF80F201C228DF80E20ADF80C9072
:104CB00006F08AFF434A03A894423A690BBF42F4C4
:104CC000001242F480023A613A610BBF3A693A69D4
:104CD00022F4001222F480023A61A38823F4407384
:104CE0001B041B0CA38023889BB243F00103238089
:104CF000A58808F01DFC0599334B25F03F05B1FB55
:104D0000F3F32D042D0C1D43ADB2A58022880025A0
:104D100022F001021204120C22802C4A03A8B1FBDB
:104D2000F2F100298AB208BF012242F400414FF497
:104D3000967253434FF47A7293FBF2F301339BB2B2
:104D40002384A1832388009A9BB243F0010323802C
:104D5000238823F4816323F002031B041B0C2380AC
:104D60004FF480432381142303FB0626737B012425
:104D70008DF80C308DF80D508DF80E508DF80F40D9
:104D80000BF09EFC337B9DF80F208DF80C308DF8D6
:104D90000D508DF80E501AB103A80BF091FC08E0ED
:104DA0005A0903F01F039C4002F12003084A42F80D
:104DB000234009B0BDE8F08FE0770108A81000207B
:104DC000001002400054004040420F00804F12008B
:104DD00000E100E010B5214C2368998A89B211F4F2
:104DE000706F1CBF012284F82F2011F4E06F2BD0CC
:104DF0001A8B9A88890522F480624FEA02424FEAB0
:104E000012429A8020D41A8892051DD41A88D0059F
:104E10000FD51A88D105FCD41A8892B242F40072D8
:104E20001A801A889205FCD494F82E00FFF7DAFE57
:104E30000AE01A8892B242F400721A809A8822F428
:104E400040721204120C9A802268938A23F47063D1
:104E50001B041B0C93820023237610BDA810002096
:104E6000064A08B5138801339BB21380044B93F8AC
:104E70002E00FFF7B7FE002008BD00BFDE100020A7
:104E8000A810002010B540001C4CC0B26072E17147
:104E90000120002121746071227220762068E36075
:104EA000636184F82F1040B383889B0515D4038871
:104EB000D9050DD447F230530288920502D5013B43
:104EC000FAD112E08BB103889BB243F48073038064
:104ED00083889BB243F44073838047F23053227E31
:104EE00012B1013BFBD100E013B9BDE81040B7E7B8
:104EF000024B93F82F0080F0010010BDA810002095
:104F000007B5F7216B4606227620FFF7BBFF9DF819
:104F100000309DF801101B0343EA01139DF80210B5
:104F2000094A43EA111313629DF803309DF80410F7
:104F30001B0343EA01139DF8051043EA1113D361E3
:104F400003B05DF804FB00BFA810002007B5F621F0
:104F500001AB03227720FFF795FF9DF805309DF800
:104F600004201B0243EA02439DF806201343054A2E
:104F7000B2F92020C2F10802D340034A936203B081
:104F80005DF804FB200B0020A810002007B5F621D7
:104F900001AB02227720FFF775FF9DF804209DF8F2
:104FA000053043EA0223024A938403B05DF804FB10
:104FB000A810002013B506220446432168206B4642
:104FC000FFF760FFA8B19DF800209DF80130012097
:104FD00043EA022323809DF802209DF8033043EA30
:104FE000022363809DF804209DF8053043EA0223E4
:104FF000A38002B010BD13B5062204463B216820F1
:105000006B46FFF73FFFA8B19DF800209DF80130E7
:10501000012043EA022323809DF802209DF80330FB
:1050200043EA022363809DF804209DF8053043EA9B
:105030000223A38002B010BD13B51F4B4000C0B2C5
:10504000587202AC1868D97104F8012D00210122B0
:105050001A745C615971DC601A721A7683F82F1029
:1050600040B38288920515D40288D4050DD447F246
:1050700030520188890502D5013AFAD112E08AB18D
:10508000028892B242F480720280828892B242F424
:105090004072828047F23052197E11B1013AFBD141
:1050A00000E012B9FFF7DCFE04E0034B93F82F0099
:1050B00080F0010002B010BDA81000207620F4217D
:1050C0003122B9E7044B772093F82020F421920194
:1050D000343202F0FC02AFE7200B00207720F421ED
:1050E0002E22A9E708B5FFF73FFD6B21802268203B
:1050F000FFF7A2FF642003F0C4F96B2103226820AC
:10510000FFF79AFF0F4B19211A786820FFF794FFD9
:105110000F2003F0B6F90C4B1A211A786820FFF71C
:105120008BFF1B2118226820FFF786FF1C2110220D
:105130006820FFF781FFBDE8084068203721002282
:105140007AE700BF640B002014000020FFF738BA94
:1051500040E6FFF735BA3DE607B5232003F091F9A5
:105160006820752101220DF10703FFF78BFE28B19E
:105170009DF80700A0F168035842584103B05DF85C
:1051800004FB00BF4D282DE9F047044600F054868B
:1051900000F2B980302800F0B48651D8222800F0FF
:1051A000908423D8032800F0058214D8012800F049
:1051B000F581022840F0F48604200AF0A9FA432081
:1051C0000AF077FA4C200AF074FA46200AF071FAD5
:1051D0004C2000F056BE042800F0F581052840F070
:1051E000DF861A200AF094FA0024FCE1282800F057
:1051F000E28515D8242800F0C985262840F0D086FD
:10520000DA4C06200AF084FAB4F85C010AF083FA5A
:10521000B4F85E010AF07FFAB4F8600100F0B3BDA3
:105220002C2800F0DB852E2800F055862A2840F037
:10523000B78601200AF06CFACC4B587900F021BEF9
:105240003D2800F0F8821ED8362800F02B860BD8B7
:10525000322800F01086342840F0A28648200AF058
:1052600057FA002500F04FBC3A2800F0B9823B28DD
:1052700000F02084382840F0938604200AF048FA91
:10528000BA4C00F089BD452800F0768627D8402822
:1052900000F0FA85422840F08386B44C10200AF0D2
:1052A00037FA60790AF005FAA0680AF03DFA94F836
:1052B00092010AF0FEF9B4F85C010AF02CFAB4F895
:1052C0005E010AF028FAB4F860010AF024FAB4F892
:1052D00082010AF020FAB4F8840100F054BD492894
:1052E00000F0B4824B2800F09885462840F058869C
:1052F0000D200AF00DFA00200AF0DBF900200AF078
:1053000013FA00F044BE702800F0F08200F2E18051
:10531000692800F0458200F2B280662800F0A08182
:1053200000F2A280642800F07781652840F038867A
:105330008F4C0B200AF0ECF920880AF0ECF9608819
:1053400080B20AF0E8F98B4B1B68C3F3C000C3F3CB
:105350008002800040EA4200C3F340021043C3F3DE
:10536000401240EAC20003F0100318430AF0D3F9D8
:10537000814B1A88636802F0080103F4475949EA2F
:10538000010903F4804149EA010903F4004149EAB3
:10539000010903F4803149EA010903F4003149EAC3
:1053A000010903F4802149EA010903F4002149EAD3
:1053B000010903F4801149EA010903F0007349EA85
:1053C0000303DFF8D49112F0010F99F8009018BF91
:1053D0004FF00208C9F3800908BF4FF0000843EA04
:1053E000090312F0020F43EA080314BF4FF0040C44
:1053F0004FF0000C12F0040F43EA0C0C14BF4FF0F6
:10540000100E4FF0000E12F0400F14BF202700279F
:105410004CEA0E0E12F0100F14BF4FF40076002667
:105420004EEA070712F0200F14BF4FF480650025E5
:105430003E4312F4807F14BF4FF4006000203543D8
:1054400012F4007F14BF4FF400110021284312F41E
:10545000806F41EA000114BF4FF0806300230020F9
:105460001943247A0346E7E0672800F02181682881
:1054700040F0968510200AF04BF9002488E16C2852
:1054800000F0A18117D86A2800F003846B2840F04F
:10549000878505200AF03CF9384B18880AF03BF95B
:1054A000374B18880AF037F9314B93F86E0000F04B
:1054B000010000F0E6BC6E282D4D00F0978100F24F
:1054C000CB8106200AF024F9E86D0AF02DF92D4B66
:1054D00084E1782800F0F98018D8742800F034832B
:1054E0000AD8722800F09583732840F05985082067
:1054F0000AF00EF90124C5E3762800F0EA8300F2F1
:105500005C832F200AF004F91F4CCBE2A42800F0A2
:10551000068414D87B2800F06B82A02840F04085D8
:105520000C200AF0F5F8194B18680AF0FDF8184B32
:1055300018680AF0F9F8174B186800F02CBDF1282C
:1055400000F0FF80FE2800F01184F02840F028854C
:10555000074C04200AF0DCF8236CB3F85A000AF078
:10556000DAF8236CB3F8580000F00DBCCC11002021
:10557000DC100020BC190020841A00203A1A0020F8
:105580003C1A0020B411002007780108E8F7FF1F3B
:10559000ECF7FF1FF0F7FF1F9730002003200AF001
:1055A000B7F800200AF085F820460AF082F80D20AE
:1055B00000F067BC0AF0ACF801200AF07AF80A2083
:1055C0000AF077F8A9E306200AF0A2F84F200AF0C3
:1055D00070F84C200AF06DF849200AF06AF8312082
:1055E0000AF067F8CEE3B04B185D01340AF061F8B9
:1055F0000B2CF8D10024AD4B185D01340AF059F89A
:10560000082CF8D10024AA4B185D01340AF051F897
:10561000072CF8D100F0C1BC07200AF079F8E72088
:105620000AF047F8A34B58790AF043F800200AF033
:1056300040F8042000F0AFBCA3420AD29E4A9D5C11
:10564000012202FA05F50D421CBF9A4010430133B6
:10565000F2E70AF069F8974B93F8B00700F011BC35
:1056600012200AF055F8954B00241B88B3F5806F83
:105670008CBF08250125924B33F91400013490FBAF
:10568000F5F080B20AF047F8032CF4D18D4CA08CD1
:105690000AF041F8E08C0AF03EF8208D0AF03BF861
:1056A000608D0AF038F8A08D0AF035F8E08D6AE3D5
:1056B00010200AF02DF80024834B185D013409F006
:1056C000F8FF102CF8D100F068BC70200AF020F828
:1056D00000260E2474437B4D01362B6C2344B3F813
:1056E00019010AF018F82B6C2344B3F81B010AF0D7
:1056F00012F82B6C2344B3F81D010AF00CF82B6C44
:10570000234493F81F0109F0D4FF2B6C234493F832
:10571000200109F0CEFF2B6C234493F8210109F0FE
:10572000C8FF2B6C234493F8220109F0C2FF2B6CB5
:105730001C44D4F8230109F0F7FF082EC9D100F06A
:105740002CBC702009F0E4FF5A4C04F1700594F869
:10575000D40009F0AEFF94F8D50009F0AAFF94F840
:10576000D60009F0A6FF94F8D70009F0A2FF94F83C
:10577000D80009F09EFF94F8D90009F09AFF073489
:1057800094F8D30009F095FFAC42E0D100F005BCDD
:105790004E4B185D013409F08CFF102CF8D1FCE35E
:1057A0004B4D00242878400000F0FE0009F0B0FFC7
:1057B0002B789C4280F0F183464B33F8140009F0BB
:1057C000AAFF0134F4E7444C062009F0A1FF208829
:1057D00009F0A1FF608809F09EFF404B1888D2E2D3
:1057E000042009F095FF374B186ED4E3072009F029
:1057F0008FFF3B4B1888FF28A8BFFF20C0B209F0DD
:1058000058FF384B186880F3100080B209F083FF0E
:10581000B5F8640009F07FFF264B93F88721324BDF
:10582000186822B10A23584380F3100001E000F306
:105830000F0080B2A7E21F4C022009F069FF94F824
:10584000E20109F036FF94F8E1011AE3022009F0C1
:105850005FFF184B988996E20B2009F059FFAB6E59
:105860000026187809F025FFAB6E587809F021FF63
:10587000AB6E144C33441879013609F01AFF032E2D
:10588000F6D1A36ED87909F014FFA36E987809F0C9
:1058900010FFA36ED87809F00CFFA36E588909F0A9
:1058A0003AFFA36E187AECE2D1970108DD97010860
:1058B000E6970108CC110020E5100020160000201A
:1058C000AE110020DC1000200C110020201100205F
:1058D00064280020702F00206E2E0020BC110020B4
:1058E000AC190020B8190020B4190020C04C1E20AB
:1058F00009F00EFF236C00251B78022B65D1236C69
:1059000005F1080253F82200BA490BF0C5FD0FF06B
:1059100081FD80F30800C0B209F0CBFE236CB649CC
:1059200003EB8503D86A0BF0B7FD0FF073FD80F32E
:105930000800C0B209F0BDFE236C05F10E0253F859
:105940002200AE490BF0A8FD0FF064FD80F30800C3
:10595000C0B2013509F0ADFE032DD0D1072D236C67
:1059600021D1586CA3490BF097FD0FF053FD80F344
:105970000800C0B209F09DFE236C9E49986C0BF0A4
:105980008BFD0FF047FD80F30800C0B209F091FED7
:10599000236C93F84C000BF027FD0FF03BFD80F3D8
:1059A0000800C0B20BE02B44587809F082FE236C4B
:1059B0002B44D87A09F07DFE236C2B44587D0135A9
:1059C00009F077FE0A2DC9D1E7E2236C2B44587801
:1059D00009F06FFE236C2B44D87A09F06AFE236C21
:1059E0002B44587D013509F064FE0A2DEDD1D4E237
:1059F0003C2009F08DFE00247D4D04F108022B6C43
:105A00007E4953F822000BF047FD0FF003FD80B2F2
:105A100009F081FE2B6C794903EB8403D86A0BF003
:105A20003BFD0FF0F7FC80B209F075FE2B6C04F122
:105A30000E0253F8220071490BF02EFD0FF0EAFC24
:105A4000013480B209F067FE032CD5D1072C2B6CF2
:105A500016D1586C69490BF01FFD0FF0DBFC80B2CA
:105A600009F059FE2B6C6549986C0BF015FD0FF091
:105A7000D1FC80B209F04FFE2B6C93F84C000BE088
:105A80002344587809F047FE2B6C2344D87A09F058
:105A900042FE2B6C2344587D013409F03CFE0A2C55
:105AA000D4D17AE214F8010F002800F0768209F0D0
:105AB00000FEF7E7012009F02BFE4D4B1B6C187818
:105AC000DFE1502009F024FE0025494B0C211C6C1D
:105AD0004B4B04EB850494F87920013501FB02332C
:105AE00093F8380009F0E5FD94F87A0009F0E1FD3B
:105AF00094F87B0009F0DDFD94F87C0009F0D9FDF5
:105B0000142DE2D149E23A4B1C6C062303FB0544F9
:105B100094F8CE0009F0CDFD94F8C90009F0C9FD54
:105B200094F8CA0009F0C5FD94F8CB0009F0C1FD56
:105B300094F8CC0009F0BDFD013594F8CD0009F0D2
:105B4000B8FD0C2DDFD128E24FF000080126002718
:105B5000274B1A7A974227DA0933FA5C00240C2380
:105B60006343274D05F13001595C914207D12B4425
:105B7000586B0FF086FA82462EB9B14605E0013423
:105B80001C2CECD10EE080440CE0D1450ADA0C2349
:105B900003FB04535B6B13F8090009F08AFD09F15C
:105BA0000109F2E70137D3E7002E00F0F6815FFA32
:105BB00088F009F0ADFD0026C9E70D4D0024287AD4
:105BC00009F0A6FD2B7A9C4280F0E7810D4B002165
:105BD000E65C0C2202FB01F3094800F13007DA5DB4
:105BE000B24211D1034493F8380009F062FD0EE08F
:105BF000DC100020000020410000C84200007A4470
:105C000008780108E510002001311C29E1D1013498
:105C1000D8E7CE4C162009F07BFDB4F8980109F0C6
:105C20007AFDB4F8440109F076FDB4F8460109F0B4
:105C300072FDB4F8480109F06EFDB4F8DA0109F01C
:105C40006AFD94F8EF0109F034FD002009F031FD00
:105C500094F8F00109F02DFD94F8870109F029FD71
:105C600094F8940109F025FD002009F022FDB84BBD
:105C70000A201B6CB3F9563093FBF0F080B209F0A8
:105C80004AFD89E0E0B2013409F013FD092CF9D195
:105C900083E1102009F03CFDAE4BAF4C187800F0CA
:105CA000020009F006FDAD4B187809F002FD2068EE
:105CB00009F03AFD606809F037FDA94B188809F032
:105CC0002AFDA84B188809F026FDA14BB3F86C00FB
:105CD00059E009F0D1FC0746122009F019FD9C4C4F
:105CE00017B9266F656F05E0102F19BF00252E46E6
:105CF000A66FE56F384609F0DCFC304609F014FD6C
:105D0000284609F011FDD4F8800009F00DFD0020AF
:105D100009F001FD002009F0FEFC0020B1E08C4DEF
:105D2000002495F884002E4680000130C0B209F0AE
:105D3000EFFC95F8840009F0BCFC96F884309C4296
:105D400080F02B81884D285D09F0B3FC05F110032C
:105D5000185D09F0AEFC05F12003185D303509F03F
:105D6000A8FC285D09F0A5FC0134E6E7082009F04D
:105D7000CFFC002009F0CFFC002009F0CCFC002073
:105D800009F0C9FC002009F0C6FC06E1042009F076
:105D9000BFFC6E4B9868FEE094F87C0109F089FC2A
:105DA00094F8800109F085FC94F87F0109F081FCEA
:105DB00094F8810165E0654C072009F0A9FCB4F86E
:105DC000820109F0A8FCB4F8840109F0A4FC94F85D
:105DD000860109F06EFCB4F88801D4E75B4C0C2016
:105DE00009F096FC94F8920109F063FCB4F89C0168
:105DF00009F091FCB4F8980109F08DFCB4F89A010F
:105E000009F089FC94F8930109F053FCB4F89E0161
:105E100009F081FCB4F8A001B5E74C4C042009F06E
:105E200077FC94F8D80109F044FC94F8D90109F002
:105E300040FCB4F8DA01A6E74C4C4D4D2078002622
:105E400000EB4000C0B209F063FC237802359E42AB
:105E500080F0A38015F8020C09F02BFC15F8010C5A
:105E6000013600EB800000EB800000F2EE2080B2F3
:105E700009F051FCE9E7012009F04AFC334B93F8A3
:105E8000940109F016FC88E0082009F041FC002488
:105E90002E4B234493F88A01013409F00AFC082CA4
:105EA000F6D17AE02A4B294C93F8C50004F120057D
:105EB000C0EBC000C0B209F02BFC94F8F60100233F
:105EC0002C4AD25C90426ED00C33302BF8D108347F
:105ED000AC42F2D161E0402009F01AFC1B4C04F105
:105EE0004005B4F8A80209F016FC94F8AA0209F0DB
:105EF000E0FB043494F8A70209F0DBFBAC42F0D1DC
:105F00004BE0E02009F004FC104C04F18005B4F8EB
:105F10002A02043400F03F0009F0FDFBB4F8260229
:105F2000C0F3861009F0F7FB94F82402000909F089
:105F3000C0FB94F8240200F00F0009F0BAFB94F8BB
:105F4000250209F0B6FBAC42E1D126E0CC110020DD
:105F5000DC100020C0190020C8190020C61900203C
:105F6000C4190020C21900206111002064280020FB
:105F70006E13002070280020132009F0C9FB0024B4
:105F8000144B185D013409F094FB0B2CF8D1002060
:105F900009F0CAFB002009F0C7FB0120BDE8F0872B
:105FA0000020BDE8F08709F084FBB4F8F80109F09F
:105FB000B2FB94F8FA0109F07CFB94F8FB0109F0BC
:105FC00078FB94F8FD0109F074FB94F8FC0109F0EA
:105FD00070FB7CE7D19701082DE9FF47CC4C0746C1
:105FE0002378CC4E002B00F0018232686368D31A0C
:105FF0007C2B40F2FB81237A6260013323724FF0E5
:10600000000808F12400C24DC0B20AF0F3FD05F10A
:106010000A0333F918000BF0EBF9BF4B81461888DF
:106020000BF0E6F9014648460BF0EAFABB490BF0E3
:1060300033FA0BF0F7FB08F1010800B20AF0C8FDD3
:10604000B8F1030FDDD130200AF0D4FDB5F910000E
:106050000AF0BEFD0AF0C6FD2B7A9A072CD141F258
:1060600088336A689A4218D910200AF0C3FD68691B
:106070004FF0640890FBF8F000B20AF0A9FD21206F
:106080000AF0B8FD686990FBF8F308FB13000028DC
:10609000B8BF404200B20AF09BFD14200AF0AAFDEE
:1060A000B4F918000AF094FD1C200AF0A3FD0020AA
:1060B0000AF08EFD0AF096FD237ADFF854825B0722
:1060C00040F0718102200AF095FDD8F81C0064238D
:1060D000323090FBF3F000B20AF07AFDB8F92650A6
:1060E0004FF0050A95FBFAF503200AF083FD8C4B6F
:1060F000ADB21B78DFF83C9213F0040F0DD008F519
:10610000D970394602F009F928B9D9F8003013F0EE
:10611000100F18BF002528B205E0D8F80438988978
:10612000B0FBFAF000B20AF053FDD9F800309F0737
:1061300040F18780DFF80092B4F8082899F8003021
:106140004FF0640808FB02325B00B2FBF3F3B4F8D3
:106150000A7806203F01BFB247EA0327BFB2C3F364
:1061600003231F430AF046FD38B20AF031FDB4F8AC
:106170000A3899F8001001339BB293FBF1F201FB4E
:106180001233A4F80A38D4F80C38614D9B7B012BEC
:1061900005D139200AF02EFDB5F908081AE0B5F846
:1061A00008586E235D43152795FBF7F53A20AFB2EB
:1061B0000AF020FDB7FBF8F528B208FB15750AF0C8
:1061C00007FD3B200AF016FDA8B2451D0A2095FBED
:1061D000F0F000B20AF0FCFC28200AF00BFDD4F825
:1061E00010380A2093FBF0F000B20AF0F1FC042012
:1061F0000AF000FDD4F80438454F9D894FF6FF732F
:10620000D7F814089842A8BF1846ADB10028ACBF13
:10621000281A28460BF0ECF842490BF03DF90746E6
:1062200028460BF0E5F8014638460BF0E9F90BF08B
:10623000F9FA6428A8BF642020EAE07000B20AF0EE
:10624000C7FCD4F81838324F9D0640F1A18097F86A
:106250001C3898071DD511200AF0CCFCB7F81E0891
:106260004FF4F3656843304B90FBF3F000B20AF053
:10627000AFFC19200AF0BEFCB7F81E0845436420A5
:1062800095FBF0F595FBF0F300FB135000B20AF01C
:106290009FFC94F81C38B4F8205813F0020F08BF84
:1062A000002501200AF0A6FC28B20AF091FC092082
:1062B0000AF0A0FC00200AF08BFC1C4B94F822583A
:1062C0001A88B2F5967F0AD9114B1B7A03F00F0397
:1062D000072B04D842F20F75954228BF15460520BA
:1062E0000AF088FCD4F80C385B7B0BB928B22DE09F
:1062F000A5F120000BF07CF80D490BF081F900218D
:1063000005460BF067FAC8B94FF07C5118E000BFA2
:10631000A41100209C2E00201600002000007A44CA
:10632000973000200000C842A08601003E000020F7
:106330006666E63F782E00203C0000204FF03F418B
:1063400028460AF0A1FF0BF06DFA00B20AF040FCFB
:1063500094F81C28C74B910703D493F82328012AEB
:1063600004D1012384F82338C34818E0D3F80C582B
:10637000C24968680BF090F80BF054FABF490290DC
:10638000A8680BF089F80BF04DFA039002A806E01C
:10639000BB4A02AB92E8030083E8030018460AF008
:1063A00039FC0AF01FFC237A282B1FD1B14B0022A5
:1063B0001A7233684FF47A70B3FBF0F83C27172059
:1063C0000AF018FCB8FBF7F5B5FBF7F007FB105027
:1063D000000200B20AF0FCFB18200AF00BFC07FBDD
:1063E000158000B20AF0F4FB0AF0FCFB94F82C389C
:1063F000A04D002B00F0638102F01CF8D5F8303876
:10640000A04AC31A9342074640F2C780002385F88A
:10641000363885F83838B5F80838DAB21B0A85F806
:10642000522885F8533885F8482885F84938D5F832
:10643000602833689A1AD5F86438D97B4FF47A7398
:106440004B439A420ED3904B1B68C5F8603895F8C1
:106450006838013B012B9FBF102385F83638022393
:1064600085F83838D4F810280A20D4F8143892FB6C
:10647000F0F293FBF0F384F85028121284F85128BC
:1064800084F8543894F81C281B1284F8553894F872
:1064900022389207774984F8833803D42D2381F872
:1064A000843878E0D4F824987848DFF8ECC199FB78
:1064B000F0FA0CFB0A924FF0060E042B0EFB02F2D0
:1064C0008CBF3323322381F88438714BD4F8286889
:1064D00092FBF3F196FBF0F003FB1122642592FB93
:1064E000F5F20CFB006C0EFB0CFE84F87528121202
:1064F00084F876289EFBF3F203FB12E393FBF5F39B
:106500000AEB8A0A4FFA81F80AEB8A0A08EB8A0139
:1065100089B284F8731800EB8000090A84F87418B3
:1065200000EB800051B201EB800292B284F878282F
:10653000120A84F8792884F87A38B4F81E281B12D5
:1065400084F87B382423534393FBF5F5B4F896384D
:106550000A2284F87C381B0A84F87D38B4F8203885
:106560004FEAD979B3FBF2F303F5FA739BB284F8DF
:106570007E381B0A84F87F38B4F89838F60F84F810
:106580007058C5F3072584F8729884F8776884F802
:10659000715884F88538C4F8307894F89A88354D65
:1065A000B8F1000F0DD1D5F8A00807F0C4FE0128FE
:1065B00007D90228374E00F0608202F067FD012300
:1065C000B370D4F8A4282B4D002A78D095F89A6897
:1065D0003EB140F6B731D5F8AC38FB1A8B4219D82A
:1065E0006DE00123D5F8A00885F89A3801F00AFD7E
:1065F000D5F8B038082193F9000002238DE848004F
:1066000032464FF4964301F082FF85F8B468C5F82E
:10661000A00852E095F8A868CEB9D5F8A008C5F84A
:10662000A46885F89A6801F0EDFCD5F8B038082127
:1066300093F9000001238DE8480032464FF4964359
:1066400001F065FFC5F8A00802F020FD35E0013E2D
:10665000F6B285F8A86895F8B41895F8B538EEB98B
:106660004A1C013385F8B42885F8B538D5F8A00858
:1066700021E000BFA4110020C81900208096184B0B
:10668000947901083F0D03009C2E0020809698000D
:1066900040420F0016000020806967FF12F8016B6E
:1066A00001337018314685F8B408D5F8A008C5F84C
:1066B000A42885F8B53807F041FEC4F8AC7894F802
:1066C000B638A14DF3B1D5F8B838DBB1D5F8BC3840
:1066D000C3B1C5F8C0381B689C4AC5F8C438D5F8A2
:1066E000C8381344187AFEF74DFDD5F8C0389879AC
:1066F00008F0DFFFD5F8C8380133092B88BF002325
:10670000C5F8C838924D94F8CC282E688E4B002AD4
:1067100000F0EE81D3F8D028002A00F0E98193F848
:10672000D438013B012B00F2E381D4F8D008864F26
:1067300007F001FEE0B1D7F8D00807F0F9FD97F8AF
:10674000D53880467E2BD5F800900ED102231B2829
:1067500087F8D43809D1D7F8D00807F0ECFD20B974
:106760000123C7F8D89887F8DC3884F8D588DCE7A7
:10677000D7F8D8282B689B1A41F6583293421ED975
:10678000032387F8D438B3E1724A32F8130010B902
:1067900003464FF403600133B0F5C06FDBB279D02C
:1067A0001ED9B0F5006F7FD032D9B0F5036F3FD15D
:1067B00084F8DD38D4F81838634F99063FD494F83C
:1067C000DC1894F8DD38002900F054812A68921B07
:1067D000012AD9D984F8DD38002384F8DC3887E130
:1067E000B0F5007F43D007D8B0F5807F49D0B0F531
:1067F000887F00F08B80E6E7B0F5806F00F0AE8018
:10680000B0F5826F00F0F380B0F5047FDBD123E0B8
:10681000B0F5E26F00F08B80B0F5E46F00F08C8093
:10682000B0F5E06FCFD184F8DD38B4F90A1087E015
:10683000B0F5046F74D0B0F5026FC4D103E197F8DE
:106840001C389A07BBD5B7F81E1824234B43642184
:10685000123393FBF1F107E184F8DD383E4B3A4FF8
:106860001B689B07ABD5B7F808380A21FBE084F812
:10687000DD38394B344F1B681905A0D5D7F81018EF
:10688000F2E084F8DD38D4F818382F4F5A0796D53F
:106890007969E9E084F8DD382F4B2B4F1B681B0525
:1068A0008DD5D7F81418DFE0D4F81818264A8F06CB
:1068B00084F8DD3883D592F81C1888077FF57FAF00
:1068C000D90711D5D2F82838192283EAE371A1EB50
:1068D000E37101EB5101B1FBF2F1002BACBF41F0D0
:1068E000004141F040410EE0D2F82438192283EAF9
:1068F000E371A1EBE37101EB5101B1FBF2F1002B6C
:10690000B8BF41F080414FF400608BE084F8DD387F
:10691000D4F818380C4F5B077FF551AF3969A3E005
:1069200084F8DD38B4F91830642159437AE084F8EA
:10693000DD38B4F90C1003E0B4F90E1084F8DD383A
:106940002C2391FBF3F16DE0A41100209479010850
:106950009C2E0020D4980108782E002084F8DD3881
:1069600094F8DE38644A0133DBB2032B88BF01237D
:1069700082F8DE3842F2107394F8DE1859435F4B08
:106980001B78D80748BF01319A0748BF02315F071B
:10699000B4F8E03848BF0431D80748BF0A319A0735
:1069A00048BF14311F0648BF2831D80548BF2831D9
:1069B0005A0748BF64311F0748BFC831980548BF10
:1069C00001F5C8719A0648BF01F57A71DF0648BF24
:1069D00001F5FA61580648BF01F57A614FF480600D
:1069E00002F020FB444B002283F8DC28E7E6D4F8D1
:1069F0001818DFF8048111F0200784F8DD3817D06B
:106A000098F81C2812F0020F14BF4FF47A7100217D
:106A100012F0010F14BF4FF4FA6300230B4494F8F3
:106A20002218194402F0FEFA002384F8DC38C6E686
:106A3000334B1B6819067FF5C2AE394602F0F2FAF5
:106A400088F8DC78BBE684F8DD38D4F818382A4FAB
:106A50009A067FF5B4AE97F81C389B077FF5AFAE6A
:106A6000B7F820386421594302F0DCFA002387F894
:106A7000DC38A4E684F8DD383AE0B37823B1C5F811
:106A80009C7886F802809CE5D5F89C38FB1AB3F513
:106A90007A6FFFF496AD0123D5F8A008B37007F024
:106AA00047FC0646D5F8A00807F042FC76067FF4BE
:106AB00088AD8A2802D08E280DD082E5D5F8183806
:106AC00098067FF57EAD95F89A38002B7FF479AD66
:106AD00005F6690306E095F89A38002B7FF471AD4E
:106AE00005F63403C5F8A4382D2385F8A83868E5E1
:106AF00004B0BDE8F08700BFA4110020973000204B
:106B0000782E0020F0B50124B0FBF4F58D4201D3BE
:106B10004C43F9E70026D4B1B0FBF4F504FB1500B3
:106B2000B4FBF1F41EB9002D01DC002CF3D1092DCA
:106B300003F1010EEFB204DD002A14BF37255725FB
:106B400000E030253D441D7001367346E3E71C70BC
:106B5000F0BDF0B50124B0FBF4F58D4201D34C43F8
:106B6000F9E70026D4B1B0FBF4F504FB1500B4FB43
:106B7000F1F41EB9002D01DC002CF3D1092D03F135
:106B8000010EEFB204DD002A14BF3725572500E0BF
:106B900030253D441D7001367346E3E71C70F0BD9F
:106BA00003685A1C0260197070472DE9F843089E6B
:106BB000002B074688461446334614BF4FF0300971
:106BC0004FF0200913F8012B0AB9254603E0002CE9
:106BD000FBDD013CF6E7002D04DD38464946C047A1
:106BE000013DF8E7354624EAE474A01B284415F873
:106BF000011B11B13846C047F7E7BDE8F883024BE7
:106C0000186807F09BBB00BF98100020F8B5074636
:106C10000C464868002115461E460AF0D1FD58B1C1
:106C200028460AF0E5FB10490AF036FC01464FF011
:106C30007E500AF0E5FC6060616830460AF024FB93
:106C4000014630460AF0DCFC2568064629463846EF
:106C50000AF018FB014630460AF01EFC01462846A1
:106C60000AF012FB2060F8BDDB0FC9402DE9F041AE
:106C700002780346202A00F10100F9D0092AF7D052
:106C80002D2A02D10346414D04E02B2A08BF0346BA
:106C90004FF07E551C460026234614F8012BA2F126
:106CA0003007F9B209290DD8394930460AF0F4FB0A
:106CB000064638460AF09CFB014630460AF0E4FAE4
:106CC0000646E9E72E2A17D1314F234614F8010B67
:106CD0003038C2B2092A0FD80AF08AFB39460AF0C6
:106CE0008FFC014630460AF0CFFA2949064638465D
:106CF0000AF0D2FB0746E8E71A7802F0DF02452ADD
:106D000039D15A782D2A02D10233012704E02B2AE7
:106D100014BF013302330027013B002413F8012F75
:106D2000303AD1B2092903D80A2101FB0424F5E73E
:106D3000B4F59A7F28BF4FF49A74A0464FF07E5363
:106D4000B8F1070F07D9184612490AF0A5FBA8F1B8
:106D500008080346F4E704F0070434B118460C4968
:106D60000AF09AFB013C0346F7E719462FB130467B
:106D70000AF046FC04E04FF07E5130460AF08CFBEE
:106D8000014628460AF088FBBDE8F081000080BF7C
:106D90000000204120BCBE4C30B5054687B00C46F3
:106DA00003A800210C220EF028F9284600210AF041
:106DB0002FFD20B1284628490AF066FA03E028464C
:106DC00025490AF05FFA25490AF066FB0AF02AFD18
:106DD000054680EAE0706946A0EBE57006F086FAA9
:106DE000002DACBF20232D2368468DF80C300EF00B
:106DF00048F9012807D130238DF80D308DF80E3079
:106E00008DF80F300CE0022805D130238DF80D30BD
:106E10008DF80E3004E0032804BF30238DF80D30C8
:106E2000694603A80EF010F903A80EF02AF90338FA
:106E3000C5B22A4603A920460EF04EF90023635539
:106E4000204607490EF000F903AB204659190EF011
:106E5000FBF8204607B030BD6F12033A00007A44B9
:106E6000F498010870B50646B6FBF2F408461546DC
:106E700014B12046FFF7F6FF05FB1464024B1B5DBF
:106E800000F8013B70BD00BFF69801082DE9F04FF6
:106E900081468A4616461C4689B00025317800296D
:106EA00000F0DB80252902D00136484674E0727874
:106EB0004FF00008302A0CBFB278B71CA2F13003A3
:106EC00012BF4FF0000BF71C4FF0010B092B19D824
:106ED000A2F13003D9B2092905D80A2202FB0838E9
:106EE00017F8012BF4E7A2F16103052B02D8A2F1F8
:106EF000570305E0A2F14103052B03D8A2F13703A4
:106F00000A2BEADD6C2A30D13A787E1C642A00F024
:106F100083800BD8252A3DD003D8002A00F09D801D
:106F2000BCE7582A0CD0632A19D0B7E7732A22D0BD
:106F300002D86E2A37D0B1E7752A5CD0782AADD155
:106F4000271D2068A2F1580462424FF010016241EF
:106F500055E02CD9582A32D0632A2AD13E464846D9
:106F60002178271DD04701350FE0642A63D00ED960
:106F7000732A14D13E462368484600935146424640
:106F80000023FFF712FE271D05443C4686E7252A0D
:106F9000DFD13E4648462521D04701357EE70AD855
:106FA0006E2A06D13E46236804341D6076E7002A27
:106FB00053D03E4672E7752A26D0782AF9D1A2F13D
:106FC000580304F1040C5A422068CDF80CC04FF06D
:106FD00010015A4105ABFFF795FDDDF80CC03E46A8
:106FE000644605AB00934846514642465B46FFF770
:106FF000DCFD054452E72068271D0A21002205AB6D
:10700000FFF7A7FD3C46ECE704F1040CCDF80CC0FB
:1070100020680A210022DDE72068271D002808DA01
:107020002D238DF8143040420DF115030A21002262
:10703000E6E705ABFAE7206804F1040C00280ADA59
:107040002D238DF8143040420DF11503CDF80CC0FE
:107050000A210022BFE705ABF8E7284609B0BDE8E2
:10706000F08F0FB413B50B4904AB08680A4953F805
:10707000042B09680193FFF709FF0446074B1868C2
:1070800001F08EFA0028F9D0204602B0BDE8104089
:1070900004B07047A4090020A00900209810002027
:1070A00080EAE073A3EBE0738B4206DB002801DD8E
:1070B000401A704702D0084470470020704770B5EE
:1070C00004460AF0AFFB2030402857D820462C4910
:1070D0000AF09EFB28B120462A490AF0D3F804465C
:1070E000F4E7204628490AF075FB28B120462549D7
:1070F0000AF0CAF80446F4E7204624490AF088FB5F
:1071000030B1224920460AF0BDF801461F480AE086
:1071100020461F490AF05EFB40B11C4920460AF098
:10712000B3F801461A480AF0ADF804462146204655
:107130000AF0B2F90546204629460AF0ADF915498C
:10714000064628460AF0A8F913490AF09BF80146BA
:1071500028460AF0A1F911490AF096F80146284696
:107160000AF09AF90E490AF08DF8014630460AF005
:1071700093F9014620460AF087F870BD002070BDE3
:10718000DB0F4940DB0FC940DB0F49C0DB0FC93FB4
:10719000DB0FC9BF9A7C2E36FAAF4F393587083CD2
:1071A000A4AA2A3E08B503490AF06EF8BDE80840D3
:1071B00085E700BFDB0FC93F2DE9F04F056885B0BB
:1071C000814628460C46FFF7EDFF80462846FFF72C
:1071D00076FFD9F8045006462846FFF7E3FF074636
:1071E0002846FFF76CFFD9F8089005464846FFF798
:1071F000D9FF82464846FFF762FF41468146504626
:107200000AF04AF94146834648460AF045F9514694
:10721000019030460AF040F94946029030460AF0A3
:107220003BF93946039050460AF036F9494620604A
:1072300007F100400AF030F929466060A560029825
:107240000AF02AF9014601980AF01EF82946E06082
:1072500003980AF021F9014658460AF013F8394616
:10726000206106F100400AF017F92946606158468E
:107270000AF012F9014603980AF004F82946A061C1
:1072800001980AF009F90146029809F0FDFF41460C
:10729000E06138460AF000F9206205B0BDE8F08FE1
:1072A0002DE9F04107688AB04668856804460846BB
:1072B00001A9FFF781FF019938460AF0EDF804991A
:1072C000804630460AF0E8F80146404609F0DCFF07
:1072D0000799804628460AF0DFF80146404609F043
:1072E000D3FF0299206038460AF0D6F80599804607
:1072F00030460AF0D1F80146404609F0C5FF08992A
:10730000804628460AF0C8F80146404609F0BCFF0E
:107310000399606038460AF0BFF806990746304680
:107320000AF0BAF80146384609F0AEFF0999064658
:1073300028460AF0B1F80146304609F0A5FFA060E2
:107340000AB0BDE8F081074B10B51A881C4622EA46
:1073500000009042188002D0012001F053F82088EC
:1073600010BD00BF841A0020064B10B51A881C46B9
:1073700010439042188002D0012001F043F8208889
:1073800010BD00BF841A0020024A936823EA00005F
:1073900090607047CC11002008B5104B1A7800237C
:1073A000D9B2914207D20E49002051F8231001337F
:1073B00009680880F4E7322001F063F8094B1B6884
:1073C0005A0309D5084B9B685B0305D4BDE8084008
:1073D00040F2DC5001F055B808BD00BF2F2A002054
:1073E000302A0020782E0020CC1100202DE9F34116
:1073F00009F0FAFE4B4A6923137040F2DC735380A4
:10740000BE231371EF2382F8D9370023194616469D
:1074100082F8DA37F25C0133514040F2DC72934279
:10742000F8D1404B404A83F8DA17404B04275A60A2
:1074300002F188325A600020013F17F0FF075ED04A
:107440003A4B34223A4CDA6004F17848A8F5FC381B
:10745000C8F3090353B100234FF4005056F80880D5
:10746000019306F0B5F80428E6D11CE04FF4302073
:1074700006F0AEF80428DFD12C4D4FF430202B69F4
:1074800043F002032B616C612B6943F040032B61D5
:1074900006F09EF841F6FD732A69042803EA020308
:1074A0002B61D8D0C8E7214D4FF400502B6943F031
:1074B00001032B611FFA88F3238006F089F8042862
:1074C00013D1A31C0193019B4FEA1848A3F8008035
:1074D0004FF4005006F07CF841F6FE732A69042848
:1074E00003EA02032B6106D0A6E741F6FE732A6980
:1074F00013402B61A0E70F4B04349C42A4D10B4AEC
:107500000428136943F08003136102D108F08EFB55
:1075100010B9052000F0BFFF09F050FE02B0BDE831
:10752000F08100BFCC1100202301674500200240FC
:1075300000F80108DCFF010810B50E4C206800F0CF
:107540009DFE20680022047A02FB02F3193B63438C
:1075500003F6C4135343192193FBF1F3064921F8B1
:1075600012300132072AEFD1BDE81040034900F084
:107570003DBE00BF44110020681000201013002001
:107580002DE9F04108F052FB10B9042000F083FF10
:10759000BF4C09F029FEBF4940F2DC7220460DF0D5
:1075A00021FD94F8B0374FF4CC71022B84BF002337
:1075B00084F8B03794F8B027B74D01FB02F303F518
:1075C0003A7020442344286093F83C0301FB0242B4
:1075D000022803F54E7384BF0020187192F83C33E3
:1075E000AE4A13700C2202FB0343AD4A03F2B2739E
:1075F000136046F20902A3681A401AB9A44A43F478
:1076000000539360A368DE0703D54FF40050FFF7E3
:10761000BBFEA368580409D50820FFF7B5FE4FF458
:107620000050FFF7B1FE0120FFF7AEFEA368190777
:1076300006D54FF40050FFF7A7FE0120FFF7A4FE88
:10764000A3689A0413D54FF40040FFF79DFE904BBA
:1076500093F88631012B03D14FF40060FFF794FEBD
:107660004FF48030FFF790FE4020FFF78DFEA368B7
:107670005B0603D54FF48030FFF786FE894B1B680D
:1076800003F42063B3F5206F07D194F88631012B02
:1076900003D14FF40060FFF777FE94F8E0217C4BB4
:1076A0002AB193F8E42112B1002283F8E4214FF0CB
:1076B000000C67467C4E7D4B1E6004EB0C03B3F858
:1076C000F8E14FEA5E0101F077314FEA9E0303F0E3
:1076D0003333C1EB0E00C11A4FEADE0303F011335E
:1076E000CB1A03EB231303F00F32FF2392FBF3F3C8
:1076F0001EF00108C3EB032318BF0137A2EB0303FD
:1077000018BFFFB2012B0ADD022B40F0BE80B8F19A
:10771000000F00F0BA801EF0BC0F00F0B6800CF134
:10772000080CBCF1200FC8D1013F012F00F2AD8041
:10773000FFF702FF302200215D480DF05EFC5D4F37
:107740005D4BD5F800801F605C4B002108F179008B
:10775000C3F8008000F0D0FD594B80F00100187094
:10776000584B07F126021A60574B07F1D4021A60F2
:1077700098F8000007F04EF82868544B00F5C572E1
:107780001A6002F0B5F8524B94F8D81107F1940240
:107790001A6064224A434F4BC8325A6000229A60F2
:1077A000DA601A615A619A61DA6183F8202083F8FD
:1077B0002120494B2D6807F12C021A60474B05F236
:1077C00019121A60464B05F289121A60454B07F1EF
:1077D00008021A60444BDFF84C811F60434B07F1ED
:1077E000A0021A6007F1AA03C8F80030404BB4F8B1
:1077F00066011E6009F0F8FDC8F80800B4F86801D9
:1078000009F0F2FD95F85C3008F1040288F80430C4
:1078100095F87830C8F80C0088F8053094F8E33112
:10782000286E88F81030334BC8F814501A60324B69
:1078300005F164021A60314909F02EFE01464FF04D
:107840007C5009F0DDFEB5F816412D4B186020463E
:1078500009F0CEFD01462B4809F0D2FE2A4909F075
:107860001BFE2A4A2A4B15602A4A186005F1680354
:107870001360294A05F211151560284A1760284A35
:10788000BDE8F041136009F099BC05F0E7FC4FE753
:10789000CC11002000F801081C110020582C0020F9
:1078A00044110020782E0020561300203C30002088
:1078B0009C0F002010130020D00F0020D40F0020B8
:1078C0001500002070020020B40E0020E00F002000
:1078D0007827002048300020C8020020601D0020CA
:1078E000D0040020002B0020042B0020E403002003
:1078F000A8040020F802002030030020DB0F4940DC
:107900002C030020000061444C3D0F44380200204D
:10791000E00300202C020020D0030020D803002028
:1079200024010020881A002008B5FFF75FFDFFF74B
:1079300027FEBDE80840012000F064BDF8B504460C
:107940000E4617460025204620210DF08CFB0446EC
:10795000D0B1013420460DF0E9FBB0F5617F05DBC5
:1079600040F634039842A8BF184601E04FF4617016
:10797000A0F56170192390FBF3F00DB9307000E0B1
:1079800070703B7801333B700DB90125DBE7204671
:10799000F8BD30B505460C46134629462246BDE8DB
:1079A00030400148FFF75DBBEC9901087FB50478D2
:1079B0000646E4B9354B1921186800EB840090F8AD
:1079C0007B5090F879204D4305F5617590F87A3039
:1079D000009590F87C00414301F5617101912C48BC
:1079E00021460134FFF73DFB142CE3D14BE00DF0B1
:1079F0009DFB1328054641DC244B701C1C6820218C
:107A000000238DF80F300DF02EFB1E35064670B1A9
:107A1000013630460DF08AFB1A289FBF04EB850320
:107A200058709DF80F30013398BF8DF80F303046F5
:107A300020210DF018FB064670B1013630460DF0DE
:107A400075FB0D289FBF04EB850398709DF80F30E0
:107A5000013398BF8DF80F3004EB85043046E11CEC
:107A60000DF10F02FFF76AFF9DF80F30042B0AD0CB
:107A7000601C002104220DF0C0FA04E0054800213A
:107A80001322FFF786FF04B070BD00BF1C11002059
:107A90000B9A0108209A0108014807F0BDBE00BFFB
:107AA000269A0108F8B50478064674B9304D214687
:107AB000B5F8C621B5F8C8312E480134FFF7D1FA20
:107AC000042C05F10405F2D1F8BD2B490DF09EFA06
:107AD000A8B9274B4FF47A714FF4FA62A3F8C61194
:107AE000A3F8C821A3F8CA11A3F8CC21A3F8CE119A
:107AF000A3F8D021A3F8D211A3F8D421F8BD3046C1
:107B00000DF014FB032805462BD8304620210DF03C
:107B1000AAFA044630B1013420460DF007FB0126D5
:107B2000074600E00646204620210DF09CFA10B9D9
:107B3000BDE8F840B0E701300DF0F8FA012EF7D1BA
:107B400040F2DC53A7F2EE229A42F1D8A0F2EE22E4
:107B50009A42EDD8064B703503EB8503DF80188120
:107B6000F8BD064800210322BDE8F84011E700BF38
:107B7000CC110020349A0108479A010864A7010833
:107B80002DE9FF4104780546002C34D16D4807F0FB
:107B900043FE6D4D6869002109F012FE002840F097
:107BA000CE8021466948FFF75CFA68696946FFF7AD
:107BB000F3F801466648FFF754FAA8696946FFF7EB
:107BC000EBF801466248FFF74CFAE8696946FFF7AF
:107BD000E3F801465E48FFF744FA286A6946FFF772
:107BE000DBF8013401465B48FFF73BFA0C2C05F14A
:107BF0001005CFD1A3E0584905220DF04BFA38B952
:107C0000514B002203441030C0285A61F8D196E04D
:107C10002846524904220DF03DFA04462846002C1D
:107C20003FD120210DF01FFA002800F08880451C6C
:107C300028460DF026FA0746494B53F824601EB932
:107C4000484807F0E9FD7AE028463146FAB20DF0DF
:107C500021FA01340028EFD13B4B0021C21810302B
:107C6000C02851619E46F7D13F4B03EBC402D2F8C6
:107C700004C09846BCF1000F04D131463B48FFF7E1
:107C8000F0F953E0002718F834309F42F5DA3B0151
:107C90000EEB0305143563440FCB013785E80F0065
:107CA000F1E70DF043FA0B28064643DC2846202175
:107CB0000DF0D9F9054648B101352846FEF7D6FF43
:107CC000214B012403EB0613586100E004462846CB
:107CD00020210DF0C8F9054640B101352846FEF7D0
:107CE000C5FF194B013403EB061398612846202188
:107CF0000DF0B9F9054640B101352846FEF7B6FF4B
:107D0000114B013403EB0613D861284620210DF0F6
:107D1000AAF910B9FFF7C0FE11E00130FEF7A6FF87
:107D2000094B032C03EB06163062F3D11048FFF722
:107D300027FF04E00F4801210C22FFF72AFE04B0C0
:107D4000BDE8F0814D9A0108CC110020689A010825
:107D50006E9A010878A40108479A0108729A0108EE
:107D6000E4930108779A01081C990108869A010892
:107D700098970108209A0108F0B5047887B0064664
:107D800014BB514B19201968062303FB041191F809
:107D9000CA5091F8CE20454305F5617591F8C93078
:107DA000009591F8CB50C831684300F5617001909F
:107DB0000879029049794548039121460134FFF73B
:107DC00050F90C2CDDD17CE00DF0B0F90B28044605
:107DD00072DC3D4B701C1D68202100238DF817308C
:107DE0000DF041F9064680B1013630460DF09EF99E
:107DF00003289FBF062303FB045383F8CE009DF89E
:107E000017309CBF01338DF81730304620210DF01C
:107E10002AF9074680B1013738460DF087F90D2859
:107E20009FBF062303FB045383F8C9009DF8173056
:107E30009CBF01338DF8173006266643A9193846D2
:107E4000CA310DF11702FFF779FD20210DF00BF972
:107E5000074670B1013738460DF068F914289FBF06
:107E60009DF817307619013386F8CC0098BF8DF84D
:107E70001730384620210DF0F6F878B101300DF0BA
:107E800055F90D289FBF062303FB045383F8CD004B
:107E90009DF817309CBF01338DF817309DF81730CF
:107EA000062B0ED0062202FB04500021C9300DF033
:107EB000A4F8FFF7F1FD04E0054800210B22FFF7CD
:107EC00068FD07B0F0BD00BF1C110020929A0108A8
:107ED000209A01082DE9F347047806464CB920465C
:107EE00001A905F003FA0134FFF7F4FF122CF6D1D3
:107EF0007AE00DF01BF9C5B2112D70D83C4C05F19C
:107F0000D00704EB4703701C202193F802800DF08A
:107F1000AAF8384E034630B9A8F10202D2F100089F
:107F200048EB020845E000F1010A597830460DF0AF
:107F30009AF860B1032D8CBF03230023801BC0B2CD
:107F40003344184490F80490B9F1030F02D1FFF7BD
:107F5000A3FD49E0A9F10203D3F1000850464FF018
:107F6000200148EB03080DF07EF8D8B1B8F1000FFE
:107F7000EDD001300DF0DAF840F2ED2380B29842F6
:107F800005DD40F6CA039842A8BF184601E040F25A
:107F9000EE20A0F2EE20192290FBF2F004EB470352
:107FA000D87002E0B8F1000FD1D104EB470383F899
:107FB000029004EB4704A378F25CB8F1000F09D0FB
:107FC000E17819234B430C48294603F2EE23FFF7CF
:107FD00048F809E029460948FFF743F804E0084853
:107FE00000211122FFF7D5FC02B0BDE8F08700BFE9
:107FF000CC110020A8790108B29A0108C49A01089E
:1080000064A70108002208490C2303FB02135968E6
:10801000814204D10022C2621A725A607047013252
:10802000042AF0D1704700BF7028002010B5084B1B
:108030000022196801EBC20393F90240844201D186
:10804000981C10BD0132042AF4D1002010BD00BFDD
:108050006C280020F0B5027887B08AB94A4C04F148
:10806000200694F8F6210023484950B2595681421F
:108070006DD00C33302BF7D10834B442F1D180E00D
:10808000002204920592451C0DF050F8C4B260B273
:10809000FFF7CCFF074618B18DF81040012400E02F
:1080A0000446284620210CF0DEFF054638B1013594
:1080B00028460DF03BF80134ADF81200E4B200267A
:1080C000284620210CF0CFFFB0B3451C28460DF008
:1080D0002DF800222E495FFA82FE51F822308342A9
:1080E00004D00132082AF5D1002300E0734651F88C
:1080F0002320824220D1022E0FD0032E12D05A1EEE
:10810000012ED2B204D0042A13D88DF814300EE018
:10811000042A0ED88DF8153009E0052B09D88DF802
:10812000173004E09A1E052A03D88DF81630013462
:10813000E4B20136042EC3D1052C03D807B0BDE844
:10814000F040A9E404AB03CB3860796019E094F8FF
:10815000FB010F4B94F8FA5153F82000B4F8F821C2
:10816000009094F8FD0153F82000019094F8FC0170
:1081700053F8200053F8253002900648FEF771FFAF
:108180007AE707B0F0BD00BFCC11002070280020B6
:108190009C820108D39A010838B1438811EA030090
:1081A00003D08B420CBF01200220704730B50A4B30
:1081B0000A491C680A78032A0AD81346551C04EB9E
:1081C000C303EAB29D882842F5D00A70981C30BDDE
:1081D0000A70002030BD00BF6C280020A01A0020CB
:1081E000014B00221A70E1E7A01A00202DE9F047A8
:1081F000877890F803C0BBB2C7F1640E03EB830627
:108200005C42C3F178001C4D5FFA8EFE7600CCF123
:108210006408A4B280B2A3B20FFA83F9B9F1000FD7
:1082200004DC002B14BF3B46012300E0734609FB2E
:1082300009F25B4302FB0CF292FBF3F3434403FBB2
:1082400009F30A2293FBF2F333449BB225F8023F71
:10825000B1F800904A880A34C9EB020A1AB202FB4C
:108260000AF24FF47A7392FBF3F3A4B24B448442C4
:108270002B80D0D1BDE8F087A01A002010B544783B
:108280000078002240F6C41102FB02F3193B63435D
:1082900003F6C4135343434393FBF1F3034921F81B
:1082A00012300132072AEDD110BD00BFBA1A0020EA
:1082B000104B043033F91000B0F5617F05DB40F658
:1082C00033039842A8BF184601E04FF461700A7862
:1082D00019235A4302F28332824208DA4A7853431E
:1082E00003F283338342B4BF002001207047002093
:1082F000704700BF702F002010B500F150030278C6
:108300008A4203D18478C278944204D304309842DC
:10831000F5D1002010BD012010BD0B4B1B6813F4DC
:10832000805F0A4BB3F9063005D0C089421A9342E8
:1083300007DD084400E0008A8342B4BF002001202A
:1083400070470120704700BF782E0020702F00205A
:108350001FB5084B1B681B0309D58DF8040003915A
:1083600001230D2001A98DF8053000F0B7FA05B002
:108370005DF804FB782E00201FB5084B1B681B031B
:1083800009D58DF80400029100230D2001A98DF874
:10839000053000F0A3FA05B05DF804FB782E00204C
:1083A00038B5064C002584F8285008F03FFF84F8C3
:1083B0002950E5622586656338BD00BFA01A0020FC
:1083C00010B510B9BDE81040EAE700230C225A436B
:1083D0000A4C1119125D824203D00133102BF5D1E2
:1083E00010BD074B586B18B14A784078824203D2CF
:1083F000002259631A86DA6210BD00BF8885010821
:10840000A01A002010B540001428A8BF1420002393
:10841000074A022199540B4499181424834201F805
:10842000014CF5DBFF21D1540F20BDE81040C7E718
:10843000842C002010B50A4A0A4B11689B6800BFC3
:1084400012689142F7D1084A4FF47A70946B00FB9E
:1084500004F2D31AB3FBF4F300FB013010BD00BFEC
:108460009C2E002010E000E0A01A002038B5044641
:10847000FFF7E0FF0546FFF7DDFF401BA042FAD300
:1084800038BD10B504462CB14FF47A70FFF7EEFFFB
:10849000013CF8E710BD2DE9F04180460B25013D78
:1084A00019D008F10106322705243846FFF7E9FF05
:1084B0003846FFF7E6FF3CB1013CF6D14FF4FA70C5
:1084C000FFF7DFFFFA27F0E7013EEED14FF47A70B5
:1084D000FFF7D7FFE3E7024A024BDA60BDE8F0811D
:1084E0000400FA0500ED00E0024A1368013313604E
:1084F000704700BF9C2E0020024BDB6B03B1184776
:10850000704700BFA01A002003685B6918472DE977
:10851000F743064689469DF8288011461A469DF87D
:108520002C3000250C2068431A4FC419C057B042A4
:1085300002D1207A20B126E00135042DF2D122E0CB
:10854000012E0AD003DCF6B90093134807E01E2E73
:108550000AD01F2E17D1012006E010480093434691
:1085600002F0CDFC044605E003F060FB4146044602
:10857000FFF7CAFF4CB10C2303FB0575267185F884
:1085800008906C6001E0002000E0204603B0BDE8E8
:10859000F08300BF702800200038014000440040F4
:1085A00003681B69184710B504462046FFF7F8FF1B
:1085B00018B90A20FFF765FFF7E710BD0368DB680D
:1085C000184700BF344B354A1B68126810B51A6053
:1085D000334A11685960516892689960DA60314A8B
:1085E000116819615168926859619A612E4A11683F
:1085F000D9615168926819625A622C4A11881985AA
:10860000518859859188D2889985DA85284A1188B8
:1086100019865188598692889A86264A1188D98661
:10862000518892881987194621F83A2F224A1078E2
:108630000022824206DA214C34F81240013221F83D
:10864000024FF6E71E4A1288A3F864201D4A1288DA
:10865000A3F866201C4A1188A3F86C1051889288F0
:10866000A3F86E10A3F87020184A3B2112689A668E
:10867000174A126892FBF1F2B2F5967FC8BF4FF02D
:10868000FF325A67134A1288A3F87820124A528997
:10869000A3F85E2010BD00BFC02C00207C3000205D
:1086A000E0290020EC290020F8290020C411002036
:1086B00000110020AE1100202F2A002020110020E0
:1086C000E42800208C10002006110020B8110020A2
:1086D00000000020401100200C1100202DE9F8437B
:1086E00005460E460D4B002493E88003B44213DA8E
:1086F0007B1933F9140008EB050333F9142009EB57
:10870000050333F9143001341344022293FBF2F3CE
:10871000C01A07F0F7FDE9E7BDE8F883C02C002098
:1087200070B5472007F03EFD174B1B681B0307D5AC
:10873000164B174A5B6810681B68C01A07F0D3FD18
:10874000144E154C154D307807F0CDFD2368286880
:10875000C01A07F0D7FD63686868C01A07F0D2FD39
:108760000F4B188807F0BFFD0E4B188807F0BBFDB4
:108770000D4B188807F0B7FD337823742B68A3607E
:108780006B68E36070BD00BF442E0020C02C002049
:108790007C300020C6190020AC2C0020C819002015
:1087A000C4190020C2190020481100207FB5264CB2
:1087B000264E274D2749284A284B20B128480088B3
:1087C000B0F5805F31D2308891F820101278ADF882
:1087D000040028781C4D1B788DF806008DF80710D2
:1087E0008DF8082001A8294606228DF809300CF0E2
:1087F000E9FB30B30198BDF808302860AB80532006
:1088000007F0D0FC208807F06EFDA07807F06BFD24
:10881000E37801A80193237902936379039307F026
:10882000C9FC0F4B00221A800BE0308891F8201011
:108830002080127828781B78A070E1702271637113
:10884000DDE704B070BD00BFE01A0020841A0020EC
:10885000C019002048300020030F0020680F0020BE
:10886000642E0020A0F17D03012B70B504460D4657
:108870000A4E05D830687D2105F060FD84F02004A3
:108880003068214605F05AFD35B12B881C4404EBB5
:10889000142404F0FF042C8070BD00BF741A002063
:1088A0000A4A138801331380094A1368013313609D
:1088B000084A138801339BB2202B01BF0023138089
:1088C000054A138808BF013313807047642E0020C7
:1088D0004C2E0020502E0020522E002038B53A4B4E
:1088E00005461B780C46083B012B6BD8452007F04A
:1088F00059FC284607F056FC0C2D23D004D80A2D2D
:108900000AD014D835B138BD0E2D4BD02ED3FF2D43
:1089100050D038BD206849E0207807F043FC6279E8
:108920006378002A14BF80200020184300E02078DC
:1089300007F038FCA07807F035FCE07807F032FC4F
:1089400020793BE0B4F9000007F0C3FCA07807F001
:1089500029FCE07807F026FCB4F9040007F0B9FC24
:10896000B4F90600BDE8384007F0B3BC637820785E
:108970008BB180F0800007F015FCA468E0B207F02E
:1089800011FCC4F3072007F00DFCC4F3074007F007
:1089900009FC200E12E007F005FC6068BDE83840D5
:1089A00007F0B0BC206807F09EFC6068BDE8384066
:1089B00007F099BC054807F0D3FB0020BDE838401C
:1089C00007F0F0BB38BD00BF9C2C0020F29A0108D4
:1089D0002DE9F04FBE4B8BB01A880193BD4F002A92
:1089E00040F0A98042F20103B7F8D607BA4EC21A86
:1089F00050425041FFF7DAFEFFF7E4FD34684920AA
:108A0000254607F0CFFBB54B04F11C09186807F0A9
:108A10006AFC55F8040B07F066FC284604F0D0FB0E
:108A200004F1100004F0CCFB4FF01008AC4D012312
:108A30002A6803FA08F3134203D0D9F8000007F0BC
:108A400061FC08F10108B8F1130F09F10409EDD137
:108A500004F1280004F0A4FBB7F84431B4F92E0067
:108A6000C01A07F040FC2B68DB0408D59D4BB4F816
:108A700064001B88181AC0F30D0007F034FC2B6843
:108A8000980403D5B4F8660007F02DFC2B6859054F
:108A900003D504F16C0004F083FB2B681A0502D5A2
:108AA000A06E07F02FFC2B685B0402D5606F07F007
:108AB00029FC2B68180403D5B4F8780007F013FCE0
:108AC000A04604F1300004F06BFB04F1360004F022
:108AD00067FBB7F8443138F93C0F0127C01A07F09B
:108AE00002FC814B1B789F4208DA38F9020FB4F977
:108AF0003C300137C01A07F005FCF2E72B689905F6
:108B000005D5B4F95E00A0F2DC5007F0FBFB32683B
:108B100076487260B260121A9110754A4A43531C2B
:108B2000032293FBF2F202EB42029A1A7C2303FB2C
:108B300002033360D6E16F4B6F4A1B6811688B42AA
:108B400006D00AA941F8203D00201360FFF7C6FEB9
:108B5000019B97F8D6171B8897F8D7070B44013B62
:108B6000B3FBF0F200FB12338B4280F086815A4F48
:108B70000120FFF71BFEFFF725FD50203E687D68B2
:108B800007F010FBBA683B6810681B687A680344FA
:108B9000106806F11C0BA3EB400007F0B3FB6A68FA
:108BA000736802A89B1A0293AA68B36805F11C08AF
:108BB0009B1A0393EA68F36810249B1A049304F049
:108BC000FFFA2A69336902A89B1A02936A697369DA
:108BD0009B1A0393B369AA699B1A049307F0EAFAF4
:108BE0003F4901220B68A2401A428A4606D0DBF8B0
:108BF0000000D8F80030C01A07F084FB0134132CB1
:108C00000BF1040B08F10408EAD106F1260005F186
:108C10002601002331F9024F30F9022F121B02AC5A
:108C200044F823200133042BF4D103214FF0000931
:108C30004FEA89035FFA83F902AB53F821206AB146
:108C400002F108000F2802D849F0010906E080323D
:108C5000FF2A94BF49F0020949F0030911F1FF31DD
:108C6000E6D24846002407F09DFAA0460DF1080B15
:108C700009F00302022A16D0032A1DD0012A4ED180
:108C8000B8F1000F05D1DBF8004090462401E4B2B2
:108C900045E0DBF800004FF0000800F00F00204333
:108CA00007F080FA3BE0B8F1000F0CD0DBF80000D1
:108CB000C0F3031020432CE0B8F1000F1ED19BF845
:108CC000010007F06FFA9BF8000007F06BFA26E04E
:108CD000502E0020CC110020C02C00204C2E002053
:108CE000442E0020402E00202F2A0020CC2C0020D3
:108CF000DF7BEFBD582E0020542E0020DBF8000053
:108D0000C0F30330204307F04DFADBF80000C0F356
:108D1000071007F047FADBF800402401E4B20BF13A
:108D2000040B06AB9B454FEA9909A1D1B8F1010F9D
:108D300002D1204607F036FADAF8003013F48054F6
:108D40001FBFB6F86420B5F864100124521A18BF8A
:108D500002929A040AD50AAA02EB8401B5F86600C9
:108D6000B6F866200134121A41F8202C580513D5A4
:108D700002AA02EB840C06F16A0E05F16A000022D9
:108D80003EF9021F30F9028FC8EB01014CF82210A6
:108D90000132032AF4D10334190508D50AAA02EBDB
:108DA0008400A96EB26E0134521A40F8202C5A0485
:108DB00008D50AAA02EB8400696F726F0134521A57
:108DC00040F8202C18040BD50AAB03EB8402B5F84D
:108DD0007810B6F8783001345B1A42F8203C00E095
:108DE000FCB1012C03D1029807F08CFA19E0631E44
:108DF000002002AA52F823204000C0B20AB140F07D
:108E00000100013BF5D507F0CDF94FF0000802ABAA
:108E100053F8280008B107F075FA08F10108A045D9
:108E2000F5DB30200321FFF759FC36200321FFF743
:108E300055FC2F4B3C201978FFF750FCDAF8003036
:108E4000990506D5B6F95E00B5F95E30C01A07F08F
:108E500059FA3A6827487B687A60121A9110264AB4
:108E6000BB604A43531C032293FBF2F202EB420223
:108E70009A1A7C2303FB02033B60204B1B681A06F3
:108E800030D51F4C1F4D22682B689A420BD1626867
:108E90006B689A4207D1019B1B88102B11D11A4B8A
:108EA0001B885B060DD1482007F07CF9206807F08D
:108EB00029FA606807F026FA23682B6063686B6004
:108EC0000EE0124A0F4B11782A7C914208D1104AC9
:108ED00099681068884203D15268DB689A4201D0D1
:108EE000FFF71EFC07F02EF90BB0BDE8F08F00BFB6
:108EF0002F2A0020CC2C0020DF7BEFBD782E002015
:108F00004C110020AC2C0020522E0020C61900204D
:108F1000C81900202DE9F84F0C9EC2EB030B394C09
:108F20000B9B002914BF4FF0060A4FF0040AF61AF3
:108F3000636805460133904613D1236853455ED2DA
:108F4000314A032B98BF294652F823202F4807F0B7
:108F500017F963680022013363602D4B05469A714F
:108F600013E0002511E02B4A1278954240DA0B9B62
:108F7000E3B109FB06F2995C01228A40264909689F
:108F80000A4213D1636801336360D4F804900A9BEA
:108F90001C4F9945E7DB2BD10A2007F003F93B680A
:108FA00001333B604FF0FF337B6021E0184A917939
:108FB00021B12C2007F0F6F8013501E00121917173
:108FC00009FB0BF3226808EB030752B958F80300BA
:108FD00007F0C6F897F9041005444B1CD2D00F488F
:108FE00002E03A440E48117907F0CAF80544C9E78F
:108FF000206850452CBF00200120BDE8F88F0020DC
:10900000BDE8F88F5C2E0020747E0108FD9A0108EF
:10901000E01A00204C000020442E00200C9B010888
:1090200090A4010830B585B004AC002524F8025D99
:109030000091ADF8060021461020FFF713FC9DF8C3
:1090400006002146FFF70EFC9DF807002146FFF7BA
:1090500009FC9DF800002146FFF704FC9DF8010083
:109060002146FFF7FFFB9DF802002146FFF7FAFBC0
:109070009DF803002146FFF7F5FB9DF80E002946F9
:10908000C043C0B2FFF7EEFB05B030BD10B5054CD4
:10909000206805F050F918B1206805F049F9F6E7A5
:1090A00010BD00BF441A002010B508F0A1F900213E
:1090B000044608F0ADFB08B1204601E004F1004091
:1090C000054908F09DFA054908F0E6F9FEF76AF847
:1090D000034B186010BD00BF8096184B35FA8E3CCC
:1090E000340000202DE9F04105460E46078A8389A9
:1090F0009BB21F40002F37D0B7FA87F24FF00043E2
:10910000D340DB4399B21F40A2F11B032982042BF9
:10911000F0D8DFE803F0221F1C190300746A24B1A1
:10912000013C0023A4B2736201E0AC8DA4B2D6F876
:109130002080B8F1000FDDD0D8F80030404621463D
:109140009847D8F80480F4E73068A98E08E0706882
:10915000298F05E0B068A98F02E0F068B5F84010EB
:10916000036889B29847C5E7BDE8F08138B50D4B73
:109170000D4D99680D4B1A681C465288114203D058
:10918000FFF758F9286007E0FFF754F92B68984279
:1091900082BFC01A064B186023685A68054B5A6193
:1091A00038BD00BF000C0140E81A0020400200203A
:1091B0000000002000040140F8B59C4B05461B68E8
:1091C000187818B1012800F06781DCE2242D984C52
:1091D0000CD006D80A2D00F0D8800D2D00F0D580D7
:1091E00044E12A2D06D02C2D04D03FE1207160717E
:1091F000A0714DE18F4B6179277900208C4A58543A
:109200002FBB1978D771472921D1597850291ED100
:109210009978472907D1D978472904D11979412963
:1092200001D10121D1719978824A522903D1D17893
:109230004D2900F0AA8299787E4A472907D1D17832
:10924000532904D11279562A04BF0322E271E2792C
:10925000774E022A38D0032A4BD0012A40F083806F
:10926000BA1E072A7FD8DFE802F004080F131A2578
:109270007E2A07F0B5FBA06075E01B78532B72D1F6
:10928000A3685B42A3606EE007F0AAFBE0606AE0BF
:109290001B78572B67D1E3685B42E36063E01B7880
:1092A000302B654B1A788CBF42F0020222F002028A
:1092B0001A7058E0002007F0F3FB207453E0002000
:1092C00007F0EEFB60824EE0072F06D0082F4AD150
:1092D000012007F0E5FBF08245E0012007F0E0FB0C
:1092E00041F2184358434FF47A73B0FBF3F0B08265
:1092F00039E0022F07D0032F0AD1002007F0D0FB5E
:109300004E4B18702FE0002007F0CAFB30762AE0A1
:1093100029D93A1F9210337E0132D2B2013B02EBBF
:109320008303DBB2102B1ED8F91EC2F1010201EB40
:109330008202D2B2012A0BD0042A11D100205E1E73
:1093400007F0AEFB3E4B002298553E4B9A5507E086
:109350003D4A5E1E0020935507F0A2FB3B4B9855FB
:10936000E3690133E361324B2A2D18BF9A7907F183
:1093700001074FF000000CBF0122554027716071BA
:109380000CBF83F820209D7182E094F82000002813
:1093900047D02F4B13F8012D2E495A708B42F9D12B
:1093A000244A234D13785278402B85BF373B1B014D
:1093B0001B01DBB298BF03F0F003402A8CBF373AA1
:1093C000303AD2B21344A279DBB29A4226D1212399
:1093D0000B70E8796B6A012803F101031D4A6B6287
:1093E0000AD002281CD172231370AA8A1A4B1A8041
:1093F000EA8A1A4B1A8013E0672313700E4B1B780E
:109400009F070ED5164BAA681A60EA685A602A7C34
:10941000144B1A706A8A144B1A8002E03F230B70B7
:109420000020002384F8203032E000BF64020020D6
:10943000E81A0020A42E0020C0190020601100208E
:109440009111002081110020611100207111002074
:10945000880B0020740B0020C21900204811002046
:10946000C8190020C6190020C4190020637994F897
:1094700020000E2B9FBFA94A591C5171A84A98BFC2
:10948000D554A64A18B993795D40957100E0002043
:10949000003018BF0120F8BDA04B002293F828101F
:1094A000082900F27081DFE801F0050C101A2B3B4F
:1094B0005E788500B52D40F0668183F82920012271
:1094C0004EE0622D08BF02224AE0032283F82820E2
:1094D00083F82A5083F82B5083F82C5053E1042250
:1094E00083F8282093F82B2093F82C102A44D2B22A
:1094F00083F82B200A4483F82C2083F82D5042E176
:10950000052283F8282093F82B2093F82C102A4466
:10951000D2B283F82B200A4483F82C20DD8532E177
:10952000062283F8282093F82B2093F82C102A4445
:10953000D2B283F82B200A4483F82C20DA8D02EB78
:109540000525ADB2B5F5AC7F82BF744A012182F822
:1095500029100022DD851A86002D40F01481072293
:1095600083F828200FE193F82B2093F82C102A443D
:10957000D2B283F82B200A4483F82C201A8EB2F53D
:10958000AC7F3EBF6549891881F834500132D98DCE
:1095900092B291421A86E2D9F5E0082283F8282097
:1095A00093F82B30AB4200F0EE805C4B012283F845
:1095B00029200FE05B4C83F8282014F8012D6270FD
:1095C000594A9442F9D193F82C10544AA94206D032
:1095D0003F232370554A536801335360D3E0516AE7
:1095E00092F829000131516210B13E232370CAE084
:1095F0002121217092F82D10062941D004D802298A
:1096000007D0032923D0F8BD122959D0302967D0BB
:10961000F8BD502121704649946B4C60D46B0C60AE
:10962000516C4FF47A7491FBF4F1424C218092F822
:109630008C11414A19B1117841F0020102E0117810
:1096400021F002011170012283F88D218DE0532158
:10965000217092F83910CE0705D592F83820D51E22
:109660006A426A4100E0024602F0010183F88C116F
:10967000002A7AD130490A7822F002020A7074E096
:109680004F21217092F83F10CC0705D592F83E206B
:10969000D11E4A424A4100E0024602F0010183F82D
:1096A0008C1122B924490A7822F002020A7093F838
:1096B0006310224A1170B3F86010214A118054E0FF
:1096C00056212170946C1F490C8042F21074D16CA9
:1096D00091FBF4F11C4C2180012182F88E1144E0B1
:1096E0004921217092F83810184A102988BF10219A
:1096F0001170174914780022A24233D20E7A154D08
:1097000056554E7A144D5655CE7A144D565511F87D
:109710000C6F134D56550132EEE700BFE81A0020DA
:10972000A42E0020880B0020740B0020440200208F
:10973000C8190020C4190020C0190020C619002033
:109740003E000020C21900204811002060110020B6
:109750001C1B0020611100207111002081110020CC
:1097600091110020DA690132DA6193F88D310B4AE8
:1097700093B192F88E317BB1002182F88D1182F87D
:109780008E111846F8BD0020F8BD1279432A7FF4E7
:1097900052AD0222E2714EE5F8BD00BFE81A00208A
:1097A0000449054B0968002218705A6199611A77BB
:1097B000704700BF9C2E002044020020F8B5101A0C
:1097C0000D461F4607F014FE0446781B07F010FEF6
:1097D000174B079E196807F05FFE21460546204695
:1097E00007F05AFE29460746284607F055FE01466F
:1097F000384607F049FD0CF071F80E4907F04CFEB1
:1098000008F036F8069B2946186004F100400BF07A
:10981000D9FE094907F040FE084907F035FD08F078
:1098200001F80028BCBF00F50C40A0303060F8BD46
:10983000340000202C7D8E3FA00CB34500A00C46C8
:1098400044F25063984203DDA0F50C40A038704705
:10985000034B9842BCBF00F50C40A030704700BFDE
:10986000B0B9FFFFF7B50368174C184D23600B68BC
:10987000174E63600068FFF717FC95E80300154B6F
:109880000196009394E80C00FFF798FF3668124B9E
:1098900060681E606B68114FC01A07F0A9FD104B7D
:1098A000196807F0F9FD07F0BDFF2A6823687860A2
:1098B0009B1A3B600B4B1E600B4B1B68DA880B4BF3
:1098C0001A8003B0F0BD00BFF82B0020C81900209B
:1098D000042C0020002C0020402C0020082C00200C
:1098E00034000020382C0020E00F0020342C002011
:1098F00070B50446407907F077FD1E4907F080FEF9
:109900001D4D1E4E2860E07B07F06EFD194907F0E3
:1099100077FEEE606860A07907F066FD184907F0F1
:109920006FFE184D2860207C07F05EFD114907F09E
:1099300067FE6860A07E07F057FD134907F060FEE0
:10994000EE60A860E07907F04FFD0D4907F058FE82
:109950000E4D2860607C07F047FD064907F050FE79
:109960006860E07E07F040FD074907F049FEEE60C1
:10997000A86070BD0000C842102C00200000FA440E
:1099800000002041202C002000007A44442C0020BC
:1099900010B50C4C23789B0713D50B4B1B78042B6D
:1099A0000FD90A4A0A4B1068526818605A60FFF7CC
:1099B0007BFB084B1A88084B1A80237843F001037D
:1099C000237010BDC0190020C6190020C81900203E
:1099D0004C110020BC110020542C0020164B13B554
:1099E0001B681B0325D5154B154C1B7815498DF8A5
:1099F0000030154B20681B788DF8013007F04CFDC6
:109A000007F036FF11498DF80200606807F044FD49
:109A100007F02EFF8DF80300A06807F029FF0C4B1C
:109A20008DF804001B780A2069468DF80530FEF792
:109A300055FF02B010BD00BF782E0020682E002018
:109A40008C2E002000002041882E002000007A4447
:109A50006C2E0020054A137883F001031370044A2A
:109A600000231360034A1360B8E700BF6C2E002088
:109A7000842E0020802E002001480249FFF732BBCF
:109A800000080040D82A002001480249FFF72ABBFD
:109A900000040040B02A00204FF080400149FFF749
:109AA00021BB00BF882A002001480249FFF71ABBEA
:109AB000002C0140602A002001480249FFF712BB38
:109AC000002C0140602A0020254B10B55A43254B3D
:109AD000254C1B680139B3FBF2F20388013AA0421E
:109AE00089B292B29BB212D004F50064A0420ED0AB
:109AF000B0F1804F0BD0A4F59834A04207D004F504
:109B00008064A04203D004F58064A04202D123F017
:109B100070039BB2154CA04206D004F58064A042AD
:109B20001CBF23F440739BB203800F4B8185984286
:109B300002850FD003F5006398420BD003F5406314
:109B4000984207D003F58063984203D003F5806301
:109B5000984201D1002303860123838210BD00BFF8
:109B600040420F0048000020002C0140001000403F
:109B700073B505460068FFF7A7FF2A68012413881C
:109B800000269BB243F001031380EB7A01A88DF805
:109B900004308DF805408DF806608DF8074006F01A
:109BA0008FFDEB7A1B2B0BD1192301A88DF8043004
:109BB0008DF805408DF806608DF8074006F080FDB1
:109BC00002B070BD0C4B800A98420CD004D8B0F59E
:109BD000801F0CD101207047084B984205D04933B3
:109BE000984206D003E00220704703207047FE2011
:109BF00070470020704700BF0100100002001000F5
:109C00002DE9F84304680746204688469146FFF749
:109C1000D9FF03284BD8BA7A9108B8F1000F06D1C2
:109C2000A589AEB202258D4026EA0505A5810A2345
:109C300003FB00131F4A42F82380043342F82390A9
:109C4000B8F1000F07D0BD7AA189AD080223AB405F
:109C50000B439BB2A3812823434303F1200111440A
:109C6000EFF31286502585F3128803F10C051C339F
:109C70001544134455F8047F17B10F602968043167
:109C80009D42F7D100230B60F3B283F311882823A0
:109C900003FB0020036A23B1A3899BB243F00103B5
:109CA00004E0A38923F001031B041B0CA381BDE87E
:109CB000F88300BF602A0020FFF758BAFFF756BAB2
:109CC000FFF754BA014801F0B7B800BF781C002074
:109CD000014801F0B1B800BFCC1C00200C4B4FF480
:109CE00000525A604FF6FE730A48D0F818221168E5
:109CF0000B401360D0F80822D0F80C329A4203D0FF
:109D000000F5F27001F0CAB8012380F828327047DC
:109D100000000240E81A002038B500240B4D6059BD
:109D2000254405F079FD696811B10948FDF799F9F5
:109D3000A96811B10748FDF794F90748103405F0F8
:109D40006BFDB4F5D87FE9D138BD00BF8C7E01082A
:109D5000309B0108369B010836A50108F0B585B097
:109D600004460BF08EF9082826D1621EE01D1F491B
:109D700012F8013F09681944497801F003010229EA
:109D800008BF203B82421370F1D1254604F1080739
:109D900015F8016B164831460BF065F920B12846DD
:109DA00031460BF060F910B1FDF776FE1CE0BD42C4
:109DB000EED1204603F07CFA0E4805F02DFD00237D
:109DC0000D4A04A91A4492F88A210A440849595CA8
:109DD0000133082B02F80C1CF2D10023074801A91B
:109DE0008DF80C30FDF73DF905B0F0BD50000020B6
:109DF000D6A101083C9B0108CC11002078A40108E1
:109E000008B5184B184C1D682068FEF7CCFB284697
:109E1000FEF7C9FB206841798B0703D441F00201AA
:109E2000FEF772FB206804F086FA68B10E4B1868E2
:109E300004F07EFA0646FFF7BFF908B104F0D8FD3A
:109E40002846314604F07AFA284604F074FA0028CD
:109E5000E8D02846266804F06BFA0146304604F044
:109E60006DFADFE7742C0020201D00202DE9F0475B
:109E700005460BF006F92F4E0446D6F8088090B937
:109E80002D4805F0C9FC2D4B53F8241049B101238E
:109E9000A34013EA080F02D02948FDF7E2F8013485
:109EA000F1E7284822E02846274922460BF0F2F83D
:109EB00058B9264805F0B0FC254C54F8041F002979
:109EC000EFD01F48FDF7CDF8F7E72B784FF00009EA
:109ED0002D2B03BF013504F1FF344FF0010A4FF081
:109EE000000A164B53F8297027B91A48BDE8F04705
:109EF00005F092BC2846394622460BF0CBF8A8B9AB
:109F0000012000FA09F0BAF1000F03D0FDF73CFA86
:109F1000114803E040EA0800B060104805F07CFCFE
:109F20003946BDE8F0470E48FDF79BB809F1010935
:109F3000D7E700BFCC110020429B01083C800108FC
:109F40004C9B010836A50108509B0108559B010850
:109F500038800108779A0108619B01086A9B010813
:109F600077A4010810B5084805F056FC074B0024FB
:109F70001C715C63064B1C7004F082FB05F024FE30
:109F8000044B1C6010BD00BF729B0108201D002007
:109F900098300020742C002070B5064600240B4B2E
:109FA000E518AA8816420AD0E1580948FDF759F881
:109FB0002846002105F0C1FB064805F02DFC40F6BF
:109FC000BC4314349C42EAD170BD00BF288701080D
:109FD0009E9B010836A50108F0B504788BB00546B4
:109FE0000CB1002436E04B4B19680E2303FB04111F
:109FF000B1F91D51B1F91921B1F91B31009591F851
:10A00000205101F58C70019591F8215101F5907165
:10A01000029590F90700039091F902103E480491CF
:10A0200021460134FDF71DF8082CDCD170E02D2B02
:10A0300014D1072C1BDC28460BF078F80AAB661C01
:10A0400003EB440424F8100C15F8013F303B092BB6
:10A05000FAD934462B78002BE9D104E0A3F1300281
:10A06000092A09D8E5E7082CBDF8182009D00BB05B
:10A07000BDE8F040FDF710BD202BF8D10135264694
:10A08000E7E7072AF3D840F2DC55BDF81A00214B68
:10A09000A0F2EE2189B2A9421B68E8D8BDF81C10D5
:10A0A000A1F2EE24A4B2AC42E1D8BDF81E6004B225
:10A0B00037B2A742DBDB0DB2AF42D8DCA542D6DB1C
:10A0C000BDF8247007F16404A4B2C82CCFD8BDF841
:10A0D00026E00FFA8EF4112CC9DCBDF82050B42D07
:10A0E000C5D8BDF82240B42CC1D812B24FF00E0C26
:10A0F0000CFB0233A3F81901A3F81B11A3F81D618F
:10A1000083F8205183F8214183F81F7183F822E1FD
:10A110000BB0F0BD1C110020A89B0108F0B504464F
:10A120008FB020460AF0ADFFC5B21DBBAB4805F0AD
:10A1300073FBAB4C94F8D61009B9AA4853E049B266
:10A1400094F8D42094F8D530009194F8D710A6480C
:10A15000019194F9D8100734029194F9D210039127
:10A1600094F8D310049129460135FCF77AFF102D9D
:10A17000E0D1E2E720469D4905220AF08BFF054623
:10A18000B8B929469A4870220AF037FF2846994BF9
:10A1900019680E2303FB001301300022082883F8FE
:10A1A000232183F8242183F8252183F82621F0D167
:10A1B00012E12046904904220AF06CFF0546204631
:10A1C000002D4AD120210AF04EFF002800F0048122
:10A1D000461C30460AF055FF2C460746874B53F87D
:10A1E00024502DB986480FB0BDE8F040FCF739BFC8
:10A1F00030462946FAB20AF04DFF01340028EDD16D
:10A20000774A164602F17001002382F8DA3082F8AC
:10A21000D63082F8D53082F8D43007328A42F3D172
:10A22000784901EBC40191F80822934210DAD1F881
:10A230000C72C3EBC302B0183A44176800F1D401A2
:10A24000C0F8D47090880133888092798A71E7E7EA
:10A2500029466D48FCF705FF8FE06C4907220AF09C
:10A2600019FF05462046002D49D120210AF0FBFEAA
:10A2700006460AF006FFC4B26CBB6548FCF7F1FE67
:10A28000214664480134FCF7ECFE0E2CF8D1554809
:10A29000FCF7E7FE002460482146FCF7E2FE0025BB
:10A2A000544A012311680E2202FB0412D2F8232122
:10A2B000AB401342594B5A495A4808BF1946013519
:10A2C000FCF7CFFE0E2DEBD146480134FCF7C9FE5A
:10A2D000082CE0D180E0304653490AF02BFF2C4691
:10A2E00000284CD0022C4FD00AF020FF06AB43F8D8
:10A2F00024004D4900200AF01DFF0134F0E74A49CF
:10A300000AF018FF002460B1082C38D00AF00EFFC4
:10A3100006AB43F82400444900200AF00BFF013447
:10A32000F1E7082C2BD1069B0F2B28D8DDF81CE079
:10A33000BEF1070F23D8089F0D2F20D8099E06F1E4
:10A340006402C82A1BD80A9DFF2D18D80B986428D0
:10A3500015D80C99642912D8884210DA0D9C032C68
:10A360000DD8324AC3EBC303134483F804E05F7192
:10A370009E71DD71187259729C722D4CD1E60FB02E
:10A38000BDE8F040FDF788BB069B072B20D8079956
:10A390000D291DD80278722A0DD06E2A18D1154ABF
:10A3A0000E20126800FB032301228A40D3F82311F8
:10A3B00021EA020209E00F4A0E20126800FB032383
:10A3C00001228A40D3F823110A43C3F8232101E074
:10A3D000FDF762FB0D4CA4E60FB0F0BDD09B010869
:10A3E000CC11002036A50108FB9B0108479A010803
:10A3F000A01200201C110020729A0108E4930108A9
:10A40000779A01088C7E0108869A0108C89B01088A
:10A410003A9B0108179C010890A4010851A9010862
:10A4200097A801081C9C0108209C01089C12002090
:10A43000989701082DE9F743047805468CB9324D09
:10A4400095F8AB12B5F8A82295F8AA322F480091DA
:10A4500021460134FCF705FE102C05F10405EFD16F
:10A460004EE00AF063FE0F28044636DC2846202121
:10A470000AF0F9FD264EE4B2D6F83880451CA40057
:10A48000002728460AF052FE5FFA87F9B9F1010F5A
:10A4900083B208D0B9F1020F0BD0B3F5B47F24D248
:10A4A000B26B13530AE0FF2B1FD8B36B2344987091
:10A4B00004E0FF2B19D8B36B2344D87028462C2115
:10A4C0000AF0D1FD054608B1013502E0B9F1020FED
:10A4D0000BD10137032FD4D112E00E4800210F22F7
:10A4E00003B0BDE8F043FDF754BA08EB04000021C7
:10A4F00004220AF082FD03B0BDE8F043FDF7CCBAB8
:10A5000003B0BDE8F08300BFCC110020229C0108FD
:10A51000201D0020209A01082DE9F04304788FB017
:10A520000546002C59D17C4B0021142209A807AE06
:10A53000D3F83C800AF061FD0722304600210AF082
:10A540005CFD00231A46A70005A8059308EB070544
:10A5500083807249B5F802E031F813C01CEA0E0F8F
:10A560000AD00E310DF1380C595C02F1010E624433
:10A5700002F81C1C5FFA8EF20133072BE9D100218F
:10A580000B46674AB5F802E011F802C01CEA0E0F4C
:10A590000AD006320DF1380C8A5C03F1010E6344D7
:10A5A00003F8242C5FFA8EF301310629E9D118F85B
:10A5B00007308DE841006A785A49029209A81A09C1
:10A5C00003F00F0306F092FA2146574809AA013416
:10A5D000FCF747FD202CA6D19BE00AF0A7FD1F2821
:10A5E000044600F3898028462021E4B20AF03BFDAE
:10A5F0001F2C02D9FDF750FA8BE0474B451CDB6B53
:10A60000002103EB8404204604220AF0F6FC002714
:10A61000464B09AE304600210A2217F803905FFA34
:10A6200087F80AF0EAFC002315F8012B32B10A2B57
:10A6300004D04A4502D0F2540133F5E74A4561D1CE
:10A6400008F1FF33032B09D8DFE803F010050242BD
:10A650000DF1230037E00DF123011FE030460AF031
:10A6600065FD2378C0B243EA001006E030460AF0E8
:10A670005DFD237800F00F001843207034E00133B3
:10A68000062B0BD02A4800F2F3269E5D9642F6D1A7
:10A69000034493F8ED2263881343638011F8012F7C
:10A6A00012B30023EEE70133072B0CD0204A02F24D
:10A6B000E6269E5D8E42F6D102EB4303B3F8D82224
:10A6C00063881343638010F8011F69B10023EDE72D
:10A6D00030460AF02BFD0F2804DC30460AF026FD38
:10A6E000607001E0002363700137052F90D10124D1
:10A6F00004F024F96CB97DE70E4800211F22FDF714
:10A7000048F906E02046002104220AF076FC0024E5
:10A71000EEE70FB0BDE8F083201D00206481010842
:10A7200079810108369C0108459C01088581010852
:10A730008C7E0108209A01082DE9F04FAB498BB0BF
:10A7400004460AF063FCAA49002820460CBF0125F4
:10A7500007250AF05BFCA7490028204608BF022510
:10A760000AF054FC002808BF0425E90740F1E68000
:10A77000A14805F051F8002004F05EFE9F4CA0486F
:10A7800005F04AF89F4805F047F863799E4A013B77
:10A7900052F823109D48FCF764FC9D48FCF761FCCF
:10A7A00026460027D6F814800021404607F008F816
:10A7B00020B19848FCF755FC002669E039469648D8
:10A7C000D6F818B0D6F81CA0D6F82090FCF749FCB3
:10A7D0004046002106F0FEFF10B1202005F014F8DD
:10A7E00006A94046FCF7D8FA01468C48FCF739FC2C
:10A7F0005846002106F0EEFF10B1202005F004F8C5
:10A8000006A95846FCF7C8FA01468448FCF729FC1B
:10A810005046002106F0DEFF10B1202004F0F4FFC6
:10A8200006A95046FCF7B8FA01467C48FCF719FC2B
:10A830004846002106F0CEFF10B1202004F0E4FFCE
:10A8400006A94846FCF7A8FA013701467448FCF708
:10A8500008FC0C2F06F11006A4D1AAE749B294F81F
:10A86000D42094F8D530009194F8D7106D48019118
:10A8700094F9D8100734029194F9D210039194F806
:10A88000D310049131460136FCF7EBFB102E03D0B8
:10A8900094F8D6100029E1D1634804F0BDFF574B6E
:10A8A000624C9F6854F8041F19B16148FCF7D9FB4A
:10A8B000F8E70E465F4B53F826404CB10123B340F6
:10A8C0003B4203D05C482146FCF7CBFB0136F1E765
:10A8D0005A4804F0A1FF2146484B0AAA0B4493F8BA
:10A8E0008A311344564A8A5C0131082903F8102C36
:10A8F000F2D1002306A953488DF82030FCF7B1FBB4
:10A90000514804F089FF5148FDF7A4FB504804F07A
:10A9100083FF4E48FFF700FE4E4804F07DFF4B4892
:10A92000FFF788FD4C48FCF79CFB4020FFF734FB09
:10A930004A4804F071FF4548FDF7CCFAAA0739D51B
:10A94000474804F069FF474804F066FF3F4804F0B9
:10A95000B3FD454804F060FF3C48FDF727F8434845
:10A9600004F05AFF3948FDF707FA4148FCF779FB34
:10A970003648FDF797F83F4804F04EFF3348FFF79D
:10A980002BFB00260E27774300243B4A0123126C41
:10A99000A3403A44D2F80A2013421ED101340E2CAF
:10A9A000F3D10136082EEDD12B48FCF75AFB80205D
:10A9B000FFF7F2FA6B0716D5304804F02DFF304848
:10A9C00004F02AFF214804F051FD2348FCF749FB1D
:10A9D0004FF48070FFF7E0FA05E03146224629483F
:10A9E000FCF73FFBDAE70BB0BDE8F08F519C0108A4
:10A9F00061A00108589C01085E9C0108CC11002050
:10AA00006C9C01087E9C0108E49301088A9C010863
:10AA1000959C0108A29C0108AF9C0108399B010884
:10AA200078A40108C79C0108B79C01083880010878
:10AA3000E69C01083C800108F49C0108019D010886
:10AA4000D6A101080D9D0108169D010898970108DF
:10AA5000259D0108319D010836A501083F9D01088B
:10AA60004C9D01085F9D01086D9D0108779D0108BF
:10AA7000869D0108949D0108201D0020A09D0108CD
:10AA8000B19D0108C39D0108026B0346C16810B562
:10AA9000406942B11A6C8C1A013A08BF0A46005D3F
:10AAA0001A64C0B210BD1A6A805C01328A4228BFA3
:10AAB0000022C0B21A6210BD436B13B190F844007B
:10AAC0007047836A406A1B1A584258417047036BAB
:10AAD00013B15B68016C01E0C369016A8B423CBF42
:10AAE000C2689B18581AC0B27047426A806A131A2B
:10AAF0005842584170474171704743799B070AD5C6
:10AB0000436A8269D154436A01690133B3FBF1F2AC
:10AB100001FB123343627047437913F001031FBFF7
:10AB2000C36803F1FF32C369006A1DBF181A1040E1
:10AB3000C0B218467047437910B513F001030446BC
:10AB40000DD0FFF7E9FF58B1236A6269E168D05C74
:10AB50000133B3FBF1F201FB1233236210BD18463F
:10AB600010BDF0B5046D8279A389467923F40053B2
:10AB700012F0020F4FEA03434FEA13430CBF0021C8
:10AB80004FF4005112F0040FA38114BF4FF4806EF4
:10AB90004FF0000E16F0010F8768054614BF042021
:10ABA0000020B307238A48BF40F008029BB223F479
:10ABB000405343EA01032382A18948BF90B289B27E
:10ABC00021F4B05121F00C014EEA010140EA0102EA
:10ABD000A281A38A87B023F440731B041B0CA382B9
:10ABE00001A802F0A5FC049E039B204A944218BFD2
:10ABF0001E46A389192272431BB2002BB4BF7E00EC
:10AC0000BE00B2FBF6F66427B6FBF7F000010109BF
:10AC100007FB1163A28912B2002AADBF1A01D90045
:10AC200032313232ABBFB2FBF7F3B1FBF7F203F0D4
:10AC30000F0302F00702B4BF104318432A6DAB792B
:10AC400080B2208113F0080F938A0BBF23F0080312
:10AC50009BB21B0443F0080308BF1B0C938293892B
:10AC60009BB243F40053938107B0F0BD003801401C
:10AC7000417176E7816074E703460A4690F8460220
:10AC8000D96A9B7900F0D2BF38B5A0F51374637907
:10AC9000A579DB0746D594F8383205F00105F3B104
:10ACA000226B1068838DC3F34E03838494F83C3287
:10ACB00023B1B4F842320133A4F84232917A6A00E7
:10ACC00000F013FE012384F83B32002384F839326C
:10ACD00084F83A3284F83832A4F8403238BD94F817
:10ACE0003B322046012B04BF94F8393284F83A32C3
:10ACF00000F0E6FD94F83B22236B3AB9012284F878
:10AD00003B221868997A05FA02F207E0002284F8DB
:10AD10003B2295421868997A08BF0222BDE8384064
:10AD200000F0E3BD38BD10B5A0F5127494F83C22D4
:10AD3000BAB9A36A616A994228D0591CA069A16274
:10AD4000C35C2069DBB25B0043F400738142A4F86A
:10AD50003E324FF00A0384F83D3228BFA26201233D
:10AD600012E094F93D327BB1B4F83E1220464B0814
:10AD7000A4F83E3201F0010100F0CAFD94F83D3222
:10AD8000013B84F83D3201E084F83C3294F83832DB
:10AD9000002B50D194F839320133DBB2092B84F8FF
:10ADA000393204D12046BDE8104000F089BD0A2B9D
:10ADB00041D194F83B322BB9B4F8403243F001034F
:10ADC000A4F840326379D9071CD5B4F84002820553
:10ADD00001D4C30705D4B4F844320133A4F8443293
:10ADE00010E0E36AC0F347000BB198470AE0E3695B
:10ADF0006269D054E369E1680133B3FBF1F201FB0E
:10AE00001233E361012284F8382294F83B220023B4
:10AE1000012A84F839320ED1A27984F83B32236BAF
:10AE200012F0010F1868997A0CBF02220022BDE8C7
:10AE3000104000F05ABD10BD026D70B51588044673
:10AE4000ADB2A90613D5036B8BB9C36A1BB1908849
:10AE500080B298470BE0E169928840694E1CD2B2FB
:10AE6000E6614254E169E268914228BFE3612B0642
:10AE700013D5636AA26A9A42236D0AD0511CA06955
:10AE8000A162825C9A802369994206D30023A3625F
:10AE900070BDDA6822F08002DA6070BD836A816971
:10AEA000426B1944D160416A994297BF0169CB1A3C
:10AEB000CB1A536096BF0023536083624FF00003A8
:10AEC00080F84430136888BF816243F00103136047
:10AED0007047436A8269D154436A026901339342DD
:10AEE00028BF00234362436B1BB11B68DB0705D4FB
:10AEF000D4E7026DD36843F08003D36070472DE937
:10AF0000F0431E46944B8DB09842894690469DF87A
:10AF1000507051D1914B924A92491A60924AC3F8AB
:10AF200008805A6102F580729A614FF48072DA608B
:10AF30001A618E4A18651A63A2F54842543ADA64D7
:10AF40009A6459638A4B9A6942F480429A615A69B9
:10AF500042F001025A6102238DF803303A074FF4A0
:10AF60000073ADF8003001D51C230FE0B30706D500
:10AF70001823804869468DF8023000F025FEF50759
:10AF80000AD54FF48063ADF800304823794869460C
:10AF90008DF8023000F018FE0E238DF804300022E8
:10AFA000012301A88DF805308DF806208DF80730B3
:10AFB0006A4C05F085FB4EE06F4B984240F0C7802D
:10AFC0006E4B674AC3F808801A604FF48072DA60EB
:10AFD0001A616B4A18655A6102F580729A61694A72
:10AFE0003C079A64DA64624BDA6942F40032DA614F
:10AFF0005A6942F001025A614FF002038DF80330A2
:10B000004FF00403ADF8003001D51C230EE0B0076B
:10B0100006D51823574869468DF8023000F0D4FD54
:10B02000F10709D50823ADF8003048235148694697
:10B030008DF8023000F0C8FD26238DF80430002280
:10B04000012301A88DF805308DF806208DF8073012
:10B0500005F036FB494C0025012384F84430256275
:10B06000E561A5626562C4F82C906671C4F8088039
:10B07000A7712046FFF775FDF20731D5206B002838
:10B0800026D0E36C039501934FF480530A938023F9
:10B090000693E36805950493202309936369079554
:10B0A000029308950B9502F0CBF901A9206B02F0F1
:10B0B000A9F9226B216D136843F0010313608B8A99
:10B0C0009BB243F040038B8253689BB2236407E03A
:10B0D0004FF6DF72236D1A80DA6842F02002DA60E0
:10B0E000B3072CD5606B28B3A36C002501934FF4F4
:10B0F00080530A93802306932369029504931023B7
:10B10000039305950795089509950B9502F098F915
:10B11000606B01A902F076F9636B1A6842F00202D3
:10B120001A60226D5D605D60938A9BB243F080037C
:10B13000938204E0226DD36843F08003D360226DD4
:10B14000204693899BB243F40053938100E0002092
:10B150000DB0BDE8F08300BF00380140CC1C0020DA
:10B160004882010844000240641D0020580002404B
:10B17000001002400008014000440040781C0020FC
:10B18000641F0020044400402DE9F74FFDF752F9F9
:10B19000A64C804626686568A768861BF643451B53
:10B1A000C71BED43FF43F60FED0FFF0F2EB93FB95D
:10B1B000002D00F08782B9462CE04FF0000929E00D
:10B1C000B14627E003EB8A0BBBF802301A050ED418
:10B1D00013F4805F1DBF964A9BF801101268954AD0
:10B1E000954B14BF52F82120126843F82A20BBF86F
:10B1F0000230D80516D499050AD5904B1B7813F068
:10B20000040F0CBF8E4A8F4A8B4B126843F82A20DA
:10B2100009F10109207B5FFA89FA8B4982450B68A5
:10B22000D0D326E0894A5046594603F017FB884B95
:10B230001B885A0603D550465946864A16E05807D9
:10B2400003D550465946844A10E0190703D55046A5
:10B250005946824A0AE09A0703D550465946804A21
:10B2600004E0DB07D4D5504659467E4A03F0F6FA8F
:10B27000CEE7DFF808E20093BEF906307822A3F5A6
:10B280007A7353434FF47A7293FBF2F3F34603F26B
:10B290002B13019300225FFA82FE864517D2009B92
:10B2A00003EB820EBEF802E01EF4806F0DD040F278
:10B2B000671ADFF88491019B39F822E09E449EFBD7
:10B2C000FAFC0AFB1CEE29F822E00132E3E74DB359
:10B2D00008F5C333A0336360637B544A13BB937395
:10B2E000614B1B6813F0020F0AD0DFF894E19EF85F
:10B2F00000E0BEF1000F03D04FF0010E82F80EE027
:10B30000DA0506D5594BDB781BB1A37B43F002036A
:10B31000A3734A4B1B7813F0050F02BFA37B43F0C6
:10B320000403A37394F80EE0BEF1000F03D13F4B6A
:10B330005B7B002B4FD094F80DC01CF0010FACF1DB
:10B340000C031DD1BCF1030F07D8DFF8E8901EF005
:10B35000040F3B4A08BF4A4600E0364AACF1040CF1
:10B36000BCF1070F05D8DFF81CC11EF0010F18BF94
:10B370006246DBB2032B0ED81EF0020F3C4B06E0F8
:10B38000DBB2032B06D82F4B2A4A1EF0020F18BF40
:10B390001A4600E0274A4FF0000C5FFA8CF3834214
:10B3A0000DD20B6803EB8C035B881B0642BFD2F8FF
:10B3B0000090214B43F82C900CF1010CEDE785B186
:10B3C000BEF1000F08D0637B184A0133DBB2142BA7
:10B3D00006D1002304E025B1637B002BF3D100E00C
:10B3E0005373002E52D0234A3223B2F90250B2F9DD
:10B3F0000020002DB8BF6D42002AB8BF524295FB15
:10B40000F3F592FBF3F2EDB2D3B2AB4238BF2B4669
:10B41000194A13B192FBF3F300E01346434423604F
:10B42000E37B024A83BB01232FE000BF642100209D
:10B43000581D0020829501081A090020973000202D
:10B440006C9501085C9501085C1D00206082010874
:10B45000841A0020668201086C8201087282010849
:10B46000788201087E820108782E00204830002072
:10B4700074950108C4110020400D0300702F0020B6
:10B480000C1A00207C9501080023D3738F4D904B3C
:10B490002D78E27BADB9002F00F00F818D4B267B1C
:10B4A0001A788D4B02F0040293F800C08B4BD2B295
:10B4B000D3F800E00B680021894D03EB86060F46A8
:10B4C000B5E01AB9874A1A61002508E0864AFAE70A
:10B4D0000A68AB00D6187688760604D40135EBB23C
:10B4E0008342F5D3D7E7814EB6F90060192E25DDEA
:10B4F00012F803E094F814C00EF00F09E145266934
:10B500000CDCDFF8CCC19CF815C0BCEB1E1FDEBF05
:10B51000D6F800C0DFF8D8E143F80EC012F803E017
:10B5200094F816C00EF00F09E14533DBDFF8A0C137
:10B530009CF815C0BCEB1E1F2CDC26E0193629DA5E
:10B5400012F803E094F814C00EF00F09E1452669E3
:10B550000CDCDFF87CC19CF817C0BCEB1E1FA2BF3F
:10B56000D6F800C0DFF888E143F80EC012F803E017
:10B5700094F816C00EF00F09E1450BDBDFF850C15F
:10B580009CF817C0BCEB1E1F04DBD6F800E0584E39
:10B5900043F806E0554EB6F90260192E1BDD12F88D
:10B5A00003C094F814E00CF00F09F14526690CDC97
:10B5B000DFF81C9199F81590B9EB1C1FDEBFD6F887
:10B5C0000090DFF82CC143F80C90D25C02F00F0C15
:10B5D000F4451EDD82E7193680DA12F803C094F8CC
:10B5E00016E00CF00F09F14526690CDBDFF8E0905E
:10B5F00099F81590B9EB1C1FDEBFD6F80090DFF864
:10B60000F0C043F80C90D25C02F00F0CF445FFF64A
:10B6100065AF94F817E0BEEB121FA2BF3668344A3C
:10B620009E505BE75888000504D404330435B342C8
:10B63000F8D122E04AB101EB0C0A06209AFBF0F99E
:10B6400000FB19A001280DDC01E057B9012793F890
:10B6500001900EEB89003EF829A090F80290C07886
:10B6600003E01746002081468246013125F802ACEE
:10B6700085F800906870C9B2D7E7174A1378013B84
:10B6800013F0FF0308BF06231370124B1B785B07F0
:10B6900041BFBBF906304FF47A72A3F57A7303EB1E
:10B6A000C30348BF93FBF2F3124A46BF0133DBB238
:10B6B000012392FBF3F34344A36003B0BDE8F04FD2
:10B6C00000F0A4B903B0BDE8F08F00BF030F002065
:10B6D00064210020973000201A000020581D00200F
:10B6E0001C0900207895010882950108C4110020EA
:10B6F0001A090020400D030010F80A3C0133DBB2A8
:10B700000A2B84BF10F8131C044A00F80A3C82BFBD
:10B71000002322F8113000F80A3C7047942F0020D3
:10B72000334A70B5136C9068194440F68C23081A9C
:10B7300098429160D060516013463BD9127893F9DA
:10B74000451010468A420BD1111F082908D893F8DA
:10B750004610182901D8013103E083F8442002E0A3
:10B76000002183F8461093F944402149A24219D19F
:10B7700091F84740B4B10C310024944206DA51F8F4
:10B78000046F1C4D25F814600134F6E70C2805D031
:10B790001849002421F810400130F7E716480178D5
:10B7A0000131017083F84520002201211A7083F8CD
:10B7B000471070BD92F84710C9B140F2DA51A0F2BB
:10B7C000EF248C4208D811780B2905D80B1D0131C4
:10B7D000117042F8230070BD002283F84720074B08
:10B7E00003F13002002143F8041F9342FAD170BDE7
:10B7F000CC090020942F0020C4000020D80900208C
:10B80000024A136C0133194411647047CC090020BB
:10B81000024B53F820301B6819807047302A0020F3
:10B82000074BA1F57A7153F820301A681B895943E8
:10B830004FF47A7391FBF3F189B21180704700BF26
:10B84000302A002037B5044603211E2006226B460D
:10B85000F9F718FB78BB9DF801309DF80000174DF3
:10B8600043EA002000B205F0C3FD296805F014FE8C
:10B8700005F0D8FF9DF8033020809DF8020043EAD0
:10B88000002000B205F0B4FDA96805F005FE05F042
:10B89000C9FF9DF80530A0809DF8040043EA002010
:10B8A00000B205F0A5FD696805F0F6FD05F0BAFFE8
:10B8B0006080012000E0002003B030BD1C000020AB
:10B8C00090F83B3210B57BB990F83A3290F8394293
:10B8D000A34209D2B0F8401201229A400A43013330
:10B8E000A0F84022DBB2F3E710BD1FB50123ADF88D
:10B8F0000830ADF80410002301A9ADF80A30ADF806
:10B900000C30ADF8062001F074FE05B05DF804FBC4
:10B910008379DB0748BFB1FA81F1D0F8343148BFF1
:10B9200049095A681B8909B113617047536170470F
:10B930001FB50123ADF808300023ADF80C30ADF889
:10B940000A30094BADF804101B7801A9012B08BF80
:10B950000323ADF8062008BFADF80C3001F049FE16
:10B9600005B05DF804FB00BFC809002038B510F829
:10B970000E2C044650F8043C52B9012200F80E2C5B
:10B9800020F80C1C997A18680222BDE83840CFE7ED
:10B9900030F80C2C20F80A1C891A89B220F8081CEF
:10B9A000074A10F80F0C002522F8101004F80E5C5E
:10B9B0001868997A2A46FFF7BBFF04F8065C38BD81
:10B9C000942F0020044B53F820301BB107289CBF54
:10B9D0001B681980704700BFF40A0020084A1368EA
:10B9E0009B020BD5074B002119704FF6FE730649D9
:10B9F000086803400B604FF400135360704700BFAA
:10BA000000000240963000206C0002402DE9F04713
:10BA1000664D2B686649581C0A788E4602F0FF0670
:10BA20000AB10346F6E737462B60687BAB6895F8AA
:10BA30000C80AA7B39B2202900F09C80DFF880C1FD
:10BA40000CEB8103DC789B783CF82110C3F1FF03F9
:10BA50009BB2002B65D04FF03C0CB1FBFCF9C3F15D
:10BA6000FF0363431B12B9F1050F5DD8DFE809F04E
:10BA7000030B1A293A4AE01A4143B1FBFCF0DAB24F
:10BA80001044C0B251E0B1FBFCF00CFB101189B2C4
:10BA9000DAB2C1F13C01E31A4B43B3FBFCFC204694
:10BAA00094442CE0B1FBFCF00CFB1011E21A89B2BB
:10BAB0004A43B2FBFCF25FFA83F84244D2B220461A
:10BAC00032E0B1FBFCF90CFB191189B2E01AC1F1AB
:10BAD0003C014843B0FBFCF05FFA83F84044C0B23D
:10BAE000224621E0B1FBFCF80CFB1811D8B289B258
:10BAF000E31A01FB03F2B2FBFCFC224684445FFA2A
:10BB00008CF412E0B1FBFCF80CFB181189B2D8B22E
:10BB1000C1F13C01E31A4B43B3FBFCF20244D2B245
:10BB200003E02246204600E044464FEA042C4CEA5B
:10BB3000004C4CEA020C17234FF0010808FA03F8F6
:10BB400006F1170118EA0C0FA1EB0301DFF874806E
:10BB500014BF4FF011094FF0090989B213F1FF33F7
:10BB600008F80190E8D218360137B6B2BFB2114BCF
:10BB7000A0465FE7AB6001238EF8003040F22A3325
:10BB8000AA730D4AE9800D4985F80C806873AE8070
:10BB9000536000238B840B889BB243F001030B801E
:10BBA000136843F001031360BDE8F0877C21002097
:10BBB00096300020882100206C00024000040040E4
:10BBC0001A090020890B0020F0B5B1F800E000232D
:10BBD0004EFA03F2D50725D58E784FEAD30CF4063A
:10BBE00048BFCC7806F00F0203F0070748BF224396
:10BBF000BF0050F82C500F24BC4025EA0404BA4082
:10BC00002243282E40F82C2005D1C46801229A40F6
:10BC100024EA020205E0482E04D1C46801229A40B9
:10BC20002243C2600133102BD2D1F0BD2DE9F04F79
:10BC30001E464FF414734343554D85B005F110046F
:10BC400080469146E718A24610B92B44514A03E0BA
:10BC5000012805D1504A2B441A641032C3F84421FC
:10BC60004FF4147303FB08F34C48EC180AEB03027F
:10BC700003F59C73343253442061E1636262A36232
:10BC800000224FF480714FF0010BD4F844310320AF
:10BC9000E1612263E2622162A263626384F84C2262
:10BCA00084F848B284F84922A4F85222A4F8542215
:10BCB000C4F818906075A67584F8568258681B8978
:10BCC00004F5A0724FF0020CADF80C3003A910235C
:10BCD00001928DF80E308DF80FC0CDF800C0FFF73F
:10BCE00073FF236CDDF800C0597B58681B898DF801
:10BCF0000E1003A9ADF80C308DF80FC0FFF764FFEC
:10BD000059463846FFF704FE3220FCF7BAFB244BB5
:10BD1000019A1B68D2F804B01A46B2FBF9F1B1F5EA
:10BD2000803F03D3012AF8D95208F6E71D4A4FF4A1
:10BD30001474B3FBF2F204FB08F8584689B2D2B28D
:10BD4000FDF716FF05EB0809174B08F512780AEB0B
:10BD500008040022C9F8583258462146FDF750FF22
:10BD6000D9F8405016F0010F0CBF022200222868BB
:10BD7000A97AFFF7BAFD0D4B2846C9F85C32211DA0
:10BD80000022FDF73DFF384605B0BDE8F08F00BF4B
:10BD90007C210020C4960108E496010884820108F1
:10BDA0004800002040420F0027AD000889AC000881
:10BDB0002DE9F7438E460546DFF8A092114699F823
:10BDC000B0440068164698467246631C89F8B03441
:10BDD000FDF77AFE2B8901A9ADF8043018238DF800
:10BDE0000630686802238DF80730FFF7EDFEAB7A66
:10BDF00009F2B447240127442A6849460C2B00F273
:10BE0000F680DFE813F00D00F400F400F4005100B8
:10BE1000F400F400F4008A00F400F400F400C2001E
:10BE2000138CDFF83CC223F001031B041B0C1384AA
:10BE3000138CB2F804E0108B624520F073004FEAD7
:10BE400000404FEA10409BB21FFA8EFE40F0700097
:10BE500014D00CF5006C624510D00CF5406C6245B6
:10BE60000CD00CF5806C624508D00CF5806C6245F6
:10BE700004D023F0020343F0030307E023F00E0392
:10BE80002EF4407E43F003034EF4807EA2F804E0DB
:10BE90001083A2F834801384138B23F008031B044F
:10BEA0001B0C43F0080336E0138CDFF8B4C123F019
:10BEB00010031B041B0C1384138CB2F804E0108BCA
:10BEC000624520F4E6404FEA00404FEA10409BB242
:10BED0001FFA8EFE40F4E04008D00CF5006C62457D
:10BEE00004D023F0200343F0300307E023F0E00305
:10BEF0002EF4406E43F030034EF4806EA2F804E05E
:10BF00001083A2F838801384138B23F400631B047E
:10BF10001B0C43F40063138369E0138CDFF840C10A
:10BF200023F480731B041B0C1384138CB2F804E0FD
:10BF3000908B624520F073004FEA00404FEA1040BA
:10BF40009BB21FFA8EFE40F0700008D00CF5006C1A
:10BF5000624504D023F4007343F4407307E023F4F4
:10BF600060632EF4405E43F440734EF4805EA2F8AA
:10BF700004E09083A2F83C801384938B23F00803A1
:10BF80001B041B0C43F0080330E0138CDFF8D0C017
:10BF900023F480531B041B0C1384108CB2F804E0B0
:10BFA000938B20F4005023F4E6431B0400041B0C85
:10BFB000000C62451FFA8EFE43F4E04340F440500B
:10BFC00003D00CF5006C624503D12EF4804E4EF484
:10BFD000804EA2F804E09383A2F840801084938BF3
:10BFE00023F400631B041B0C43F4006393832B7B3B
:10BFF00043B1B2F844306FEA43436FEA53439BB214
:10C00000A2F8443013889BB243F001031380AB7A4B
:10C010000C2B19D8DFE803F0071818180B1818189C
:10C020000F18181813000B1902F134000AE00B194D
:10C0300002F1380006E00B1902F13C0002E00B1996
:10C0400002F14000C3F8B40438460C44A4F8BC64C0
:10C05000C4F8B82403B0BDE8F08300BF7C21002001
:10C06000002C01402DE9FF415B4B1B689BB11A6816
:10C070001AB15A49886902438A619A889868ADF86A
:10C08000042002228DF8072004220DEB02018DF816
:10C090000620FFF799FD3220FCF7F3F90021112269
:10C0A0001E20F8F7C9FF012160221E20F8F7C4FF07
:10C0B0006420FCF7E6F9002402A8FFF7C3FB27463B
:10C0C00026460A25022101221E20F8F7B5FF32205C
:10C0D000FCF7D7F902A8FFF7B5FBBDF90820BDF9B9
:10C0E0000A1014448A42A8BF0A46BDF90C300F4416
:10C0F00093421E44A8BF134613F5805F04DD013D43
:10C10000E0D14FF0010801E04FF000081E200021AF
:10C110001222F8F791FF0A25022101221E20F8F7CA
:10C120008BFF3220FCF7ADF902A8FFF78BFBBDF9BE
:10C130000820BDF90A10A41A8A42A8BF0A46BDF910
:10C140000C307F1A9342A6EB0306A8BF134613F5E3
:10C15000805F02DD013DDFD101E04FF000082046A5
:10C1600005F046F901461E4805F04AFA1D4D20F03B
:10C1700000402860384605F03BF90146184805F0B4
:10C180003FFA20F000406860304605F031F9014682
:10C19000154805F035FA20F00040A8600021702213
:10C1A0001E20F8F749FF012120221E20F8F744FF46
:10C1B0001E2002210022F8F73FFF6420FCF761F9FE
:10C1C000B8F1000F04D14FF07E532B606B60AB6071
:10C1D00004B0BDE8F08100BF680B002000100240F1
:10C1E00000406F461C00002001C05E46064B1B78D5
:10C1F00003F0040303F0FF001BB1044B1888C0F3E5
:10C20000C01000F00100704797300020841A002011
:10C210002DE9F04F89B00593BE4B0026B3F902908B
:10C22000B3F90030B9F1000FB8BFC9F10009002B14
:10C23000B8BF5B429945B8BF99468046B24634467E
:10C24000B9F5FA7F04910392A8BF4FF4FA790190EF
:10C2500000960296B04D2B88990754D0AD4B6100E3
:10C2600033F91420AD4B33F9143003EB4202039B36
:10C270005B429A4203DB039B9342A8BF1346A84A42
:10C280008F5E059ADB1B32F914001F18FFF7AEFF13
:10C2900090B1A44B384613F804A005F0A9F8A249C0
:10C2A00005F0AEF90146504604F028FA9E4905F023
:10C2B000F3F805F0B7FA074698F8083064227B4394
:10C2C00093FBF2F398F81C206FF0040A0AFB02FAC1
:10C2D000534504DB02EB820A9A45A8BF9A4642F214
:10C2E0001072924B53F8240038449042A8BF104675
:10C2F0008F4A9042B8BF104643F8240098F8123095
:10C300005843031302932D8805F00303012B38D003
:10C31000804B884933F91430A6000093019B51F8F3
:10C32000247093F801E0844B33F9140080EAE07341
:10C33000A3EBE073B3F5206F16DC009A50235A4349
:10C3400092FBFEF3042290FBF2F0181A0744B7F5B3
:10C350007A5F7A4BA8BF4FF47A579F42ACBF41F83F
:10C36000247041F8243002E0002341F824308B5936
:10C370007D2693FBF6F6019BDB7A7343402693FB05
:10C38000F6F6AA0712D5009A09FB06F509FB02F793
:10C390000298C9F5FA7303FB0A7703FB00534FF4C5
:10C3A000FA7297FBF2F193FBF2F505E0EB0755BF4C
:10C3B000354651460099029D5F4B042733F91430EE
:10C3C0005F4A93FBF7F3A25C6FF04F07534393FB75
:10C3D000F7F398F851204FEA440BCF1872B1384662
:10C3E000069205F005F85749574B01EBC401069A30
:10C3F0001B68FAF70BFC05F015FA07464E4B534A3B
:10C400003BF803003BF9021003B25B1A042193FBD3
:10C41000F1F102F1040E5EF824302BF802000C3228
:10C4200052F8240042F8243098F8502018444FEA7B
:10C43000840C08444EF8241082B1CDF81CC006923A
:10C4400004F0D6FF4249404B01EBC401069A1B6839
:10C45000FAF7DCFB05F0E6F9DDF81CC03D4BDFF830
:10C4600010E11B5D7A195843202390FBF3F3D21A95
:10C470002BF80E20384A5B424CF80230019B3748BB
:10C48000374901334CF801504CF800700193754660
:10C490000CB90124DEE61F4B0427B3F90440049BCA
:10C4A000244E9B79D6F808E00F335B006343224C9F
:10C4B0005B11B4F90440002B94FBF7F7A3EB0707DB
:10C4C000B8BF5B42322B98F80D400BDC04FB07E44D
:10C4D000244BA342A8BF2346234CA342ACBFB36066
:10C4E000B46001E00023B36098F8034004FB07F355
:10C4F0001E4C9B112478032C3DD9B8F84E40B4F55E
:10C50000FA7F38D26742BB4234DBA342A8BF23463E
:10C5100031E000BFC4110020841A002090300020B8
:10C520006E2E0020D082010800002041F02600205D
:10C53000F0D8FFFF902900200011002080C1FFFFEC
:10C54000182A0020742900208C290020F8260020B9
:10C55000C02900202C2A0020F8290020E0290020F2
:10C56000EC290020FEFFFF0F020000F02F2A002020
:10C57000D82900203B46B4686FF0FF0644F34F34DF
:10C58000B4F5807FA8BF4FF48074B442B8BF34467E
:10C5900083601E190023AE808C60936009B0BDE8F3
:10C5A000F08F2DE9F04F87B00393B44B81461D887F
:10C5B000029105F00205ADB2019295B1B04BB3F90D
:10C5C0000250B3F90030002DB8BF6D42002BB8BF48
:10C5D0005B429D42B8BF1D46B5F5007FA8BF4FF432
:10C5E0000075CB460026A64BA64933F91620A64B6C
:10C5F0004FEA460A33F91630520083EAE374A4EB9B
:10C60000E374B4F5206F4FEA860851F8260011DC78
:10C61000042493FBF4F3D31A0344B3F57A5F9B48E5
:10C62000A8BF4FF47A538342ACBF41F8263041F89B
:10C63000260002E0002341F8263051F808709BF8EC
:10C640000B30FF119BF801405F438C4B54431B8818
:10C65000BF119B074FEAA41456D08D4B3AF9033013
:10C660001A44019B5B429A4203DB019B9342A8BFA1
:10C670001346884A3AF902209B1A039A32F9162087
:10C680001A440492FFF7B2FD049A98B1824B104607
:10C690009B5D049304F0ACFE804904F0B1FF049B61
:10C6A0000146184604F02AF87C4904F0F5FE05F02E
:10C6B000B9F8024642F21070794958F80130134433
:10C6C0008342A8BF034677488342B8BF034648F871
:10C6D000013099F8081099F81C004A4300EB8000DB
:10C6E000D21141428A4203DB8242A8BF0246114670
:10C6F00099F81220641A53431B13FF1A6F436C43BB
:10C7000003EB672701EB64245F4B04223AF9033003
:10C7100093FBF2F2644B9B5D534399F85120A4EBD9
:10C72000A31472B12046049204F062FE5F49604B8C
:10C7300001EBC601049A1B68FAF768FA05F072F873
:10C74000044651495B4B3AF801003AF903E002B262
:10C75000CEEB02024FF0040E92FBFEF22AF8030029
:10C760009E440C3358F80EC058F8030048F80E20C9
:10C770006044104499F8502048F803C08C467AB1C0
:10C780000591049204F034FE4B49494B01EBC6017C
:10C79000049A1B68FAF73AFA05F044F8DDF814C079
:10C7A000464BDFF834E19B5DE21943435B11D21A3B
:10C7B0002AF80E2042484349434A5B4248F8004069
:10C7C00048F8017048F802300BF1010B74460EB9BD
:10C7D000012608E72A4B0427B3F90450029B294E8F
:10C7E0009B79D6F808E00F335B006B43BCF904502B
:10C7F0005B1195FBF7F7002BA3EB0707B8BF5B4274
:10C80000322B99F80D500BDC05FB07E52F4BAB42A3
:10C81000A8BF2B462E4DAB42ACBFB360B56001E064
:10C820000023B36099F8035005FB07F3294D9B11D2
:10C830002D78032D0CD9B9F84E50B5F5FA7F07D2F3
:10C840006F42BB4203DBAB42A8BF2B4600E03B4636
:10C85000B5686FF0FF0645F34F35B5F5807FA8BF8B
:10C860004FF48075B542B8BF354683605E1900232A
:10C87000A6808D60936007B0BDE8F08F841A002019
:10C88000C4110020902900200011002080C1FFFF6A
:10C89000903000206E2E0020D08201080000204140
:10C8A000F0260020F0D8FFFF182A0020742900206D
:10C8B0008C2900200C270020C02900202C2A0020D1
:10C8C000E0290020EC290020F8290020FEFFFF0FBE
:10C8D000020000F02F2A0020D82900202DE9F04F77
:10C8E00089B00593AE4B0027B3F90280B3F900304D
:10C8F000B8F1000FB8BFC8F10008002BB8BF5B4209
:10C900009845B8BF98468246B946BB463C46B8F5FE
:10C91000FA7F0492A8BF4FF4FA7802900397A14DD2
:10C920002B88990757D0022C55D09D4B610033F9C5
:10C9300014209D4B33F9143003EB4202049B5B42FD
:10C940009A4203DB049B9342A8BF1346974A8E5E2C
:10C95000059A9B1B32F914001E18FFF747FC90B193
:10C96000934B304613F804B004F042FD914904F0B3
:10C9700047FE0146584603F0C1FE8E4904F08CFD87
:10C9800004F050FF06469AF808306422734393FB84
:10C99000F2F39AF81C206FF0040101FB02FB5B45E7
:10C9A00005DB02EB82029342A8BF13469B4642F28C
:10C9B0001072814B53F8240030449042A8BF1046B7
:10C9C0007E4A9042B8BF104643F824009AF81230CD
:10C9D000584303130393298801F00303012B01D16A
:10C9E000022C3DD16E4B764D33F91490029BA00082
:10C9F00093F801E0734B55F8247033F9146086EA1C
:10CA0000E673A3EBE673B3F5206F1CDC022C14D0A5
:10CA1000502303FB09F292FBFEF3042296FBF2F68D
:10CA20009E1B3744B7F57A5F674BA8BF4FF47A5720
:10CA30009F42ACBF2F502B5007E089EAE973A3EB6C
:10CA4000E973642BE4DD00232B505D4B7D27C35835
:10CA500093FBF7F7029BDB7A7B43402793FBF7F7C7
:10CA60008A0713D5022C11D008FB07F508FB09F63D
:10CA70000398C8F5FA7303FB0B6603FB00534FF4EE
:10CA8000FA7296FBF2F193FBF2F508E0CB0704D5BE
:10CA9000022C02D0039D594601E03D464946630001
:10CAA0000193484B042633F91430484A93FBF6F3BC
:10CAB000A25C6FF04F06534393FBF6F39AF85120B4
:10CAC000CE18E2B1022C069230460BD104F090FC55
:10CAD000069A530803D09A42A8BF1A4600E00122E2
:10CAE0003B4905E004F084FC3A49069A01EBC40195
:10CAF000394B1B68FAF78AF804F094FE0646314B6E
:10CB0000019A0198D15A354B0AB2C05E4FEA840CA3
:10CB1000121A042092FBF0F20198C15203F10801AD
:10CB2000143351F824E053F8240041F824207044D1
:10CB300010449AF8502043F824E082B1CDF81CC08C
:10CB4000069204F055FC2649234B01EBC401069ADA
:10CB50001B68FAF75BF804F065FEDDF81CC0214B9A
:10CB6000214A1B5D01995843202390FBF3F0731970
:10CB70001B1A8B521D4B40424CF803601C4B013476
:10CB80004CF803501B4B032C4CF80300029B03F1A1
:10CB9000010302937FF4C3AE09B0BDE8F08F00BF7C
:10CBA000C4110020841A0020903000206E2E002036
:10CBB000D082010800002041F0260020F0D8FFFFBD
:10CBC000902900200011002080C1FFFF182A0020BA
:10CBD00084290020742900208C290020202700208F
:10CBE000C02900202C2A0020D8290020E02900207C
:10CBF000EC290020F82900202DE9F04F89B0059399
:10CC00009D4B80461B880C469B0702924DD540F2F7
:10CC1000E631129B994AD889B2F900301B1A03F207
:10CC2000F3158D4203D8002BB8BF5B4201E04FF4EF
:10CC3000FA73B2F90220101A40F2E63200F2F31150
:10CC4000914203D80028B8BF404201E04FF4FA7087
:10CC500098F84C503DB39842B8BF1846C0F5FA70EA
:10CC600004F0C6FB864904F0CBFC4FF07E5104F083
:10CC700009FB0646642090FBF5F004F0B9FB014681
:10CC8000304604F009FC4FF07E5104F0FDFA00211B
:10CC9000074604F09FFD30B938464FF07E5104F04E
:10CCA000B7FD20B101E0002701E04FF07E57E31C03
:10CCB0000393CDF800800024039B022C13F8015F3E
:10CCC000704E039309D1B6F904000A35684304F0A5
:10CCD0008FFB6D4904F094FC74E036F9140004F005
:10CCE00087FB8146029804F07FFB654904F088FCCD
:10CCF0000146484604F0D0FB644B814633F91400EA
:10CD000004F076FB0146484604F0BEFA029B8146D9
:10CD1000584204F06DFB8346484659464FEA440AA0
:10CD200004F058FD48B9029804F062FB8346484677
:10CD3000594604F06DFD00B9CB46554B33F90A0056
:10CD400004F056FB0146584604F09CFA059B8146C8
:10CD500033F9140004F04CFB0146484604F094FA01
:10CD60004C4904F04DFC8146FFF740FA28B14A4B8C
:10CD70004946185D03F0C2FC81463F4BB3F800B052
:10CD80001BF0010F05D04846D8F8441004F084FB8E
:10CD900018E036F90A001435684304F029FB3A49D3
:10CDA00004F02EFC1BF0020F05460CD0D8F84810FA
:10CDB000484604F071FB394604F06EFB01462846F4
:10CDC00004F062FA054663000493344B344E33F9A1
:10CDD000140004F00DFB334B196E04F05DFB0146AB
:10CDE000284604F04FFA009B8246196A04F054FB6F
:10CDF0002D4B0546185D04F0FBFA0146284604F069
:10CE00004BFB2A4904F0FCFB98F85120814692B173
:10CE1000022C09D1530803D09A42A8BF1A4600E059
:10CE200001224846224902E0224901EBC40133684D
:10CE3000F9F7ECFE8146336850461946019304F039
:10CE40002BFB009BDFF878B0D96A04F025FB114971
:10CE500004F022FB5BF8241004F016FA1649A50032
:10CE6000064604F0B7FC68BB3046144904F0D0FC19
:10CE700048B3124E27E000BF841A0020702F002014
:10CE80000000FA43C4110020000048429030002006
:10CE90006E2E002000002041D082010800110020E9
:10CEA0008C290020F0260020702900200000C842B4
:10CEB000842900207429002000007AC300007A43EE
:10CEC0000C2A0020444E4BF80560DFF83CB1504678
:10CED00055F80B1004F0D6F945F80BA0069001990F
:10CEE0004FF07E5004F08CFB069B0146184604F080
:10CEF000D3FA82460BF10C03EA580BF1180B1046DB
:10CF000055F80B100793069204F0BEF9514604F051
:10CF1000BBF9069A079B45F80B2098F8502001466C
:10CF200045F803A032B12D49019B01EBC401F9F78B
:10CF30006DFE014608462A4904F062FB009B996B8E
:10CF400004F0AAFA274B8246185D04F051FA014614
:10CF5000504604F0A1FA244904F052FB23498246CA
:10CF600004F038FC38B95046214904F051FC20B196
:10CF7000DFF87CA001E0DFF874A03146484604F0F9
:10CF800083F9514604F080F908F044FA194BB0F5E2
:10CF90007A7FA8BF4FF47A709842B8BF1846049AB7
:10CFA000154B0134D052484604F03CFC134B585109
:10CFB000304604F037FC124B5851504604F032FC16
:10CFC000104B032C5851009B03F1040300937FF492
:10CFD00073AE09B0BDE8F08F00007AC3C02900200D
:10CFE00000004040702900200000C842000096C3A5
:10CFF0000000964318FCFFFFD8290020E0290020FC
:10D00000EC290020F829002054270020044B00229E
:10D010001A605A60034B00221A605A60704700BFC2
:10D02000F0260020042A002010B50C4C0123E370E8
:10D030004FF48060022384F82030FAF795F9084A0B
:10D04000084BD2F888201B685278642101FB023318
:10D05000636123880133238010BD00BF4830002066
:10D06000F02600209C2E0020084BDA68D10709D456
:10D07000DA68520708D4DB6813F0100F14BF0320DE
:10D0800004207047012070470220704700200240B2
:10D09000704701207047704703788B4286BF024B70
:10D0A00033F81100002070478027002008B50021C8
:10D0B000062207F0A2FF012008BD08B500210622C4
:10D0C00007F09BFF012008BD70B50546FBF7B2F9DC
:10D0D000324CA369A061C31AB3F5FA5FE36182BF62
:10D0E000002384F8203084F8213094F820302BB9C4
:10D0F000A12D02BF294A012182F8211094F82110A4
:10D10000264A31B1D118EDB2013381F8225082F8AC
:10D11000203094F8205094F84330AB423CD11F4B60
:10D1200093F84430052B02D0062B03D02FE00020CB
:10D1300003F0D0FF94F823301E2B28D100200246A4
:10D14000C1B26B1E99421ADA214491F822300821AB
:10D15000DBB283EA0206F60744BF83F01803C3F389
:10D16000460301F1FF3154BF5B0843F0800311F027
:10D17000FF01C2F34702ECD101301A46E0E7234435
:10D1800093F822309A4202D1032003F0A3FF002338
:10D1900084F8213084F8203070BD00BF8027002043
:10D1A00010B50446B0F9000003F0ACF8B4F9020081
:10D1B00003F0A8F8B4F90400BDE8104003F0A2B8E9
:10D1C00010B50446006803F09DF8606803F09AF813
:10D1D000A068BDE8104003F095B82DE9F74F012095
:10D1E000FAF7FEFF002488B3012C2FD84FF04C092A
:10D1F00009FB04FA174E06EB0A0808F19007BD7800
:10D2000015B10134E4B2EEE790F9003090F804E093
:10D210001846114B03228DE8240001212A4653F8B9
:10D220002E30FBF774F9834660B106F14800504494
:10D2300029464A4607F0E1FE01231C44C8F848B0DD
:10D24000BB70E4B20120FAF7B1FFCCE703B0BDE850
:10D25000F08F00BF802700209C820108002122223D
:10D2600010B5104807F0C9FE0F4B002219460F48B1
:10D270000424105C013283F8F60183F8FB41052099
:10D280000024042A83F8FA0183F8FD4183F8FC01A5
:10D2900003F10803EBD10123A1F8F831522381F8FF
:10D2A000F43110BDC0130020CC110020D2A1010820
:10D2B00070B50646441E14F8011F89B1094D284671
:10D2C00007F0D1FE0028F6D005F1080398423FBFD1
:10D2D000054B401BC018A31B38BF80F88A31EAE712
:10D2E00070BD00BFD6A10108CC110020031EB8BF3D
:10D2F0002D2210B5B8BF58420C46B8BF01F8012B1B
:10D300000A22F9F7AFFD00230370204610BD07B5D0
:10D310001C4B03F1E402C3F8E0201B4A92F892216F
:10D320005AB1012A14D1032183F8E610072183F8AA
:10D33000E82083F8E7100C2208E0022183F8E610C9
:10D34000032183F8E82083F8E710072283F8E4201C
:10D350000E4A0F4B40201A60FAF742FF70B10122CB
:10D36000002390F9000040218DE80C00094A4FF499
:10D37000E133FBF7CCF8003018BF012003B05DF8B3
:10D3800004FB00BF80270020CC1100208D0E010877
:10D3900028000020410F01080120002102F09AB965
:10D3A000174AF0B5164692F8E930D2F8ECE0032BB4
:10D3B00010D85C1C0EEBC3039D1CE4B208D09A8805
:10D3C000D10705D5104203D008E00131042907D167
:10D3D0002346ECE786F8E9300020F0BD9F78002175
:10D3E0000C2202FB01F3064D05F1F00C1CF80320A2
:10D3F0009742EAD12B4485F8E940D3F8F400F0BD18
:10D40000802700208A6810B50C6A036814430A69F3
:10D4100023F4FF4314434A6923F0700314438A69D9
:10D420001443CA6914434A6A14438A6A2243134361
:10D430000360CB6843600B6883604B68C36010BDBA
:10D440004FF6FE73026813400360002303604360DD
:10D450008360C360284B984201D1284A27E0284BBB
:10D46000984201D1254A2AE0264B984201D1234A0D
:10D470002DE0254B984201D1204A30E0234B9842C1
:10D4800001D11E4A33E0224B984204D11B4A536813
:10D4900043F470032EE01F4B984204D1174A53689F
:10D4A00043F0706326E01C4B984204D11B4A53683A
:10D4B00043F00F031EE01A4B984204D1174A5368F9
:10D4C00043F0F00316E0174B984204D1134A536817
:10D4D00043F470630EE0144B984204D10F4A536832
:10D4E00043F4704306E0114B984204D10B4A536851
:10D4F00043F470235360704708000240000002406C
:10D500001C0002403000024044000240580002402B
:10D510006C00024080000240080402400004024007
:10D520001C040240300402404404024058040240FB
:10D53000224A10B5536803F00C03042B03D0082BC8
:10D5400004D01F4B14E01F4B5B6811E05368516817
:10D55000C3F38343C90303F1020301D41A4906E06C
:10D56000516811F4003F1749496818BF49084B43F7
:10D5700003605368154CC3F30313234493F820103E
:10D580000368CB4043605168C1F30221214491F804
:10D59000201023FA01F181605168C1F3C2212144B6
:10D5A00091F82010CB40C3605268C2F3813222440C
:10D5B00092F83020B3FBF2F3036110BD001002407B
:10D5C00000127A002800002000093D009C8201081A
:10D5D00010B50446FFF748FD012806D11CB1FFF73E
:10D5E00043FD013CF8E7052010BD002C08BF0520D5
:10D5F00010BD0A88F0B54B888E88B1F808E0CC8859
:10D60000002A3AD1028C43F0010322F001021204F5
:10D61000120C0284058B078CADB225F0F30545EAA8
:10D620000E1189B241EA06027A49BFB2884212D08D
:10D6300001F5006188420ED0B0F1804F0BD0A1F50A
:10D640009831884207D001F58061884203D001F506
:10D650008061884202D127F0020701E027F00A0723
:10D660001F4302830784038B23F00C031B041B0C52
:10D670000383038B9BB21C4344E0042A44D1028CF5
:10D6800022F010021204120C0284018B058C21F48A
:10D6900040721205120D42EA0E325E4992B242EA1F
:10D6A00006228842ADB292B212D001F500618842E2
:10D6B0000ED0B0F1804F0BD0A1F59831884207D041
:10D6C00001F58061884203D001F58061884207D16D
:10D6D00025F0200141EA03139BB243F0100304E05C
:10D6E00025F0A00143F010030B4302830384038B56
:10D6F00023F440631B041B0C0383038B9BB243EA9C
:10D700000424A4B20483F0BD082A028C3ED122F482
:10D7100080721204120C0284828B3E4D92B222F06F
:10D72000F307018C47EA0E1292B2A84289B242EA8C
:10D73000060212D005F50065A8420ED0B0F1804F68
:10D740000BD0A5F59835A84207D005F58065A8420D
:10D7500003D005F58065A84207D121F4007141EAA4
:10D7600003239BB243F4807304E021F4206143F46B
:10D7700080730B4382830384838B23F00C031B048D
:10D780001B0C8383838B9BB21C4341E022F48052A9
:10D790001204120C0284858B018C25F440752D0532
:10D7A0002D0D45EA062545EA0E321A4D89B2A842EA
:10D7B00092B212D005F50065A8420ED0B0F1804FAC
:10D7C0000BD0A5F59835A84207D005F58065A8428D
:10D7D00003D005F58065A84207D121F4005141EA44
:10D7E00003339BB243F4805305E047F6FF5543F4FF
:10D7F00080530D402B4382830384838B23F4406347
:10D800001B041B0C8383838B9BB243EA0424A4B2C6
:10D810008483F0BD002C0140CA78F0B5D40648BF1F
:10D820008C780D8802F00F0348BF234315F0FF0FDB
:10D830001DD0016800240126A64006EA0507B7426C
:10D8400011D14FEA840E0F2606FA0EF621EA0601E0
:10D85000282A03FA0EF641EA060101D1476102E0E7
:10D86000482A08BF07610134082CE4D10160FF2D6C
:10D870001FD94168002404F108070126BE4006EACA
:10D880000507B74211D14FEA840E0F2606FA0EF6AD
:10D8900021EA0601282A03FA0EF641EA060101D11F
:10D8A000476102E0482A08BF07610134082CE2D131
:10D8B0004160F0BD0F4B1A6842F001021A605968CE
:10D8C0000D4A0A405A601A6822F0847222F48032AB
:10D8D0001A601A6822F480221A605A6822F4FE0242
:10D8E0005A604FF41F029A60044B4FF000629A6036
:10D8F000704700BF001002400000FFF800ED00E09C
:10D900002DE9F8435B4C0368013AC4F82031838861
:10D910000D46A4F82431072A42D8DFE802F0040AB1
:10D92000101822292F35B4F820310B80B4F8223199
:10D9300013E0B4F822310B80B4F8203105E0B4F8DC
:10D9400020315B420B80B4F822315B4205E0B4F831
:10D9500022315B420B80B4F820316B80B4F8243163
:10D960001DE0B4F820315B420B80B4F8223112E0A4
:10D97000B4F822310B80B4F820310CE0B4F8203137
:10D980000B80B4F8223105E0B4F822315B420B8001
:10D99000B4F820315B426B80B4F824315B42AB8039
:10D9A000354B1B7A002B62D1B5F9000003F020FD46
:10D9B0008046B5F9020003F01BFD0746B5F90400E7
:10D9C00003F016FDD4F828110646404603F064FD26
:10D9D000D4F834118146384603F05EFD01464846CE
:10D9E00003F052FCD4F840118146304603F054FD58
:10D9F0000146484603F048FC07F00CFDD4F82C1112
:10DA00002880404603F048FDD4F838118146384656
:10DA100003F042FD0146484603F036FCD4F84411B9
:10DA20008146304603F038FD0146484603F02CFCA1
:10DA300007F0F0FCD4F830116880404603F02CFD6C
:10DA4000D4F83C118046384603F026FD0146404696
:10DA500003F01AFCD4F848110746304603F01CFDC9
:10DA60000146384603F010FC07F0D4FCA880BDE85E
:10DA7000F88300BF802700202800002044F6FB71B7
:10DA8000084B1A68137803EB431300FB0313507819
:10DA9000C0EB0030B3FBF0F39078B3FBF0F080B252
:10DAA000704700BFA819002008B50A480A2290F85C
:10DAB0004D3100EB4303B3F85C1100F5B47089B24B
:10DAC00020F8041C00F03DFC80B2FFF7D7FF024BAA
:10DAD000188008BD80270020AC1900202DE9F04FE8
:10DAE00089B00593A04B80461B880492980737D5D0
:10DAF00040F2E632129B9D48DC89B0F900301B1BD6
:10DB000003F2F315954203D8002BB8BF5B4201E046
:10DB10004FF4FA73B0F9022040F2E630121B02F221
:10DB2000F314844203D8002AB8BF524201E04FF4F4
:10DB3000FA729342B8BF13460522C3F5FA7393FBFA
:10DB4000F2F30A22643B534398F81C20D21053434B
:10DB5000642293FBF2F3134423EAE373DBB200E0A5
:10DB60006423C1460193CB1C03930024039B022C26
:10DB700013F8016F7E4F03934FEA440A05D1B7F9BA
:10DB800004301B365E4376114AE07A4B37F9142095
:10DB900033F9143003EB4202049B5B429A4203DBED
:10DBA000049B9342A8BF1346734A32F90A50059A60
:10DBB0005B1B32F9145003EB050BFEF717FB88B122
:10DBC0006E4A5846155D03F013FC6D4903F018FDCD
:10DBD0000146284602F092FD694903F05DFC03F01E
:10DBE00021FE8346604A1288D10714D437F90A50BF
:10DBF0001B366E4393074FEA261611D598F812503C
:10DC00009DF9042005FB0BF35343642293FBF2F3CD
:10DC100006EB231604E098F8085005FB0BF52E11CF
:10DC2000584B042533F90A30574F93FBF5F5751B14
:10DC300099F80160E35D6E435E430293642396FBB3
:10DC4000F3F698F851B0F611BBF1000F1BD0022C7F
:10DC500030460CD103F0CCFB5FEA5B0304D05B459C
:10DC6000A8BF5B461A4600E00122484905E003F0E0
:10DC7000BFFB5A46391D01EBC401FB69F8F7C6FF2B
:10DC800003F0D0FD0646424B99F80B7019883E4BC5
:10DC900001FB05F203F1200E5EF82400D21207FB0F
:10DCA00002073C4AB7F5001FA8BF4FF40017974280
:10DCB00003F12C00B8BF174650F8242040F8245038
:10DCC0004FF6FF700909B0FBF1F1AA1A4A4303F1BC
:10DCD000380103F144054EF8247051F824E055F85A
:10DCE000240045F824E098F85050921170444FEA0F
:10DCF000840C7F13104441F824208DB1CDF818C056
:10DD0000079303F075FB079B2A4603F1500101EBD3
:10DD1000C401DB69F8F77AFF03F084FDDDF818C071
:10DD200099F81530F2195843029B013443431846C1
:10DD3000642390FBF3F0184B0012024423F80A20EE
:10DD400003F108024CF80260032C03F1140203F102
:10DD500020034CF802704CF8030009F101097FF42C
:10DD600005AF09B0BDE8F08F841A0020702F0020A5
:10DD7000C4110020903000206E2E0020D0820108B7
:10DD8000000020410011002070290020842900207B
:10DD9000DC1000200000E0FFD82900202DE9F04F22
:10DDA000054690F850008DB008910592099318B17E
:10DDB0003228A8BF322000E0012003F019FB014601
:10DDC000AA4803F01DFCAA4B04461888002808BF87
:10DDD000012003F00DFBA749069003F05DFB0190C5
:10DDE0000199204603F050FA0146019803F008FC1F
:10DDF000A14B07901B889A0724D5A049B1F90030A0
:10DE0000B1F9020083EAE37280EAE071A2EBE37207
:10DE1000A1EBE07191420C46B8BF1446B4F5E17F26
:10DE200012DA914203DD0028D8BF404203E0002B04
:10DE3000CCBF1846584203F0DBFA914903F0E0FBEF
:10DE4000064603E0002601E04FF07E564FF0000941
:10DE5000CA4603950024630004938A4B33F91400E7
:10DE600003F0C6FA884903F017FB03F0DBFC03F06C
:10DE7000BFFA864903F010FB804B029033F914007F
:10DE800003F0B6FA7C4B07461B889B077ED0014601
:10DE900003F0FAF97E4B804633F9140003F0A8FA38
:10DEA0000146404603F0F0F903F0BCFC059B5B42E1
:10DEB000984203DB059B8342A8BF0346754A049939
:10DEC000885E099A1B1A32F91400184403F090FA7C
:10DED0008046FEF78BF970B16F4B40466F4914F8DE
:10DEE000039003F08DFB0146484602F007FC6B49A6
:10DEF00003F0D2FA8046287F03F076FA684903F0EF
:10DF0000CBFA8246287A03F06FFA0146404603F0C6
:10DF1000C3FA644903F0C0FA03F084FC81460AF1B5
:10DF2000004003F07FFC814505DB504603F07AFC9E
:10DF30004845A8BF484603F05BFADFF88C91019989
:10DF40008246404603F0A8FA59F8241003F09CF9E1
:10DF500055494FEA840B804603F03CFC38B94046F3
:10DF6000524903F055FC20B1DFF8408101E0DFF8B1
:10DF7000388149F80B80A87C03F036FA0146404608
:10DF800003F08AFA4A4903F087FA81463A4BB3F81C
:10DF900000B01BF0010F40F099803A4B049ADFF873
:10DFA0002081D35E002BB8BF5B42B3F5206F4FEAF0
:10DFB00084030A9303DD002348F824302AE03D4916
:10DFC000384603F069FA039B0B90587803F00CFA7B
:10DFD0000B9A0146104603F013FB029903F052F925
:10DFE000019903F059FA58F8241003F04DF9324919
:10DFF000804603F0EFFB38B94046304903F008FC97
:10E0000020B1DFF8B88001E0DFF8AC802C4A0A9B31
:10E0100042F80380039BD87A03F0E6F9284B53F8C3
:10E02000241003F039FA274903F036FA1BF0020FE7
:10E0300080464DD03846514603F024F9014630461B
:10E0400003F02AFA0146504603F01EF949460746F6
:10E05000404603F017F90146304603F01DFA014629
:10E06000484603F011F9804632E000BF83F9223EB2
:10E07000DC100020BD378635841A0020C411002032
:10E080000000E143001100200000A03ECDCC4C4038
:10E09000903000206E2E0020D08201080000204128
:10E0A0000000A0406F12033C0000F0C10000F041EE
:10E0B0000AD7A33D0000A043000040C30000404336
:10E0C0000C2A00200AD7233C042A0020C8465746C1
:10E0D000DFF83CB20BF1A803185D03F089F90146A3
:10E0E000029803F0D9F9894903F0D6F90146384678
:10E0F00003F0C8F895F85120034642B10BF1040132
:10E10000DBF81C3001EBC401F8F780FD0346804FBB
:10E11000029807F1AC0B5BF824100A9303F0B2F8F5
:10E12000019903F06DFA029B07F1B4024BF8243019
:10E1300052F824B00292594603F0A4F80146079819
:10E1400003F0AAF90146584603F09EF8029A834666
:10E1500042F8240007F1BC02105D03F049F90146C2
:10E16000584603F099F96B4903F096F983460A9BE8
:10E170004146184603F088F8594603F083F807F043
:10E1800049F9049B07F16802D0520A9B07F170021B
:10E190001846029203F046FB029A07F17C0342F80C
:10E1A00024004046029303F03DFB029B07F18808E0
:10E1B00043F824000BF1004003F034FB039B48F8C4
:10E1C0002400013303930CB9012444E6089A524B0E
:10E1D0009479B3F90430640028345C434F4B6411E4
:10E1E000B3F9040003F004F94FF07A5103F054F945
:10E1F00007F010F9201A03F0FBF8002CB8BF6442B6
:10E20000322C064602DD0023BB6224E0069803F0B0
:10E2100009FB20F0030003F0EBF88046687B03F075
:10E22000E3F80146304603F037F93D4904464046DD
:10E2300003F0E6F90146204603F02EF903F0F2FA66
:10E24000BB6A1844374B9842A8BF1846364B9842D1
:10E25000ACBFB862BB62BB6A6FF0FF005B13B3F583
:10E26000807FA8BF4FF480739842B8BF184603F070
:10E27000BFF88046304603F0D5FAEB78584380115A
:10E2800003F0B6F897F8BF300446032B11D9B5F860
:10E290004E60B6F5FA7F0CD203F0C4FA734298428E
:10E2A00003DBB0420346A8BF3346184603F0A0F88C
:10E2B000044695F8512062B1530803D09A42A8BF92
:10E2C0001A4600E0012220461849FB69F8F79EFC37
:10E2D00004464146204602F0D7FF03F0A3FA00B2FD
:10E2E00003F086F807F096F8A7F86C00204603F0D4
:10E2F00099FAB867404603F095FA0023C7F88400FE
:10E30000C7F890300DB0BDE8F08F00BFA69B443B2E
:10E3100070290020F7CC9238C41100200011002091
:10E3200000803B45FEFFFF0F020000F08429002023
:10E3300003689B68184703685B68184703681B6895
:10E340001847B0F902302DE9F74F93421CBF002364
:10E35000037090F800A004460E469146BAF1000FF3
:10E3600040F0AB80104603F043F8864903F094F880
:10E37000854903F091F84FF07C5103F08DF807F0D8
:10E38000A9F80146054603F087F8804983462846E8
:10E3900003F082F8034658461946019302F074FFD1
:10E3A0004FF07E5102F070FF01464FF07E5003F0B7
:10E3B00027F92946804603F06FF8294603F06CF8E8
:10E3C00007460146606002F05FFFE7604FF07E574E
:10E3D0002946A0602761284602F056FF294603F02F
:10E3E0005BF84FF0804102F04DFF0146404603F0DC
:10E3F00053F8019B60611946584602F043FF3946C5
:10E4000002F042FF0146404603F046F840F2DC537A
:10E41000A0462746554663651023A4F852301823BA
:10E42000A061A4F850304FF09741D8F8100003F0E5
:10E4300033F80021824603F0CDF928B150464FF061
:10E440007C5102F01FFF04E050464FF07C5102F077
:10E450001BFF03F049FAC7E90E014FF09741D8F8C6
:10E46000040003F019F80021824603F0B3F928B143
:10E4700050464FF07C5102F005FF04E050464FF04B
:10E480007C5102F001FF03F02FFA0135032DC7E99B
:10E49000080108F1040807F10807C4D1A6F2DC530B
:10E4A0001B042367E3676367C4F88030A367C4F87D
:10E4B00084300123A4F802902370D4F85490B4F966
:10E4C0005280C9EB0606636A06FA08F67343276AA8
:10E4D0004FEAE67B206F07FB0B332667A7FB066737
:10E4E000E26F1F44636CD4F840C053434FEAE27BB1
:10E4F0000CFB0B3ED4F88010C4F88020ACFB022348
:10E500007344B61A67EB0307E36AA26A43434FEA10
:10E51000E07B02FB0B3EA2FB00237344B6185F4175
:10E52000E36C656F4B436067A06C4FEAE17B00FBD7
:10E530000B33C4F88410A0FB01011944636B361A35
:10E5400005FB03F3206B4FEAE57B00FB0B3367EB26
:10E550000107A0FB0501801919447941B4F9502045
:10E56000A56702F07DFE08F1FF3201239340E067CA
:10E57000C01841EBE371424602F072FE484403B01A
:10E58000BDE8F08F6F12833ADB0F4940F404B53FCA
:10E590002DE9F8430024254BE0B293F8BF60B04268
:10E5A0000DD203EB8003224AD3F8C03032F81010AA
:10E5B0001BB10B2801D8DB6898470134EBE71D4BF2
:10E5C0001B685B032FD500242346E2B2B2422AD255
:10E5D000DFF858904FEA840809F1C00757F8242063
:10E5E00055689D4217D02846FBF7ECFAEFF31283EB
:10E5F000502282F312882821AA8C01FB009092B24B
:10E600000132C0F81421AA8ADBB292B242F00102B0
:10E61000AA8283F3118857F8083000221B6801345E
:10E620001A802B46D1E7BDE8F88300BF702900208F
:10E6300020110020782E002008B50E4B1B6813F423
:10E64000805F0D4B14BFD3F89021D3F8942193F839
:10E65000BF1092880023D8B2884204D2074820F81D
:10E6600013200133F7E7FFF793FFBDE8084032209E
:10E67000F9F707BF782E0020702900202011002014
:10E680000A4B30B51A680A4B02F48052D3F8904115
:10E69000D3F8945100230AB1A18800E0A988054865
:10E6A00020F8131001330C2BF5D130BD782E00204B
:10E6B000702900205A2C002070B5124D00242146EC
:10E6C00005F29910702285F8984106F096FC2146D3
:10E6D000D5F80C320B4A0B4493F9020088B11E683E
:10E6E00002F299140E5108199C88073184809B7995
:10E6F0007029837192F8983103F1010382F89831FF
:10E70000E6D170BD70290020094B1A680E2303FB67
:10E710000020437AFF2B07D0064A12789A4203D989
:10E72000054A32F8130000E0808800B2704700BF4D
:10E73000601D002064280020702F00202DE9F74F75
:10E74000304C0546D4F810723846F8F72BFD0646D3
:10E750003846F8F7B4FCD4F8147281463846F8F716
:10E7600021FD01903846F8F7AAFCD5F804A0074629
:10E770003146504602F090FED5F80880834649465F
:10E78000404602F089FE0146584602F07BFD019B9F
:10E7900029688346184602F07FFE494605465046E2
:10E7A00002F07AFE394602F077FE0146284602F072
:10E7B0006BFD39460546404602F06EFE314602F0DA
:10E7C0006BFE0146284602F05FFD0146584606F002
:10E7D000F9FE0D4902F060FE0C4902F011FFD4F879
:10E7E000181202F051FD0A4902F00AFF06F012FE6B
:10E7F00083B21A0444BF00F5B47083B218B203B0F8
:10E80000BDE8F08F702900200000E144DB0F494093
:10E810000000204101380A4B042804D8DFE800F04A
:10E820000507090B0D00074A08E0074A06E0074AFA
:10E8300004E0074A02E0074A00E0074A1A6070470E
:10E8400040000020DDC80008DDDA0008F9CB000830
:10E85000A3C5000811C200089DDD000810B54B8853
:10E86000DC0641BF2F4B14791B6853F8244044BF8A
:10E870002D4B43F820404B889B0641BF294B5479D0
:10E880001B6853F8244044BF274B43F820404B8873
:10E890001C070ED5254B0C781B78B3EB141FA1BFBA
:10E8A000204BD4781B6853F82440A4BF1E4B43F878
:10E8B00020404B889B070ED51D4B0C781B78B3EB83
:10E8C000141FDFBF174B54781B6853F82440DCBF7C
:10E8D000154B43F820404B88DC070FD5154C0B78BF
:10E8E000247803F00F03A342DFBF0E4B14781B689C
:10E8F00053F82440DCBF0C4B43F820404B885B07A7
:10E900000FD50B780C4903F00F0309788B42A1BF98
:10E91000044B92781B6853F82220A4BF024B43F8A3
:10E92000202010BD581D00201A0900207B21002046
:10E9300079210020782100207A210020254A002317
:10E94000F0B515681C461A462348244903700B701D
:10E950002E1976884EB92F5D3FB9037000230A70D7
:10E960004B7007781C461A460CE0360548BF01324A
:10E9700004F1040403F1010348BFD2B2802CDBB2DE
:10E98000E6D1EAE7E0B2B8420CD215F8240001342F
:10E9900006099E4200F00F00A8BF731C9042A8BF5A
:10E9A000421CEFE78A704B70C2F3470102F001028C
:10E9B0000A444C1E0A490B480A70C3F3470203F08D
:10E9C0000103134404700849501E084A087013706C
:10E9D000F0BD00BF5C1D0020702100208C2B0020AA
:10E9E0007A210020782100207B210020792100203D
:10E9F000924B2DE9F04FDA68914D1A612A6891B077
:10EA0000DA60904A0295136843F0200313608E4B3E
:10EA10001A78012A0CBF002201221A708B4B1A7837
:10EA2000910740F14D838A490978042940F24883CF
:10EA30008849097801F0040101F0FF0011B922F0C2
:10EA400001021A701B78DB0702D408B1FAF7A0FFA5
:10EA50008149CA78531C052293FBF2F202EB820231
:10EA60009A1A7E4BCA701F7892000023DFF810823A
:10EA7000DFF8109258F82310794C91FBF9FE04F15D
:10EA8000080040F823E0774844F8231000FB0E11FB
:10EA900042F2107091FBF0F004F1100680B226F8FB
:10EAA00013004FF0140C04F114060CFB036C04F17A
:10EAB0003C0A5AF823605CF802504CF80210761BAE
:10EAC000314405264AF8231091FBF6F109FB0E119B
:10EAD0004434012F44F823104FEA830B444605D1F8
:10EAE0000238B0F5797F98BF4BF808100BB90123B5
:10EAF000BCE7594E029BB2461868336DC01A02F04B
:10EB000073FC594902F07CFD029B4FF07E511B685B
:10EB10000746336502F05EFE08B94FF07E574B4B57
:10EB2000CAF854701B78514E13F00103504D12D0A7
:10EB30000DAA00924F4B0EAA01920CCB94E8030051
:10EB4000FAF73CFE0D9A6421B2FBF1F20E9B328083
:10EB500093FBF1F300E033802B809AF858303E4D60
:10EB6000002B35D0696D4FF07E5002F049FD07460D
:10EB7000EB6D2068C01A02F03BFC394602F08CFCB9
:10EB800002F050FE2B6E86B2606836B2C01A02F0F8
:10EB90002FFC394B196802F07FFC394602F07CFCEF
:10EBA00002F040FEB5F9662000B28118B5F9642084
:10EBB0000220B31891FBF0F193FBF0F389B29BB202
:10EBC000A5F86A10A5F86830A5F86610A5F86430B5
:10EBD00001238AF85830294B61681B88206803F0AC
:10EBE00030031D4E264DCAF86010CAF85C00002B99
:10EBF00000F0668206F17403009306F17803019336
:10EC0000F26E336FFAF7DAFD6B68306FC01A02F0FC
:10EC1000EFFB194B196802F03FFC02F003FEF36EA4
:10EC20002A68C6F880009B1AF3670C4B1B78012BEF
:10EC30002AD0022B00F0E68042E200BF440200200E
:10EC40009C2E0020BC1900204A110020C019002071
:10EC5000C6190020973000208C2B0020DC0F0020EC
:10EC6000902B0020806967FF00007A443A1A002048
:10EC70003C1A00204C11002034000020841A00208F
:10EC8000C819002080969800D6F88430D6F8A040A5
:10EC90000293D6F8943004F100400393D6F89830EC
:10ECA000776D059302F0BEFD8146204602F0BAFD65
:10ECB000D6F89C30BB4C0493BB4B06901B684FF0BE
:10ECC000000B0793B94E4FEA4B0356F82B80A6F181
:10ECD0001402404632F81B50089302F089FB029957
:10ECE00002F0DAFB02F09EFD401B1FFA80FA283684
:10ECF00026F81BA00FFA8AFA504602F079FB039916
:10ED000002F0CAFB02F08EFD86B20AEB080002F0A8
:10ED10006FFB059902F0C0FB394602F0BDFB21688C
:10ED200002F0B2FA02F07EFD484504DB069B9842F1
:10ED3000A8BF184600E0484602F05AFB206002F0E7
:10ED400071FD079B304486B2987802F04DFB9849DC
:10ED500002F0A2FB01464FF07E5002F051FC394612
:10ED600002F092FA0146384602F04AFC09906068C7
:10ED7000D4F808A0C0EB080002F03AFB394602F0D4
:10ED80003FFC514602F07EFA099A0146104602F015
:10ED900083FB0146504602F077FA3135ADB2622D61
:10EDA00001462061C4F80480A0600ED9049802F0E6
:10EDB00073FB02F037FD7F4AB0F5FA6FA8BF4FF43E
:10EDC000FA609042B8BF104600E0002040F6B8322A
:10EDD000064436B29642A8BF1646774A089B96422A
:10EDE000B8BF1646754A54F8140B9E52142202FB03
:10EDF0000BF273495050BBF1000F40F061814FF0AE
:10EE0000010B5FE7684BB6F8A8401F68736F3D8938
:10EE100002935B089D4228BF1D4623B29D4202DC3F
:10EE20001FFA85F90AE06749706D02F035FB02F0C0
:10EE3000F9FC20441FFA80F9A6F8A890DAF8786067
:10EE4000DAF8AC40341B2046FAF7FAFC41F293138F
:10EE50000028D8BF40429842CCBF0020012078B3A0
:10EE6000204602F0C5FA584902F016FBF8F727F9D8
:10EE70000446029802F0B8FA0146204602F00CFB64
:10EE800002F0D0FC40F6B83380B2AAF8B00000B26D
:10EE90009842A8BF1846484B9842ACBF3018F018AB
:10EEA00048F6A043984203DDA0F50C40A03804E0EA
:10EEB0000028BCBF00F50C40A030CAF8B40001E047
:10EEC000CAF8B460DAF8B4300026C3F50C50283024
:10EED000039302F08DFA3C4902F0DEFA0446F8F79B
:10EEE00061F90F902046F8F7EAF8DAF8B830DAF866
:10EEF000C4400593DAF8BC300E9004F1004008934A
:10EF000002F090FC0490204602F08CFCDAF8C0304D
:10EF1000DAF854802A4C09900793730048460A9304
:10EF200002F066FA0EAB53F8261002F0B5FADFF8DD
:10EF3000A0A005463AF9160002F05AFA0146284602
:10EF400002F0A0F902F06EFC05B2204BB5F57A7F15
:10EF5000A8BF4FF47A759D42B8BF1D460AF13C0A1E
:10EF6000A8B22AF8160000B202F042FA05998246C9
:10EF700002F092FA02F056FC089983B250460693CA
:10EF800002F08AFA414602F087FA216802F07CF921
:10EF900002F048FC049B98421CDB099B9842A8BFE6
:10EFA000184618E018100020E00F0020082C002060
:10EFB000DB0FC94030F8FFFF48F4FFFFEA0F0020E5
:10EFC000401000200000C842D302373918FCFFFF70
:10EFD000F42B0020049802F00BFA20608346B878E6
:10EFE00002F002FA384902F057FA01464FF07E501B
:10EFF00002F006FB414602F047F90146404602F0A6
:10F00000FFFA0B906068D4F808A0281A02F0F0F913
:10F01000414602F0F5FA514602F034F9DDF82CC011
:10F020000146604602F038FA0146504602F02CF9DB
:10F03000656001462061A060079802F02DFA02F099
:10F04000F1FB069B1434034458469A4602F0EAFB4F
:10F0500040F6B832504400B29042A8BF10461B4A56
:10F060000A9B9042B8BF1046194A1A499852142276
:10F07000724342F801B00EB901264EE73B792BB13D
:10F08000039A642392FBF3F3134A13803B88029A9A
:10F09000124C9A420DD9D4F8AC30A06FC01AFAF7CE
:10F0A000CFFB42F2107380EAE072A2EBE0729A4268
:10F0B00006DD0B4B01221A70B4F8C820064B1A80EB
:10F0C00011B0BDE8F08F00BFDB0FC94048F4FFFF6F
:10F0D000EA0F002018100020D80F00208C2B0020F1
:10F0E000DC0F0020F0B5974D87B02B78023B082B42
:10F0F00000F29581DFE813F009002E004E00630056
:10F100007B008D0009016E0179018F4B8F4C1A68CD
:10F11000636864339A4240F2828100268C4B8D4AA8
:10F120001B789E420ADA2368884FD05C30B101F028
:10F1300039F83B68013601333B60EFE72168834BC8
:10F14000525C002A40F06B811A604FF0FF325A6027
:10F15000032354E1262300937F4B492003F10C0243
:10F16000019302925021A3F10A020233F9F7D2FE71
:10F17000002840F05481794B4FF0FF311B6813F0A9
:10F180008002724B03D083E80300042337E11A6046
:10F1900059602AE0724A02230021009301910291F2
:10F1A000482002F10803F9F7B5FE002840F0378146
:10F1B000664B4FF0FF3218605A6005231FE10723AA
:10F1C0000093684B472003F10C0201930292002147
:10F1D000A3F108020433F9F79DFE002840F01F81D7
:10F1E0005A4B4FF0FF3218605A60062307E15E4A1F
:10F1F00005230021009301910291532002F108039D
:10F20000F9F788FE002840F00A81504B1860072368
:10F21000F5E04E4C236813B96360012323604C4B27
:10F220001A7863681344402BA8BF4023132B6360F4
:10F2300040F3F580454B1B680D2B00F2E780DFE8BB
:10F2400003F060070B0E121923282D3134404B5167
:10F25000464800F085FF51E0454846493FE04648B2
:10F260004649474A48E0474B474893F8D61793F832
:10F27000D72741E0434B0C2193F8B027434801FBCB
:10F28000023393F8B2172AE03E4B4148B3F84411D9
:10F2900025E03C4B3F48B3F8461120E03E4B3F4849
:10F2A00019691CE03E483F4B18E03F4B1B68D804EF
:10F2B00004D5344B3D4893F87C1110E00C232360B7
:10F2C0001FE0304B3A4893F8801193F8812193F86E
:10F2D0007F3100F055FF11E03648374B198800F0B8
:10F2E0004FFF0BE01D4B1B6819050AD5254B334812
:10F2F000B3F88411B3F9822100F042FF6368181A51
:10F30000606023680133236089E02D4B1B689A01FC
:10F3100014D52C4B1B888BB92B4B0E201B6804A9D2
:10F3200004932A4B1B680593F9F7D8FA284B4FF43E
:10F3300080521A8009232B70F9F74AFBF9F7B0FACB
:10F340006DE000BF9C2C00209C2E00205C2E002035
:10F350004C000020D48201083E830108782E002052
:10F36000FC8401081485010860850108EBA10108EF
:10F3700008A20108E697010820A20108D197010818
:10F38000DD970108CC11002037A201084BA201082B
:10F3900058A201086AA20108402700207CA20108A7
:10F3A0008FA2010816000020442E00209CA2010814
:10F3B000ACA20108C8A20108402E0020D6A2010874
:10F3C000E0100020502E00204C2E00207C30002029
:10F3D000642E0020134B1B78002BADD0124B1B6802
:10F3E0009B01A9D408232B70A8E7104B1A68104B77
:10F3F0005B68C8339A4204D900F08AFE01232B705F
:10F400000DE000F09FFE0028F6D108E000F09AFE23
:10F4100028B1084B4FF480521A800923EFE707B058
:10F42000F0BD00BF482E0020E01000209C2E0020E0
:10F430005C2E0020642E002007B5064B0649009381
:10F44000064B074A01930748074BF7F70AFE03B03C
:10F450005DF804FBDD97010816A40108E697010892
:10F4600020A40108F6A30108D197010808B5037884
:10F4700033B90C4B0C481978BDE80840F7F7F1BDDB
:10F4800005F054FE02280CD8064B0C221870074BCE
:10F4900002FB0030064B02301860F8F74DF80548C3
:10F4A000E5E708BD582C002027A401087C1900209E
:10F4B000441100209897010808B503783BB90B4B1D
:10F4C0000B4893F8B017BDE80840F7F7CABD05F040
:10F4D0002DFE022808D8054B83F8B007F7F786FF02
:10F4E000F8F74EF80348E8E708BD00BFCC1100204C
:10F4F0002BA401089897010838B5037803BB214B6A
:10F500001B6801330F2B07D81F490C2202FB031283
:10F5100095681C462DBB00E01C4601340F2C01DD14
:10F52000002400E005D818490C2202FB041295685B
:10F53000BDB99C42F1D11548BDE83840F7F791BDFF
:10F5400005F0F4FD0F28044605D80F4A0C2303FBF1
:10F5500000239D682DB92146BDE838400C48F7F7D7
:10F5600080BD084B1C60F8F71BFF21462A4609485E
:10F57000F7F777FD0C235C43034B185DBDE838407B
:10F58000F8F71EBF380000208885010838A401085C
:10F590004EA4010866A4010873B5037813B9F8F7FF
:10F5A0007BFA3DE01F4901AA05F021FE0024014637
:10F5B0002646254699B134B1012C08D1084605F0FC
:10F5C000B5FD064603E0084605F0B0FD05461549C1
:10F5D000002001AA05F00BFE01340146EAE70B2DDD
:10F5E00002D911480C220BE0022C10D1A6F57A7337
:10F5F000B3F57A7F07D90D484FF47A714FF4FA6268
:10F60000F8F7C7F90CE00A4B03EB45035E80084BA3
:10F61000084803EB45032946B3F90220F7F721FD1B
:10F6200002B070BD209C0108209A0108839F010848
:10F63000582C00207DA4010838B50D4C05462368E0
:10F64000834206D1F8F7DEFC204600214C2205F06B
:10F65000D4FCE36CAB4209D12846F8F7D3FCBDE8F3
:10F660003840044800214C2205F0C7BC38BD00BF1B
:10F67000C827002014280020034B1A68D379591C8E
:10F680001344D171187A7047641A002010B5FFF73F
:10F69000F3FF84B2FFF7F0FF04EB002080B210BD4F
:10F6A00010B5FFF7F3FF0446FFF7F0FF04EB00404F
:10F6B00010BD10B50446054B21461868FEF73EFE06
:10F6C000034B1B6898796040987110BD681A002040
:10F6D000641A002038B504460D462420FFF7E9FFE0
:10F6E0004D20FFF7E6FF002C084C14BF21203E20E0
:10F6F000FFF7DFFF2368002228469A71FFF7D9FF42
:10F70000236893F84900BDE83840D2E7641A002026
:10F7100001460020DEE710B50446C0B2FFF7C9FF7E
:10F72000200ABDE81040C4E710B5044680B2FFF7D8
:10F73000F2FF200CBDE81040EDE737B58288836802
:10F74000044610060D4641BF29494FF4CC7091F88C
:10F75000B01700FB0133D10542BF26490C200978C0
:10F7600002F03F0248BF00FB0133042A12D006D842
:10F77000012A0DD0022A2FD193F900102DE0102A72
:10F780000AD0202A0AD0082A26D1B3F9001024E092
:10F79000197822E0198820E019681EE06946186887
:10F7A000F7F7FAFA01461448F7F75BFCF5B1E068A1
:10F7B00001F01EFE6946F7F7EFFA01460F48F7F72A
:10F7C00050FC206901F014FE6946F7F7E5FA01469E
:10F7D0000A48F7F746FC09E000210948F7F741FC21
:10F7E00025B10848E1682269F7F73BFC03B030BD5A
:10F7F000CC110020582C0020399B0108329B0108B5
:10F8000090A401088CA40108024B0146D869FEF7B8
:10F8100095BD00BF582C002010B5441E14F8011FE0
:10F8200021B1034BD869FEF789FDF7E710BD00BF92
:10F83000582C0020F7B52A492A4B08782A4D1C6815
:10F840002A4B05EB80001A88D0F8C010284B2948B5
:10F850001B7800914FF47A71B4FBF1F1F7F701FCDA
:10F86000254B26481968264B0026B1FBF3F1F7F724
:10F87000F8FB244B1F68F3B205EB8302D2F8D010DB
:10F88000E9B101249C403C4217D0220715D01E4A02
:10F890000B20D25C00FB0323134A1C4802EB8303BA
:10F8A000D3F8F020F7F7DDFB022C06D1184B93F8C4
:10F8B000281011B11748F7F7D4FB0136DBE71648DB
:10F8C000FFF7AAFF154B16481A88164B92B21988F3
:10F8D00040F2DC7303B0BDE8F040F7F7C2BB00BFF5
:10F8E0000C1A00209C2E002088850108AC190020ED
:10F8F0003C00002093A4010848000020D6A4010881
:10F9000040420F00BC19002044000020E6A401087A
:10F91000582C0020EEA4010836A50108DE100020B6
:10F92000F2A40108DC1000202DE9F04100248046FB
:10F9300025460F4E4146A759384605F0DFFB58B122
:10F9400039460C48F7F78DFB30190021FFF7F5FE1B
:10F950000948FFF761FF013540F6BC4314349C426F
:10F96000E7D11DB9BDE8F041044855E7BDE8F08195
:10F9700028870108A29B010836A50108779A01088B
:10F980002DE9F74F824605F07CFB054628B101289A
:10F9900019D19AF800302A2B15D15948FFF73CFFAE
:10F9A0000024584E5848A159F7F75BFB30192946F7
:10F9B000FFF7C3FE5548FFF72FFF40F6BC43143452
:10F9C0009C42EED198E050463D2105F04CFB0028CA
:10F9D00000F08D8003461D4613F8012D202AFAD031
:10F9E000441C204605F0A2FB81462046F7F73EF96D
:10F9F0000746CAEB05054FF0000B142404FB0BF47B
:10FA0000DFF8208108F5D073E6580193304605F001
:10FA100038FB8446314662465046CDF800C005F0BA
:10FA200039FBDDF800C0019B002856D1EAB26245DF
:10FA300053D11D194444D4F8AC0101F0D9FC01465E
:10FA4000384601F0DBFE002845D0D4F8B00101F0C3
:10FA5000CFFC0146384601F0C7FE00283BD0B4F881
:10FA6000A4319A0658BF4F46142202FB0B881C068D
:10FA700048BF2748D8F8A82142BF90F8B0074FF4F4
:10FA8000CC7404FB0022D80542BF22480C24007825
:10FA900003F03F0348BF04FB0022042B39460BD080
:10FAA00004D8013B012B0CD817700AE0102B05D0AD
:10FAB000202B05D0082B04D1118002E0176000E054
:10FAC000176031461448F7F7CCFA2846002103B0F6
:10FAD000BDE8F04F31E6114805E00BF1010BBBF139
:10FAE000A30F8AD10E4803B0BDE8F04F94E650460C
:10FAF00003B0BDE8F04F17E703B0BDE8F08F00BFDB
:10FB000024A5010828870108A29B010836A5010841
:10FB1000CC110020582C002039A5010844A501086B
:10FB2000779A01088885010870B50546284605F0D2
:10FB3000A8FA064658B9194B19485A79194BBDE825
:10FB4000704003EB8203D3F8581EF7F78ABA2846B1
:10FB50001549324605F09EFA60B91448FFF75CFE7D
:10FB6000134C54F8041F19B11248F7F77AFAF8E762
:10FB7000114805E00024114B53F8241019B910481E
:10FB8000BDE8704048E62846324605F083FA013465
:10FB90000028F0D1014B0B4D5C71C7E7CC11002060
:10FBA00064A5010888850108509B010870A501081B
:10FBB000E09301084C9B010836A50108E493010875
:10FBC000779A01089897010808B50748FFF724FEBF
:10FBD000064BD869F8F7E7FCFEF72EFDF7F7DCFBDC
:10FBE000034A044BDA6008BD83A50108582C0020A5
:10FBF0000400FA0500ED00E008B50548FFF70CFE2B
:10FC000000F036F8F7F7F2FBBDE80840DCE700BF8C
:10FC10008FA5010808B50448FFF7FEFDF7F7E6FBDE
:10FC2000BDE80840D0E700BFA5A501080E4B1A7833
:10FC3000692A16D140F2DC725988914211D11A79A1
:10FC4000BE2A0ED193F8D9270020EF2A0BD113F842
:10FC5000012B5040054A9342F9D1B0FA80F0400997
:10FC6000704700207047704700F80108DCFF01086A
:10FC70002DE9F74FEA4C002140F2DC72204605F0F6
:10FC8000BCF9E84B04F53A721A60E74B00221A708F
:10FC9000E64B04F2B2711960692323700323637188
:10FCA0004FF48073A3604FF41673A4F86631FA23FF
:10FCB000A4F86831BC23A4F864314FF4FA73A4F8B3
:10FCC0006E31012384F8623184F87E3184F8863104
:10FCD000052384F8273240F2DC53A4F8983140F22F
:10FCE0004C43A4F89A3140F26C73A4F89C3140F272
:10FCF0007533A4F89E3140F64303A4F8A03123469F
:10FD0000202184F86A116E2184F87C110A2184F87C
:10FD10007D112B2184F87F11212184F8801123216A
:10FD200084F881114FF4C871A4F88211032ACCBF62
:10FD30000121002102F1010283F8A21114BF1E214A
:10FD40007521122A83F8A31103F10203EED140F2C8
:10FD50007E41A4F8441140F23A71A4F8461140F2F1
:10FD60007E51A4F84C1140F2EA5140F2DC50A4F864
:10FD70004E1140F2B4514FF4FA63A4F8C831A4F81C
:10FD8000CC31A4F8D031A4F8D431052384F8E23181
:10FD9000C82301264FF47A774FF0320BA4F8E631EE
:10FDA000DFF880924FF4C8734FF01E0A1922A4F8AE
:10FDB000EA31A4F84A01A4F85011A4F8C671A4F8D5
:10FDC000CA71A4F8CE71A4F8D27184F8E46184F801
:10FDD000E56184F8E861A4F84871A4F852B184F8A8
:10FDE00095A184F8E32100920190A4F8543184F89D
:10FDF000E16184F8EE61A4F856B184F8F161FDF791
:10FE00002DFAD9F80030009A00254FF00F0E267415
:10FE1000E673A573A58183F805E0DA714FF0220E31
:10FE20002122172183F806E05A744FF00E0E532258
:10FE30005975997583F810E0DA7655210A224FF04A
:10FE4000350E4FF02808D97083F81AE02D214FF0B5
:10FE50005A0E9A7400924FF0780C642283F80BA02B
:10FE600083F80CA0597383F808E01A771D7083F8A3
:10FE7000018083F80280DD7583F804B09D731D76E0
:10FE8000DD735D7683F8098083F80AC019754FF435
:10FE9000FA71A3F84E103C2183F85110112183F818
:10FEA00050106349DFF8A8C19963D9636149C3F869
:10FEB0002CC099626049C3F830C0DFF898C159631B
:10FEC0004FF07F5A5D490198C3F820A0C3F824A0E1
:10FED000C3F848C04FF0000A4FF04B0C59649E77AE
:10FEE00083F85250C3F840A083F84CC084F8B2E7BE
:10FEF000A4F8BC074FF0410E042084F8B3E784F85F
:10FF0000B4B784F8B55784F8B95784F8BA5784F869
:10FF1000B65784F8B75784F8B85783F85C00A3F84D
:10FF20005850A3F85A50A3F856501966152183F873
:10FF3000681043494348D966434983F86480196788
:10FF4000424983F86580596783F87860FDF7B0F916
:10FF5000D9F80030009A18464FF4487183F81151CF
:10FF600083F8125183F8138183F8146183F81851D0
:10FF7000A3F8161184F8D821C82284F8D921642264
:10FF8000A4F8DA7184F8DC51A4F8DE210E2202FB19
:10FF900005326FF0170482F81941032482F81A41E0
:10FFA0006FF02F0482F81B41072482F81C416FF088
:10FFB000230482F81D41052482F81E4101355A248C
:10FFC00080F8204180F821416422FF24082D80F828
:10FFD0001F2180F822414FF0000100F10E00D5D121
:10FFE000C820A3F88A01142083F88C01A3F890217B
:10FFF0001E204FF4967283F88D01A3F89221012000
:020000040801F1
:10000000282283F8891183F88E01A3F894210B46E6
:10001000034D5A191033C02BC2F814A01CE000BFC6
:10002000CC1100201C110020582C0020441100206D
:100030008FC2F53C000060406666663F0000A0404D
:100040009A99193F8BB00108F6287C3F3D0A773F0B
:10005000CDCCCC3E00004040DAD105F52A7000211D
:10006000402204F0CAFF0023264EEA1899590433AF
:100070000868382B244CC2F8A802F5D104F50A70A0
:100080000021802204F0B9FF06F13801702204F546
:100090000A7004F0A7FFFEF751FCD9F800600023B6
:1000A0000125314604F590604FF4CC7284F8D837BE
:1000B00084F8D65784F8D75704F094FF04F5C3604A
:1000C00031464FF4CC7204F08DFF104B1B681A6858
:1000D000C4F8BE275A68C4F8C2279A68C4F8C6276D
:1000E0001A68C4F8CA275A68C4F8CE279A68022347
:1000F000C4F8D22784F8D45484F86C3603B0BDE831
:10010000F08F00BFA8940108CC11002044110020FA
:1001100038B5094B93F8D85765B9084C2068F7F7FC
:1001200071FF074B25601B78022B03D1BDE83840D7
:10013000FDF753B838BD00BFCC110020A82C00201B
:10014000A42C0020044B93F8D8371BB9034B186834
:10015000F8F726BA00207047CC110020A82C002008
:1001600038B505460446204614F8011B21B1034B5F
:100170001868FEF7E3F8F6E7401B38BDA82C00200E
:100180000FB407B504AB53F8042B054900200193C5
:10019000F6F77CFE03B05DF804EB04B0704700BFD7
:1001A0000D030108024B01461868FEF7C7B800BFEF
:1001B000A82C0020F8B5011F06460023083051F88E
:1001C000042F02F120043F2C3AD802F108040F2C2E
:1001D00006D80232032A04D9002B08BF012300E00D
:1001E00002238142EBD1012B30680ED0022B1AD0B2
:1001F000736800F0030003F003039B0043EA001060
:10020000B36803F00303184317E000F00F0040F059
:100210004000FFF7C7FFB068736800F00F0040EAC6
:100220000310C0B209E000F03F0040F08000FFF78B
:10023000B9FF3079FFF7B6FF307ABDE8F840B1E793
:1002400006F10C0734463A46002552F8043DAD004D
:1002500003F18001FF2910D903F50041B1F5803F7A
:1002600002D245F0010508E003F50003B3F1807FF9
:1002700034BF45F0020545F00305B242E5D165F013
:100280003F00C0B2FFF78EFF05F00303022B20787A
:1002900007D0032B0CD0012B13D1FFF783FF60781D
:1002A0000FE0FFF77FFF6078FFF77CFFA07808E0A2
:1002B000FFF778FF6078FFF775FFA078FFF772FF10
:1002C000E0780434FFF76EFFBC424FEAA505DBD1AE
:1002D000F8BD10B50446C0B2FFF764FFC4F30720B1
:1002E000BDE810405EE710B504467F2C06D964F0E7
:1002F0007F00C0B2FFF756FFE409F6E7E0B2BDE8C1
:1003000010404FE7430083EAE070ECE7084649E716
:100310002DE9F04F94498BB00B7813F0010F03F0E7
:10032000040200F07A81002A40F084818F48066838
:1003300016F0806640F07E81980700F16E8143F0F0
:1003400004030B708A4B8B4C1A888B4B1A802368E2
:100350001B0340F14381894B80201E70FDF720F87C
:1003600008B1FFF769F9864F3D78012D40F03681DD
:10037000844B93F8D61721B193F8D7270AB191424D
:1003800003D3012283F8D62711E096460846BEF132
:10039000000F06D090FBFEFC0EFB1C0C7046E646E0
:1003A000F5E791FBF0F192FBF0F283F8D61783F8B2
:1003B000D72793F8D8271AB1724A002182F8D817A4
:1003C00041F669017A6893F8D89702EBC2028A4233
:1003D00084BF40F2E241B2FBF1F26B498CBFD2B272
:1003E00004220A70B9F1000F1FD18020F7F7F8FE40
:1003F0008046D0B18021F7F7CFFE98F80620634BF6
:10040000022153F822303872B3F5613F0CBF02224B
:10041000002298F900008DE8060080214A46F8F78E
:1004200076F8DFF85C81F86010B900233B70D5E006
:10043000494608F11000142204F0DFFD08F13003F2
:10044000C8F8243008F1AC034E49C8F8283008F544
:100450009473C8F82C304E4B91F8940122681B8895
:100460000028A8F8A431C2F3C03318BF012391F8C3
:1004700086010593C2F3402C02F40063C2F34008E6
:10048000444A04901068C0F38002C0F3C009487960
:10049000A0F119077C427C41012814BF20460120AD
:1004A000039091F8D60791F8D71788422CBF002106
:1004B00001210691384939488A460078D1F800B0C0
:1004C00002906F1EFFB2791E132945D8DFE801F0B4
:1004D0000C0C0C0C0C0C0C0C0AACAE31333D3F1266
:1004E000121241470399A2E00299B942B4BF002415
:1004F000012430E09BF80010022913D1B91E5BF8EB
:1005000021000021CDF824C00893079201F058F98A
:1005100007AA4FF0010492E80C1008B14FF0000454
:10052000E4B218E00BEB07014C79003418BF01244A
:1005300011E041467BE023B10499481E414241410C
:1005400000E0194601F0010171E061466FE0059994
:100550006DE006996BE014B10121B9400E43142DF2
:100560001ED80135EDB2ACE797300020E010002036
:10057000BC110020782E0020DA0F0020692800200E
:100580009C2C0020CC1100204C0000209C820108F3
:10059000E4280020BC1900201C1100202F2A002074
:1005A000DAF80000254C79301921C4F8A861F7F772
:1005B000A3FE0023C4F8B031A4F8B431A4F8B631D6
:1005C000C4F8C0311E4BD4F8BC211B6884F8AC01C0
:1005D000C4F8C4310223C4F8B8212370184B194A57
:1005E0001B6892F8E2214FF47A7101FB0233164A3C
:1005F0001360164B1B681A0609D5154B1B789B0711
:1006000005D5144B1B78042B01D9062000E00520EA
:100610000BB0BDE8F04FF7F7D3BE5AB901200BB0CD
:10062000BDE8F04FF7F7EEBE494600E0114600295D
:1006300092D196E70BB0BDE8F08F00BF9C2C002054
:100640009C2E0020CC1100208C0F0020782E002042
:10065000C0190020C619002010B5154A1378590793
:1006600025D523F004031370124B1B681B0319D507
:10067000114C2378A3F10802012A0BD8FF20002196
:10068000F8F72CF90D4B1B68C4F8C431FFF75AFD7D
:100690000A2306E0012B05D90A2B03D0FFF738FD0A
:1006A000012323700420BDE81040F7F789BE10BD78
:1006B00097300020782E00209C2C00209C2E0020BB
:1006C0000C4B0D49DA684378D243C2F30222C2F1DF
:1006D0000402934002781B01DBB20A4482F8003323
:1006E00003780122580903F01F0302FA03F341F8CB
:1006F0002030704700ED00E000E100E02DE9F74F09
:10070000AE4C2378013B012B00F253816678864280
:1007100040F04F81A378022B00F04B81A84B9B5DEA
:100720007600E37023791BB1A319B3F9060007E043
:10073000E36803F10043E360A319B3F90600404204
:1007400000F056FE9F4900F05BFF2369074618033F
:100750009A4D2BD5E86801F065F88DF802006869BC
:1007600001F060F897498DF80300384600F094FED8
:1007700004F08CFE01F07CF89249ADF80000A86905
:1007800000F08AFE04F082FE01F072F88D49ADF8A7
:100790000400E86900F080FE04F078FE01F068F8DB
:1007A0006946ADF806000C20F8F798F8D4F81C80DC
:1007B00000214046814D01F003F8002860D0D5F8B3
:1007C00018803846414601F023F818B1EB68AF6154
:1007D0006B61DAE04046002101F01AF8002800F0D1
:1007E000D48095F820303BB1022B00F2CE806B6BA9
:1007F000EF61FA33AB63C8E0E968384600F042FDC8
:100800004FF07E514FF0010500F0F8FF00B90546AA
:10081000EDB28DB16C49A06A00F03EFEDFF8BC81FC
:10082000664F4146814600F0D5FF10B9C7F82890C1
:1008300007E0C7F8288004E0A06A644900F02CFEB5
:10084000A06223695D4A190311D5116BD3788DF825
:1008500000500B445A780B208DF80120DA7A694653
:100860008DF802205B7D8DF80330F8F737F801230F
:10087000226B84F82030E37813440022DA7282E09D
:100880003846414600F0A6FF00B1EF61D4F8189059
:10089000D4F81CB04846594600F0F4FC636BA56BD5
:1008A00082465D1B6FEA05084FEAD878B8F1000F61
:1008B0000BD14FF07E5100F0ABFF002865D03846D9
:1008C000594600F0A5FF00285FD0484661694FF007
:1008D000010500F09DFF00B90546EDB23DB1606A2B
:1008E000394900F0D9FD39496062E06A07E05046B5
:1008F0004FF0804100F08CFF28B1E06A324900F0EF
:10090000CBFDE06204E0606A304900F0C5FD606242
:100910002C49606A00F0C0FD00F0AAFFD4F830A0B6
:10092000E7785FFA80F9574487F80190E06A00F0B1
:100930009FFF2369C0B21B0378750ED545EA4805B1
:100940008DF800508DF80190FB7A69468DF8030010
:100950000B208DF80230F7F7C1FF94F82020174BD9
:10096000022A0DD1002283F820201D6BDA78986AC4
:100970001749154400F090FD00F07AFFE87202E09C
:10098000022283F82020F9F765F822790B4B0AB18F
:10099000104A00E0104A2644DA60B6F9060000F07A
:1009A00027FD084900F02CFE0146E06800F06AFCD3
:1009B00000E0084603B0BDE8F08F00BF682E0020BD
:1009C0008095010800002041EC51783F0AD7833F11
:1009D00000007A440000A0410000A0C16F12833AD9
:1009E0002B4BF0B52B4D1E6805F110002F782C46CF
:1009F000F3195978013501F0040101F0FF0219B132
:100A00008542F3D10020F0BD224D631B022B0ADD8D
:100A10001AB102EB82025200D2B215F8013B303B10
:100A20001A44D2B2F1E70021AC420AD919B101EB64
:100A300081014900C9B215F8013B303B1944C9B2E4
:100A4000F2E72E2F16D1013404200023257803EB82
:100A5000830377197F785B007F079BB244BF303DEB
:100A60005B1900F1FF3044BF01349BB210F0FF006E
:100A7000ECD100E0002308484143642000FB03134D
:100A80000620B3FBF0F3054800FB0230F0BD00BFC9
:100A900050000020A42E002040420F0080969800B5
:100AA00000231A4630B510498C1894F83C40BCB16C
:100AB0002E2C06D1013298B18C180444002584F8FC
:100AC0003C500A241144634391F83C10A1F13004D6
:100AD000092C9CBF303B5B180E2A03D80132E2E799
:100AE000184630BD002030BD682E00200EB40FB572
:100AF000074906AB0190074A01A80393F6F7C6F928
:100B0000019B00221A7004B05DF804EB03B070473B
:100B1000A16B0008369C01080028114AB8BF40426A
:100B200090FBF2F330B50F4C3C2504FB0300684307
:100B30000D4D90FBF2F22D682D7B25B903EB83035D
:100B400003EB830301E0C3EB031302EB830304FB1A
:100B500002020B804FF47A7392FBF3F24A8030BDAD
:100B600080969800806967FFB0190020022803D0A2
:100B7000431E584258417047064B1B681B7823B1EF
:100B8000054B1868C0F3C0407047044B1878C0F399
:100B900080007047B40E0020E01000209730002045
:100BA00010B50A4C5E280146206805D15D21FDF78D
:100BB000C5FB20683E2105E05D2903D1FDF7BEFBA2
:100BC00020683D21BDE81040FDF7B8BBB42E0020E1
:100BD00010B50446C0B2FFF7E3FFC4F30720BDE839
:100BE0001040DDE7024B5E211868FDF7A7BB00BF90
:100BF000B42E002038B50546054C5E212068FDF76F
:100C00009DFB20682946BDE83840FDF797BB00BF33
:100C1000B42E002013B5044601A90068FFF77CFF3D
:100C20001320FFF7E7FFBDF90400FFF7D1FF1B20FA
:100C3000FFF7E0FFBDF90600FFF7CAFF2320FFF72B
:100C4000D9FF2368002BB4BF53204E20FFF7C0FF0D
:100C500001A96068FFF760FF1220FFF7CBFFBDF925
:100C60000400FFF7B5FF1A20FFF7C4FFBDF9060027
:100C7000FFF7AEFF2220FFF7BDFF6368002BB4BF74
:100C800057204520FFF7A4FF02B010BD674B73B596
:100C90001878FFF76BFF664D04462B78834220D00F
:100CA000C8B1644B1B68E3B193F9000002230093C1
:100CB000614B04211B6800225B78003318BF0123BD
:100CC00001934FF41653F7F722FC5C4B186040B1C8
:100CD00001232B7005E0594E3068F7F793F9346023
:100CE0002C70574B574D1878FFF740FF2B78044670
:100CF000834218D088B1544B1B68A3B10022012451
:100D000093F9000008214FF4964300940192F7F7FD
:100D1000FEFB4E4B186028B905E04C4E3068F7F7E3
:100D200071F934602C704A4B4A4D1878FFF71EFF5A
:100D30002B78044683422E4643D0002838D0464BB9
:100D40001A68002A3DD0D37992F90000002B4FF0A9
:100D50000202424C08BF02230092002254F82330C2
:100D600001921021F7F7D3FB3D4B0546186040B3C5
:100D70003C4C94F84A30022B0BD094F89620022A6F
:100D800001D14C3405E023B1002A04F14C0418BF12
:100D90000024354B1C6044B1204600214C2204F055
:100DA0002CF90223256084F84A300123337008E0CF
:100DB0002B4E3068FEF740FC3068F7F723F93460BB
:100DC0002C702A4B2A4D1878FFF7D0FE2B7804465A
:100DD000834229D000B3274B1B682BB3264A93F9D3
:100DE00000001268032352782021002A0CBF082239
:100DF0000922009301924FF461430022F7F787FB29
:100E00001E4B186080B11E4A012313702B701D4BBE
:100E10001A681D4B1A6007E0184E3068F7F7F2F8B1
:100E2000174B34601C702C7002B070BDBC0E0020DB
:100E3000A4110020B80E0020B0190020B42E00200C
:100E4000BD0E0020D0190020541A0020441A0020A2
:100E5000C80E00205A1A0020C40E00209C820108EF
:100E60005C1A0020C8270020601A0020D40E002041
:100E7000701A0020D00E0020CC0E0020741A002022
:100E8000781A00209C2E00207C1A002003788B42C8
:100E90000AD9064B1A78064B53F8210002B14008D4
:100EA00000F5777080B270470020704768280020F6
:100EB000B82E002007299DBF024B03EB8101088E4D
:100EC00000207047B82E0020034B03EB4101B1F81E
:100ED0005000C008704700BFB82E002008B5084B6E
:100EE00003EB8101086F00F07FFA064900F0D4FAA5
:100EF000054900F0C9F900F0BBFC80B208BD00BF95
:100F0000B82E00200000203F00005C44024B03EBA1
:100F10004101B1F8B8007047B82E0020024B03EB36
:100F20004101B1F8DC007047B82E0020024B03EB02
:100F30004101B1F8DC007047B82E00200020704756
:100F400010B50446F7F776FA41F288310E4BE4B259
:100F5000D3F8F420C3F8F400821A8A42C3F8F820C8
:100F600084BF002283F8FC2093F8FC2006490F2A56
:100F7000134418BF013283F8FD4012BF81F8FC20F2
:100F8000012381F80D3110BDB82E002010B50446A4
:100F9000F7F750FA41F288310E4BD3F81021C3F81D
:100FA0001001821A8A42C3F8142184BF002283F8F8
:100FB000182193F818210749142A134418BF013245
:100FC00083F8194112BF81F81821012381F82E31CD
:100FD00010BD00BFB82E002038B50446F7F72AFA36
:100FE000274A2749D2F83031C2F83001C31AB3F585
:100FF0007A6F84BF002382F8343192F8343133B9E8
:10100000A82C3BD181F83531A1F8363106E0022B0E
:1010100002D181F8384101E0242B02D8D11881F89F
:10102000394192F8381101330231DBB249008B4269
:10103000134D82F8343118DAB5F83631E0B283EA6C
:101040000020082310F4004F4FEA400018BF80F43E
:10105000815003F1FF3318BF80F0010013F0FF034C
:1010600080B2EFD1A2F8360138BD01318B4201BF09
:10107000002385F83431012385F8353138BD00BFB0
:10108000B82E002010B50446F7F7D4F940F6AC515D
:101090000F4AD2F86031C31A8B42C4BF002382F8D2
:1010A000643192F86431D11881F8654123B90F2C6D
:1010B0000DD10749C1F860010133DBB2192B044996
:1010C00082F864310CBF0123002381F87E3110BD0A
:1010D000B82E00200022134670B5214C1118615C17
:1010E00083EA0123082113F4004F4FEA430318BF9A
:1010F00083F4815301F1FF3118BF83F0010311F034
:10110000FF019BB2EFD10132192AE6D100F1190299
:10111000A55C00F11A02A25C02EB052292B29A428F
:101120001DD1104E96F87F51CAB2AA4214D2431C68
:1011300003EB4203DBB2E25C0133E35C03EB02232B
:101140009BB24FF4AF625343074A1B1303F5487336
:1011500022F811300131E7E7012386F8803170BDB4
:10116000A2270020B82E00208027002030B5114A89
:101170004300D2F88411CC18257E15B1022D10D071
:101180000BE0022805D9032807D10B4B1B68DB04B1
:1011900001D5C88930BD888A30BD1344B3F8B80082
:1011A00030BD607E00EB800000EB800000F2EE209E
:1011B00080B230BDB82E0020782E002008B5F7F799
:1011C00039F9074B022283F88C21064AC3F88801BB
:1011D0001268C3F89821012283F8B12108BD00BF2D
:1011E000B82E00209C2E002008B5F7F723F9084BF5
:1011F000022283F88C21D3F8982100F5B71000F56E
:10120000587002F2DC52C3F88801C3F8982108BD77
:10121000B82E002042F20102034B1B681A420CBF99
:1012200001200020704700BF782E002008B5F7F796
:1012300001F9044B00F5F42000F59070C3F8B401F7
:1012400008BD00BFB82E002008B5044B1B7803F082
:101250000503052B01D1FDF7EFF9FEE77030002003
:10126000D0400B1C1141203A03D49C461341184333
:101270006346524293401843704700BF80F00040DD
:1012800002E000BF81F0004142001FBF5FEA41035E
:1012900092EA030F7FEA226C7FEA236C6AD04FEA5E
:1012A0001262D2EB1363C1BFD218414048404140A3
:1012B000B8BF5B42192B88BF704710F0004F40F455
:1012C000000020F07F4018BF404211F0004F41F471
:1012D000000121F07F4118BF494292EA030F3FD03D
:1012E000A2F1010241FA03FC10EB0C00C3F1200350
:1012F00001FA03F100F0004302D5494260EB4000DF
:10130000B0F5000F13D3B0F1807F06D340084FEA49
:10131000310102F10102FE2A51D2B1F1004F40EB3E
:10132000C25008BF20F0010040EA030070474900A6
:1013300040EB000010F4000FA2F10102EDD1B0FA71
:1013400080FCACF1080CB2EB0C0200FA0CF0AABF66
:1013500000EBC25052421843BCBFD0401843704704
:1013600092F0000F81F4000106BF80F4000001320A
:10137000013BB5E74FEA41037FEA226C18BF7FEAE1
:10138000236C21D092EA030F04D092F0000F08BF23
:101390000846704790EA010F1CBF0020704712F00A
:1013A0007F4F04D1400028BF40F00040704712F149
:1013B00000723CBF00F50000704700F0004343F0AE
:1013C000FE4040F4000070477FEA226216BF0846E4
:1013D0007FEA23630146420206BF5FEA412390EAA7
:1013E000010F40F4800070474FF0000304E000BF9D
:1013F00010F0004348BF40425FEA000C08BF70474E
:1014000043F0964301464FF000001CE050EA010211
:1014100008BF70474FF000030AE000BF50EA010226
:1014200008BF704711F0004302D5404261EB410113
:101430005FEA010C02BF84460146002043F0B64338
:1014400008BFA3F18053A3F50003BCFA8CF2083A5D
:10145000A3EBC25310DB01FA02FC634400FA02FC66
:10146000C2F12002BCF1004F20FA02F243EB02006D
:1014700008BF20F00100704702F1200201FA02FCCF
:10148000C2F1200250EA4C0021FA02F243EB0200C2
:1014900008BF20EADC7070474FF0FF0C1CEAD05206
:1014A0001EBF1CEAD15392EA0C0F93EA0C0F6FD0C7
:1014B0001A4480EA010C400218BF5FEA41211ED0A5
:1014C0004FF0006343EA501043EA5111A0FB013191
:1014D0000CF00040B1F5000F3EBF490041EAD37166
:1014E0005B0040EA010062F17F02FD2A1DD8B3F1E2
:1014F000004F40EBC25008BF20F00100704790F051
:10150000000F0CF0004C08BF49024CEA502040EAA2
:1015100051207F3AC2BFD2F1FF0340EAC250704768
:1015200040F400004FF00003013A5DDC12F1190FA6
:10153000DCBF00F000407047C2F10002410021FA18
:1015400002F1C2F1200200FA02FC5FEA310040F130
:10155000000053EA4C0308BF20EADC70704792F0A9
:10156000000F00F0004C02BF400010F4000F013AE1
:10157000F9D040EA0C0093F0000F01F0004C02BFDC
:10158000490011F4000F013BF9D041EA0C018FE74B
:101590000CEAD15392EA0C0F18BF93EA0C0F0AD051
:1015A00030F0004C18BF31F0004CD8D180EA010077
:1015B00000F00040704790F0000F17BF90F0004F10
:1015C000084691F0000F91F0004F14D092EA0C0FF2
:1015D00001D142020FD193EA0C0F03D14B0218BF85
:1015E000084608D180EA010000F0004040F0FE40CB
:1015F00040F40000704740F0FE4040F44000704767
:101600004FF0FF0C1CEAD0521EBF1CEAD15392EAE5
:101610000C0F93EA0C0F69D0A2EB030280EA010CD5
:1016200049024FEA402037D04FF0805343EA11116E
:1016300043EA10130CF000408B4238BF5B0042F1CC
:101640007D024FF4000C8B4224BF5B1A40EA0C0071
:10165000B3EB510F24BFA3EB510340EA5C00B3EBA3
:10166000910F24BFA3EB910340EA9C00B3EBD10F91
:1016700024BFA3EBD10340EADC001B0118BF5FEAE3
:101680001C1CE0D1FD2A3FF650AF8B4240EBC2500C
:1016900008BF20F0010070470CF0004C4CEA5020CD
:1016A0007F32C2BFD2F1FF0340EAC250704740F41C
:1016B00000004FF00003013A37E792F0000F00F00E
:1016C000004C02BF400010F4000F013AF9D040EA8C
:1016D0000C0093F0000F01F0004C02BF490011F420
:1016E000000F013BF9D041EA0C0195E70CEAD15318
:1016F00092EA0C0F08D142027FF47DAF93EA0C0FFF
:101700007FF470AF084676E793EA0C0F04D14B02E2
:101710003FF44CAF08466EE730F0004C18BF31F094
:10172000004CCAD130F000427FF45CAF31F000438E
:101730007FF43CAF5FE700BF4FF0FF3C06E000BF27
:101740004FF0010C02E000BF4FF0010C4DF804CD4A
:101750004FEA40024FEA41037FEA226C18BF7FEA5A
:10176000236C11D001B052EA530C18BF90EA010F5C
:1017700058BFB2EB030088BFC81738BF6FEAE170EB
:1017800018BF40F0010070477FEA226C02D15FEA87
:10179000402C05D17FEA236CE4D15FEA412CE1D0F3
:1017A0005DF8040B704700BF844608466146FFE7BA
:1017B0000FB5FFF7C9FF002848BF10F1000F0FBD9C
:1017C0004DF808EDFFF7F4FF0CBF012000205DF895
:1017D00008FB00BF4DF808EDFFF7EAFF34BF01201A
:1017E00000205DF808FB00BF4DF808EDFFF7E0FFB3
:1017F00094BF012000205DF808FB00BF4DF808ED04
:10180000FFF7D2FF94BF012000205DF808FB00BF66
:101810004DF808EDFFF7C8FF34BF012000205DF848
:1018200008FB00BF4FEA4002B2F1FE4F0FD34FF06A
:101830009E03B3EB12620DD94FEA002343F000433D
:1018400010F0004F23FA02F018BF404270474FF0EB
:101850000000704712F1610F01D1420205D110F072
:10186000004008BF6FF0004070474FF00000704725
:1018700042000ED2B2F1FE4F0BD34FF09E03B3EBFA
:10188000126209D44FEA002343F0004323FA02F026
:1018900070474FF00000704712F1610F01D1420212
:1018A00002D14FF0FF3070474FF00000704700BF8B
:1018B0007BB972B90029BEBF00204FF0004106E09D
:1018C00008BF00281CBF6FF000414FF0FF3000F050
:1018D00075B882B0EC462DE9005000F03FF8DDF815
:1018E00004E002B00CBC704710B500210446FFF7BD
:1018F00071FF20B92046BDE8104000F009B804F19E
:10190000004000F005F8404261EB410110BD00BF0E
:10191000D0B500F0B9F900220E4B06460F4600F094
:1019200007FA00F017FC044600F08CF900220A4B7D
:1019300000F0FEF902460B463046394600F044F806
:1019400000F008FC2346002242EA00021046194635
:10195000D0BD00BF0000F03D0000F0412DE9F04196
:10196000069C904606460F461D4600F013FC08FBF9
:1019700001FCA8FB002300FB05C5B21A2B4467EB52
:1019800003038646C4E90023BDE8F0812DE9F8434E
:10199000089E1746804689461D4600F051FD00FB13
:1019A00005F3A0FB074507FB0137B8EB04043D44F2
:1019B00069EB0505C6E90045BDE8F883704700BF3F
:1019C00081F0004102E000BF83F0004330B54FEAF0
:1019D00041044FEA430594EA050F08BF90EA020F5D
:1019E0001FBF54EA000C55EA020C7FEA645C7FEAF0
:1019F000655C00F0E2804FEA5454D4EB5555B8BF13
:101A00006D420CDD2C4480EA020281EA030382EA83
:101A1000000083EA010180EA020281EA0303362D15
:101A200088BF30BD11F0004F4FEA01314FF4801CE8
:101A30004CEA113102D0404261EB410113F0004FFA
:101A40004FEA03334CEA133302D0524263EB4303B1
:101A500094EA050F00F0A780A4F10104D5F1200E4F
:101A60000DDB02FA0EFC22FA05F2801841F10001AA
:101A700003FA0EF2801843FA05F359410EE0A5F17E
:101A800020050EF1200E012A03FA0EFC28BF4CF0AF
:101A9000020C43FA05F3C01851EBE37101F0004565
:101AA00007D54FF0000EDCF1000C7EEB00006EEB72
:101AB0000101B1F5801F1BD3B1F5001F0CD34908FC
:101AC0005FEA30004FEA3C0C04F101044FEA445253
:101AD00012F5800F80F09A80BCF1004F08BF5FEADA
:101AE000500C50F1000041EB045141EA050130BDBA
:101AF0005FEA4C0C404141EB010111F4801FA4F15D
:101B00000104E9D191F0000F04BF01460020B1FAB1
:101B100081F308BF2033A3F10B03B3F120020CDAE9
:101B20000C3208DD02F1140CC2F10C0201FA0CF0C7
:101B300021FA02F10CE002F11402D8BFC2F1200C2C
:101B400001FA02F120FA0CFCDCBF41EA0C019040E2
:101B5000E41AA2BF01EB0451294330BD6FEA04042B
:101B60001F3C1CDA0C340EDC04F11404C4F1200216
:101B700020FA04F001FA02F340EA030021FA04F328
:101B800045EA030130BDC4F10C04C4F1200220FA7F
:101B900002F001FA04F340EA0300294630BD21FABD
:101BA00004F0294630BD94F0000F83F4801306BF83
:101BB00081F480110134013D4EE77FEA645C18BF77
:101BC0007FEA655C29D094EA050F08BF90EA020F0E
:101BD00005D054EA000C04BF1946104630BD91EA06
:101BE000030F1EBF0021002030BD5FEA545C05D109
:101BF0004000494128BF41F0004130BD14F5800448
